:020000040800F2
:1000000000000120E5450008B5270008B7270008D3
:10001000B9270008BB270008BD2700080000000022
:10002000000000000000000000000000BF270008E2
:10003000C127000800000000C3270008C5270008EA
:100040003546000835460008C9270008354600082F
:100050003546000835460008D5270008DB2700088C
:1000600035460008354600080D28000835460008CA
:10007000E1270008E3270008E5270008F12700082A
:10008000FD27000809280008354600083546000805
:1000900000000000354600080F280008354600081B
:1000A0003546000835460008354600083546000844
:1000B0003546000835460008354600083546000834
:1000C0003546000835460008354600083546000824
:1000D0003546000815280008354600083546000852
:1000E0003546000811280008212800083546000878
:1000F00035460008000000000000000035460008FA
:1001000035460008354600082D2800083546000809
:1001100035460008354600083546000835460008D3
:1001200035460008354600083546000835460008C3
:080130003546000835460008C1
:1001380010B5054C237833B9044B13B10448AFF319
:1001480000800123237010BD5C0100200000000026
:100158001011010808B5034B1BB103490348AFF35D
:10016800008008BD00000000600100201011010897
:1001780014214160704714207047406A704700009E
:10018800790100087F01000883010008990100082F
:1001980010B5044604F1100000F05CFCC4F8F80047
:1001A8000148C4F87C0110BD88010008F8B5E6B024
:1001B80004460D4616461F460A4906A800F0CAFE20
:1001C80070996F9A05910492009733466E996D9ACB
:1001D800039102922A466C990191214600F060F839
:1001E80067B0F0BD94010008F8B5E6B004460D46C6
:1001F80016461F46094906A800F0ACFE6F996E9A8C
:100208000491039200976D996C9A0291019233467A
:100218002A46214600F087F867B0F0BD940100082F
:1002280038B500281CBF01680029184A23D1184B8B
:100238001C684FF6F0710C404CF24025AC421FBFD1
:100248001B6819404CF27024A14212D1114D296843
:1002580079B911490B68C3F30B03B3F58A6F1FBF54
:100268000968C1F30B0140F28343994204BF01219D
:10027800117028B905E0094B994204BF012111709A
:100288004068BDE8324001F09FBE00BF7801002001
:1002980000ED00E0002004E00010005C000037489A
:1002A8002DE9F04104460D46216816464A681F4666
:1002B80090478046B8F5403F2ED122680A99936846
:1002C800204698478046B8F5403F25D12368089ACC
:1002D8000799D3F80CC02046E0478046B8F5403F60
:1002E8001AD12368069A39461F692046B8478046BE
:1002F800B8F5403F10D1236829465D69324620464B
:10030800A8478046B8F5403F06D123680B9A09995B
:100318009D692046A847804621680A68204690477C
:100328004046BDE8F0812DE9F04104460D462168BC
:1003380016464A681F4690478046B8F5403F2ED17A
:1003480022680A999368204698478046B8F5403F46
:1003580025D12368089A0799D3F80CC02046E047AE
:100368008046B8F5403F1AD12368069A39461F6976
:100378002046B8478046B8F5403F10D12368294643
:100388005D6932462046A8478046B8F5403F06D109
:1003980023680999DD6900222046A847804621681C
:1003A8000A68204690474046BDE8F0814FF4403047
:1003B80070470000F0B50C4685B0114600281A4673
:1003C8001CBF0568002D0B4B11D082B104B971B95F
:1003D8000D9860B10F9E0E9F0A9B0290049603979A
:1003E8000B980C9E009001962046A8470346184695
:1003F80005B0F0BD020003002DE9F04F0646D0B06D
:100408000868F56DD6F860E0726EB76EF36E00BAE4
:1004180000906C46486800BA60600DF14008886832
:1004280000BAA060C86800BAE060086900BA206134
:10043800486900BA6061886900BAA061C86900BAF1
:10044800E061086A00BA2062486A00BA6062886A95
:1004580000BAA062C86A00BAE062086B00BA2063FA
:10046800486B00BA6063886B00BAA063C86B00BAB7
:10047800E063402058F80C1C58F820CC58F838ACE9
:100488008CEA010158F840CC8AEA01018CEA01099A
:100498004FEAF979401E48F8049BEBD187EA02003D
:1004A80000EA0E00784010EBF5610098DFF824C4EC
:1004B80041186144C81882EABE032B404FEAF06134
:1004C80053405918636859186144CF194FEAB50366
:1004D80083EABE01014081EABE0111EBF765A1681C
:1004E8004D196544A91883EAB0023A404FEAF1650C
:1004F8005A405519E26855194FEAB70282EAB0071F
:1005080065440F4005EBBE0E97EAB00717EBFE6592
:1005180027697D194FEAB10782EA0701654401EAB4
:100528000E01EB18514011EBF36561694D194FEA63
:10053800BE0187EA010E65440EEA030E15EBB00012
:100548008EEA070E0EEBF065D4F818E075446544A2
:10055800AA1881EAB30505404FEAF26E4D40AE4451
:10056800E569AE44E64477444FEAB00080EAB30E4A
:100578000EEA020E8EEAB30E0EEBF765D4F820E011
:1005880075446544691880EAB2053D404FEAF16E4A
:100598004540AE44656AAE44E6440EEBB3034FEA09
:1005A800B70787EAB20E0EEA010E8EEAB20E0EEB1C
:1005B800F365D4F828E075446544281887EAB1053E
:1005C8001D404FEAF06E7D40AE44E56AAE44E64415
:1005D8000EEBB2024FEAB30383EAB10E0EEA000E45
:1005E8008EEAB10E0EEBF265D4F830E0754465443E
:1005F800EF1983EAB00515404FEAF76E5D40AE4447
:10060800656BAE44E6440EEBB1014FEAB20282EAF2
:10061800B00E0EEA070E8EEAB00E0EEBF165D4F8B6
:1006280038E075446544EB1882EAB7050D404FEA97
:10063800F36E5540AE44E56BAE44E6440EEBB000B5
:100648004FEAB10181EAB70E0EEA030E8EEAB70E41
:100658000EEBF065D4F840E07544654481EAB30ECA
:10066800AA180EEA000E4FEAF2658EEA010E7544EA
:10067800DDF844E04FEAB000754480EAB30E654403
:100688000EEA020E15EBB7078EEAB30E0EEBF7650E
:10069800DDF848E04FEAB202754480EA020E65448C
:1006A8000EEA070E69188EEA000E0EEBF165DDF80A
:1006B8004CE07544654405EBB3034FEAB70E1427C5
:1006C8000DF1500CDFF810528EEA010B82EA0B0B89
:1006D8000BEBF36A5CF804BBDA44AA44504483EA9F
:1006E800B10B4FEAF06A8EEA0B0BDA445CF804BBF4
:1006F800DA44AA44524480EAB30B4FEAF26A8BEA1E
:10070800B10BDA445CF804BBDA444FEAB000AA44FF
:1007180080EA020BD6448BEAB30B0BEBFE6A5CF85B
:1007280004BBDA444FEAB202AA4482EA0E0B0AEB8F
:10073800B10180EA0B0B0BEBF16A5CF804BBDA44FD
:100748007F1DAA44282F0AEBB3034FEABE0EBBD382
:100758003C2F61D3502F4DD204EB870CC7F15407BF
:100768005E4CA7FB04A504465D4FA8088EEA010A63
:1007780082EA0A0A5CF804BB0AEBF3655D447D195A
:100788002C1983EAB10A4FEAF4658EEA0A0A55443D
:100798005CF804AB5CF804BB55447D19AA1884EADC
:1007A800B30A4FEAF2658AEAB10A55445D444FEA52
:1007B800B4047D1984EA020AAE448AEAB30A0AEB51
:1007C800FE655CF804AB55444FEAB2027D1982EA33
:1007D8000E0A15EBB10184EA0A0A5CF804BB0AEBBD
:1007E800F1655D447D1915EBB303401E4FEABE0E5B
:1007F800BCD12046F46D1B19F365336EC9183166F8
:10080800716E71447166B36ED218B266F16E40189B
:10081800F06650B0BDE8F08F4EEA010B0EEA010A0F
:100828000BEA020B4BEA0A0A0AEBF36554F827A015
:10083800DFF8B0C0554443EAB10B654403EAB10A96
:100848000BEA0E0B28184BEA0A0A7F1C0AEBF06524
:1008580054F827A0554440EAB30B654400EAB30AAC
:100868000BEAB10BAA184BEA0A0A7F1C0AEBF265DD
:1008780054F827A055444FEAB00040EA020B6544FB
:1008880000EA020A0BEAB30BAE444BEA0A0A7F1CE1
:100898000AEBFE6554F827A055444FEAB20242EA33
:1008A8000E0B654402EA0E0A0BEA000B15EBB101C8
:1008B8004BEA0A0A7F1C0AEBF16554F827A0554455
:1008C8007F1C65443C2F05EBB3034FEABE0EA3D350
:1008D80040E700BF9979825AA1EBD96ECDCCCCCC38
:1008E800D6C162CADCBC1B8F00B581B00168074A5B
:1008F800914200D110B9064801B000BD7C2110F02A
:100908006DFB4FF4003001B000BD00BFFC090008CA
:10091800030002002DE9F0410B4A92E8F85188B033
:10092800694681E8F8510268084B9A4200D118B923
:10093800074808B0BDE8F0811422083000F04FFBEA
:1009480008B0BDE8F08100BFDC090008FC09000818
:1009580003000200152904D20268044B9A4200D110
:1009680008B903487047083000F048BBFC09000884
:100978000300020010B481B013460268074CA2427B
:1009880000D118B901B010BC0548704701B000F19A
:10099800240210BC083000F035BB00BFFC09000879
:1009A8000300020010B481B013460268074CA2424B
:1009B80000D118B901B010BC054870470A4601B00B
:1009C80000F1240110BC083000F070BBFC090008DD
:1009D800030002000123456789ABCDEFFEDCBA981E
:1009E80076543210F0E1D2C300000000000000008D
:1009F80000000000F10800081D0900085D09000852
:100A08007D090008AD09000801040008790F0008F5
:100A1800C50F0008810F0008F0B5A3B004460B48C5
:100A280002900D4616461F46094B0822402104A88D
:100A380000F0D1FA28980190009733462A462146BB
:100A480002A800F01BF823B0F0BD00BFFC090008A5
:100A5800100A000810B5040008BF002408D0054893
:100A6800054B20600822402104F1080000F0B3FA89
:100A7800204610BDFC090008100A00082DE9F041C5
:100A880004460E46216817464A681D469047804628
:100A9800B8F5003F19D1226806999368204698470F
:100AA8008046B8F5003F10D123683146DE683A46E3
:100AB8002046B0478046B8F5003F06D12368079A1C
:100AC80029461D692046A847804621680A682046AD
:100AD80090474046BDE8F08110B500F033FA4FF476
:100AE800403400280EBF034C4FF4C07110F076FA62
:100AF800204610BD0200030010B5044600F022FA9B
:100B080008B9054810BD0021A160D0F87C21116802
:100B180088474FF4403010BD0200030070B504460A
:100B28000D4600F00FFA064E40B1D0F87C0141683E
:100B38008847A84224BF65604FF44036304670BDF0
:100B4800020003002DE9FF4715000C4600D02CB128
:100B5800064600F0F7F95FEA000801D16448C3E0EF
:100B6800D8F8F80001684A689047B0F5003F17D1F7
:100B7800D8F87C118A68404690478146B9F1810FC0
:100B880080F09E80A94508F1FC0A17D2D8F8F80031
:100B98000368D3F80CC02A462146E047B0F5003F69
:100BA80040F08E80D8F8F8000368D3F810C06A4681
:100BB8005146E047B0F5003F76D10AE0002004E056
:100BC800215C0AF800100098401C00900098A84288
:100BD800F6D34FF0000C4749474A484B01AC009800
:100BE800844558D2D3E9007001ADC5E9007010788A
:100BF80000281ABF042086464FF0000E085854F803
:100C08000E5028443E4D05600127D0F800E087606B
:100C1800019D4F681AF80C007D408EEA050585F0A5
:100C2800040E65680F687D4085F0FC05754485F005
:100C3800A30568400AF80C000CF1010CCFE7D3E9D2
:100C4800004501A8C0E9004510782E4D002814BFC2
:100C58004FF0040E4FF0000E01A8744651F80EE054
:100C68000459A6440127CEF80050DEF80040CEF81B
:100C780008704D68019F40687D406C400D68684071
:100C880084F0040480F0FC00041984F057040AF886
:100C98000C400CF1010CCC45D1D3D8F8F800016810
:100CA8004A689047B0F5003F0AD1D8F8F8000368C1
:100CB800D3F80C804A465146C047B0F5003F01D0F2
:100CC800114811E0002006E05AF8201081F06A313E
:100CD8004AF82010401CB0EB990FF5D3B06840F0EB
:100CE8000100B0604FF4403004B0BDE8F08700BFA9
:100CF800020003007C11010878010020240F00087D
:100D0800ADBE4ED70DBE75A10100030038B50C4627
:100D1800017A1546CA0702D500F014F908B908483F
:100D280032BDD0F8F80003682146DC682A46A0479F
:100D3800B0F5003F01D0034832BD4FF4403032BD1A
:100D480002000300010003002DE9F84191B00546B7
:100D58000E461746402101A810F040F9297AC80725
:100D680004D5284600F0EEF8040002D1DFF8A4808C
:100D78004BE0D4F8F800DFF8A0800368D3F810C07F
:100D88006A4601A9E047B0F5003F3ED1D4F8F80023
:100D980001684A689047B0F5003F36D1D4F87C1115
:100DA8008A6820469047D4F8F830024618461B68EF
:100DB800D3F80CC004F1FC01E047B0F5003F24D1A2
:100DC800D4F87C0141688847D4F8F83002461846C0
:100DD8001B68D3F80CC001A9E047B0F5003F14D157
:100DE800D4F8F8000268696893689847B0F5003F3E
:100DF8000BD1D4F8F80003681C693A463146A0477D
:100E0800B0F5003F08BF4FF44038404612B0BDE887
:100E1800F08100BF02000300010003002DE9F84142
:100E2800A5B0074688461646402115A810F0D6F802
:100E380000220492402105A810F0D0F8387AC107A2
:100E48005ED5384600F07EF8050059D0D5F8F80090
:100E58002D4C0368D3F810C06A4605A9E047B0F5E1
:100E6800003F3CD1D5F8F80001684A689047B0F5D2
:100E7800003F34D1D5F87C118A6828469047D5F8C8
:100E8800F830024618461B68D3F80CC005F1FC017F
:100E9800E047B0F5003F22D1D5F87C01416888478A
:100EA800D5F8F830024618461B68D3F80CC005A9D7
:100EB800E047B0F5003F12D1D5F8F800026879682C
:100EC80093689847B0F5003F09D1D5F8F800036852
:100ED8001D6904AA15A9A847B0F5003F01D020460E
:100EE8000FE00A4B0A490B4A0396029101924046C9
:100EF8001C68049B009415AA796800F0E5F900E0E5
:100F0800054826B0BDE8F0810100030084110108FE
:100F1800936E030026C703000200030004B001011A
:100F280000170145E10A0008010B0008250B00081D
:100F3800B50300084D0B0008150D0008510D0008F9
:100F4800250E00080168024A914218BF0020704728
:100F58002C0F000810B5040008BF002404D0034873
:100F68002060204609688847204610BD2C0F0008DD
:100F780020225C3010F030B8F0B58468A308002255
:100F880004F0030407E000F15C0555F8226035BA67
:100F980041F82250521C9A42F5D300220BE000F18E
:100FA8005C0502EB830755F82360D500C5F11805E9
:100FB800EE40CE55521CA242F1D3F0BD30B5C46804
:100FC80003690022E31AD5188C5C0544521C082AD0
:100FD8002C77F8D330BD0360C1600261704738B523
:100FE800044615460022626023685A68904700202C
:100FF8006061A061A5604FF4003032BD81604FF49C
:10100800003070472DE9F84304462079D4F80C8065
:10101800450748BF244845D466691D46A8F1010024
:1010280000EAD60306EBC506B6EBC50F666102D229
:10103800A669761CA6611746A66906EB5576A661D1
:101048000E46E918884225D2A8EB03094A463146DC
:10105800F8180FF0C1FF2268136839460FE04246BE
:1010680038460FF0B9FF23681A683946204690477A
:1010780007E0311811F00300F1D122681368204607
:101088009847484600EB0809A9F10101A942F0D3A5
:10109800002300E000202A1A3118F8180FF09CFFEE
:1010A8004FF40030BDE8F283040002002DE9FC4F44
:1010B800024685B0D0681369DFF86CC1DFF86C812F
:1010C800A0EB030A506840F004005060002703A812
:1010D80002900DF10C0ED8E9003403A8544DC0E974
:1010E80000342878534D00280CBF00230423994668
:1010F8005CF803305EF80940234401261D601C6833
:101108009E60DCF80430039DDCF80090DEF8046093
:101118005D406540484C654089EA0606474C664094
:101128007519474C6540D8E9006B03AC0028C4E941
:10113800006B0EBF002404200424029E5CF800000B
:10114800345920183F4C04600126046886600398CF
:10115800029E43406340384C7068634089EA00004F
:10116800364C6040034438484340280018BF0120EB
:101178005B1E9B41042F2CBFC0B2D80F02F1140391
:1011880053F8200007F00303C3F10303DB00D84042
:101198000DF807007F1C082F9DD315460C466A6979
:1011A800AB69E868D20842EA4372401E00EA0207C7
:1011B800002302409B420AD8524508D28020E055BD
:1011C8007F1C574516D2AAEB0701E01910E08020D2
:1011D800E05500E0E355E8687F1C8742FAD32A68A7
:1011E800136828469847BAF1000F03D051462046A5
:1011F8000FF0F4FE2A68069E059F93686946284604
:1012080098472A68D2F8009021462846C8472B6894
:10121800DA683946284690470EB1A86830604FF41E
:10122800003007B0BDE8F08F7C11010854120008A7
:10123800780100205FC5109304850012FC68017ACC
:10124800C0F524FF24AF33D426AF698B04B0010165
:1012580000170145F8B501240094002300240DE08F
:10126800009D065D0F5D7E40F643761CF60F86F006
:10127800010635400095641C009DEB189442EFD39D
:101288001846F2BDF8B5002301240094002A11E0A5
:10129800009C85188F1815F8016C17F8015C6E40D2
:1012A800F643761CF60F86F0010634400094009C45
:1012B800E318521EECD11846F2BD00005D1200087A
:1012C8008D120008010000002DE9F84F1D46DDF8D9
:1012D80028900B9F0D9C4FF0FF3300930E469246CB
:1012E800D9F800B0804632465146D847834664B3A1
:1012F800D9F8043032465146404698476FEA0B0207
:10130800521C42EA0B0200996FEAD2735B1C194027
:10131800C2430091521C024300996FEAD2735B1CCE
:101328001940009186F05531484087EA000181F064
:101338005531216080F05531C943491C0843009A52
:101348006FEAD070401C82430092D9F80800012847
:1013580009D17540E943491C0D4300986FEAD572DD
:10136800521C90430AE0F11C85EA9102D243521CB8
:10137800154300986FEAD5735B1C984386F0AA362C
:10138800009086EA0B0686F0AA33F243DB430C98FA
:10139800C2F3C0725B1C42EAD3720099D243521C5A
:1013A80091430091774000998843009987F0AA37C4
:1013B8000F403843BDE8F28F034613F8012B002A8B
:1013C800FBD1181A0138704781F0004102E000BFD4
:1013D80083F0004330B54FEA41044FEA430594EAED
:1013E800050F08BF90EA020F1FBF54EA000C55EA28
:1013F800020C7FEA645C7FEA655C00F0E2804FEAF9
:101408005454D4EB5555B8BF6D420CDD2C4480EADA
:10141800020281EA030382EA000083EA010180EA0A
:10142800020281EA0303362D88BF30BD11F0004F58
:101438004FEA01314FF4801C4CEA113102D040428E
:1014480061EB410113F0004F4FEA03334CEA1333C9
:1014580002D0524263EB430394EA050F00F0A780E1
:10146800A4F10104D5F1200E0DDB02FA0EFC22FADC
:1014780005F2801841F1000103FA0EF2801843FAD0
:1014880005F359410EE0A5F120050EF1200E012AC1
:1014980003FA0EFC28BF4CF0020C43FA05F3C018FF
:1014A80051EBE37101F0004507D54FF0000EDCF178
:1014B800000C7EEB00006EEB0101B1F5801F1BD321
:1014C800B1F5001F0CD349085FEA30004FEA3C0C25
:1014D80004F101044FEA445212F5800F80F09A801B
:1014E800BCF1004F08BF5FEA500C50F1000041EB1F
:1014F800045141EA050130BD5FEA4C0C404141EB23
:101508000101013C28BFB1F5801FE9D291F0000F1D
:1015180004BF01460020B1FA81F308BF2033A3F1CC
:101528000B03B3F120020CDA0C3208DD02F1140CC3
:10153800C2F10C0201FA0CF021FA02F10CE002F1FE
:101548001402D8BFC2F1200C01FA02F120FA0CFCF7
:10155800DCBF41EA0C019040E41AA2BF01EB045140
:10156800294330BD6FEA04041F3C1CDA0C340EDC3E
:1015780004F11404C4F1200220FA04F001FA02F381
:1015880040EA030021FA04F345EA030130BDC4F13F
:101598000C04C4F1200220FA02F001FA04F340EA34
:1015A8000300294630BD21FA04F0294630BD94F0E5
:1015B800000F83F4801306BF81F480110134013DCC
:1015C8004EE77FEA645C18BF7FEA655C29D094EA3D
:1015D800050F08BF90EA020F05D054EA000C04BFBB
:1015E8001946104630BD91EA030F1EBF00210020A6
:1015F80030BD5FEA545C05D14000494128BF41F045
:10160800004130BD14F580043CBF01F5801130BDA8
:1016180001F0004545F0FE4141F470014FF0000033
:1016280030BD7FEA645C1ABF194610467FEA655CE4
:101638001CBF0B46024650EA013406BF52EA033586
:1016480091EA030F41F4002130BD00BF90F0000F74
:1016580004BF0021704730B54FF4806404F13204B0
:101668004FF000054FF0000150E700BF90F0000F69
:1016780004BF0021704730B54FF4806404F1320490
:1016880010F0004548BF40424FF000013EE700BF60
:1016980042004FEAE2014FEA31014FEA02701FBFF0
:1016A80012F07F4393F07F4F81F06051704732F022
:1016B8007F4208BF704793F07F4F04BF41F4002179
:1016C800704730B54FF4607401F0004521F00041D7
:1016D8001CE700BF50EA010208BF704730B54FF061
:1016E80000050AE050EA010208BF704730B511F062
:1016F800004502D5404261EB41014FF4806404F19A
:1017080032045FEA915C3FF4D8AE4FF003025FEA1F
:10171800DC0C18BF03325FEADC0C18BF033202EBA3
:10172800DC02C2F1200300FA03FC20FA02F001FAFD
:1017380003FE40EA0E0021FA02F11444BDE600BFA0
:101748004FF0FF3C06E000BF4FF0010C02E000BF85
:101758004FF0010C4DF804CD4FEA410C7FEA6C5C68
:101768004FEA430C18BF7FEA6C5C1BD001B050EA0B
:10177800410C0CBF52EA430C91EA030F02BF90EAF6
:10178800020F0020704710F1000F91EA030F58BFB5
:10179800994208BF90422CBFD8176FEAE37040F017
:1017A800010070474FEA410C7FEA6C5C02D150EAB5
:1017B800013C07D14FEA430C7FEA6C5CD6D152EA70
:1017C800033CD3D05DF8040B704700BF8446104635
:1017D80062468C461946634600E000BF01B5FFF734
:1017E800B7FF002848BF10F1000F01BD4DF808ED04
:1017F800FFF7F4FF0CBF012000205DF808FB00BFD5
:101808004DF808EDFFF7EAFF34BF012000205DF82E
:1018180008FB00BF4DF808EDFFF7E0FF94BF01207B
:1018280000205DF808FB00BF4DF808EDFFF7CEFF7C
:1018380094BF012000205DF808FB00BF4DF808EDBB
:10184800FFF7C4FF34BF012000205DF808FB00BF8C
:101858004FEA410212F5001215D211D56FF47873D0
:10186800B3EB625212D94FEAC12343F0004343EA73
:10187800505311F0004F23FA02F018BF404270474E
:101888004FF00000704750EA013005D111F00040D8
:1018980008BF6FF0004070474FF00000704700BF6E
:1018A80080F0004002E000BF81F0004142001FBF0D
:1018B8005FEA410392EA030F7FEA226C7FEA236C16
:1018C8006AD04FEA1262D2EB1363C1BFD21841400B
:1018D80048404140B8BF5B42192B88BF704710F0A1
:1018E800004F40F4000020F07F4018BF404211F044
:1018F800004F41F4000121F07F4118BF494292EAAC
:10190800030F3FD0A2F1010241FA03FC10EB0C00D7
:10191800C3F1200301FA03F100F0004302D5494264
:1019280060EB4000B0F5000F13D3B0F1807F06D311
:1019380040084FEA310102F10102FE2A51D2B1F109
:10194800004F40EBC25008BF20F0010040EA0300FE
:101958007047490040EB0000013A28BFB0F5000F7E
:10196800EDD2B0FA80FCACF1080CB2EB0C0200FA34
:101978000CF0AABF00EBC25052421843BCBFD04083
:101988001843704792F0000F81F4000106BF80F4FD
:1019980000000132013BB5E74FEA41037FEA226CC0
:1019A80018BF7FEA236C21D092EA030F04D092F08B
:1019B800000F08BF0846704790EA010F1CBF0020BF
:1019C800704712F07F4F04D1400028BF40F000401C
:1019D800704712F100723CBF00F50000704700F03C
:1019E800004343F0FE4040F4000070477FEA226263
:1019F80016BF08467FEA23630146420206BF5FEA34
:101A0800412390EA010F40F4800070474FF0000333
:101A180004E000BF10F0004348BF40425FEA000CFA
:101A280008BF704743F0964301464FF000001CE0A2
:101A380050EA010208BF70474FF000030AE000BFF8
:101A480050EA010208BF704711F0004302D5404236
:101A580061EB41015FEA010C02BF844601460020A8
:101A680043F0B64308BFA3F18053A3F50003BCFAC3
:101A78008CF2083AA3EBC25310DB01FA02FC634470
:101A880000FA02FCC2F12002BCF1004F20FA02F277
:101A980043EB020008BF20F00100704702F120026A
:101AA80001FA02FCC2F1200250EA4C0021FA02F2CB
:101AB80043EB020008BF20EADC7070474FEA40029F
:101AC800B2F1FE4F0FD34FF09E03B3EB12620DD964
:101AD8004FEA002343F0004310F0004F23FA02F0CE
:101AE80018BF404270474FF00000704712F1610F75
:101AF80001D1420205D110F0004008BF6FF000404C
:101B080070474FF00000704753B94AB9002908BF21
:101B180000281CBF4FF0FF314FF0FF3000F070B9C4
:101B2800ADF1080C6DE904CE00F006F8DDF804E02C
:101B3800DDE9022304B070472DE9F047089E0D4601
:101B480004460F46002B4AD18A42944665D9B2FA18
:101B580082F343B102FA03FCC3F120029F4020FA4A
:101B680002F217439C404FEA1C4E1FFA8CF5B7FB54
:101B7800FEF1220C0EFB117742EA074201FB05F049
:101B880090420AD91CEB020201F1FF3780F01B8159
:101B9800904240F2188102396244121AA4B2B2FB90
:101BA800FEF00EFB102244EA024400FB05F5A542B4
:101BB8000AD91CEB040400F1FF3280F00681A5422B
:101BC80040F203816444023840EA0140641B00216A
:101BD8001EB1DC400023C6E90043BDE8F0878B4214
:101BE80008D9002E00F0EC800021C6E9000508465F
:101BF800BDE8F087B3FA83F1002949D1AB4202D39B
:101C0800824200F2F780841A65EB0302012017462E
:101C1800002EE2D0C6E90047DFE702B9FFDEB2FADC
:101C280082F3002B40F08F808A1A4FEA1C471FFA74
:101C38008CFE0121B2FBF7F507FB1520220C42EAC6
:101C480000420EFB05F0904208D91CEB020205F198
:101C5800FF3802D2904200F2CA804546121AA4B256
:101C6800B2FBF7F007FB102244EA02440EFB00FE29
:101C7800A64508D91CEB040400F1FF3202D2A645A0
:101C880000F2BA801046A4EB0E0440EA05409FE734
:101C9800C1F120078B4022FA07FC4CEA030C05FA35
:101CA80001F420FA07F3FD40234300FA01F94FEA53
:101CB8001C401FFA8CFEB5FBF0F81C0C00FB1855F5
:101CC80044EA054408FB0EF5A54202FA01F20BD9D5
:101CD8001CEB040408F1FF3A80F08780A54240F22B
:101CE8008480A8F102086444641B9DB2B4FBF0F33D
:101CF80000FB134445EA044403FB0EFEA64508D93D
:101D08001CEB040403F1FF306BD2A64569D9023BF2
:101D1800644443EA0840A0FB0283A4EB0E049C42FF
:101D2800C6461D4655D352D056B1B9EB0E0364EBE7
:101D3800050404FA07F7CB40CC401F43C6E90074FA
:101D48000021BDE8F087C3F1200102FA03FC20FA64
:101D580001F225FA01F19D402A434FEA1C471FFA78
:101D68008CFEB1FBF7F007FB1015110C41EA054199
:101D780000FB0EF58D4204FA03F408D91CEB0101AF
:101D880000F1FF382FD28D422DD902386144491B0A
:101D980092B2B1FBF7F507FB151142EA014205FBC8
:101DA8000EF1914208D91CEB020205F1FF3816D258
:101DB800914214D9023D6244521A45EA004139E77A
:101DC8003146304609E73946E7E61046FCE6C145A4
:101DD800AAD2B8EB020E63EB0C050138A4E745461E
:101DE800EAE7034695E74046D1E7D0467CE7023D5F
:101DF800624433E708460BE76444023843E700BF10
:101E0800704700BF1348144A08B54FF00043C0E9B3
:101E180000230422002342610122C2614FF4805151
:101E280007220383C0E90233C0E90933C0E90C1271
:101E38000361837680F8203080F82C30826380F844
:101E48003C30C36402F048FC18B1BDE8084000F01B
:101E580009BC08BD7C010020002401400268084B31
:101E68009A4282B00AD14FF0B0431A6E42F400721F
:101E78001A661B6E03F400730193019B02B070474E
:101E8800002401400268054B9A4201BF4FF0B0425E
:101E9800136E23F400731366704700BF00240140DB
:101EA80030B585B000240546CDE901440394FFF719
:101EB800A9FF144802F0A8FF08B100F0D3FB1148AD
:101EC800039401A9CDE9015402F064FD08B100F0C2
:101ED800C9FB0C4802F0C2FE08B100F0C3FB4FF08A
:101EE800FF31084802F0F8FC064802F06FFF054889
:101EF80002F04CFD0446034802F012FF204605B0EC
:101F080030BD00BF7C010020014B024A1A607047B7
:101F18007C0100200024014008B50948FFF7C0FFF4
:101F280068B1084BB3F8AA304FF6FF72934216BF58
:101F380040F6E442044B5343B3FBF0F398B208BDB8
:101F4800002000B40075FF1FD8084C0013B500230B
:101F5800ADF80630FFF7E0FF04461948FFF7A0FF89
:101F6800184BB3F8C820B3F8A8108A4204FB00F055
:101F780018D040F6E443B0FBF3F364205B1A434304
:101F8800521A93FBF2F31E331BB2ADF80630BDF8BC
:101F980006305BB21B02ADF80630BDF8060000B291
:101FA80002B010BD4FF47A7240F6FF73B0FBF3F342
:101FB8005343A3F53923A3F50C6340F6C412E0E7B5
:101FC800001000B00075FF1F4FF0B04382B09A6A4E
:101FD80022F480529A629A6C42F480529A649B6C02
:101FE80003F480530193019B002002B070474FF027
:101FF800B04382B09A6C02439A649B6C034001938D
:10200800019B02B0704708B50420FFF7F0FF0120DC
:10201800FFF7EDFF0220FFF7EAFF002211460B2031
:1020280002F090FF0B2002F0BFFF002211460C20A7
:1020380002F088FF0C2002F0B7FF002211460D20A5
:1020480002F080FF0D2002F0AFFF002211460E20A3
:1020580002F078FF0E2002F0A7FF002211460F20A1
:1020680002F070FF0F2002F09FFF0022114610209F
:1020780002F068FF102002F097FF0022114611209D
:1020880002F060FF112002F08FFF00223620114677
:1020980002F058FFBDE80840362002F085BF000076
:1020A80008B503F0C9F910B16FF0040008BD064B7C
:1020B8009A6942F040429A614CF2FA321A6103F08E
:1020C800CDF90028F2D0EFE700400058F0B585B010
:1020D80000230C4600930646A8B3FFF7E1FF054628
:1020E80070BB03F0A9F988BB1A481B4A0223019365
:1020F800D0F8E01506F1784302EA8121B3FBF1F745
:1021080001FB1733DB0A0293D0F8E00504F17841AC
:102118000139314402EA8022B1FBF2F002FB1011CE
:10212800C3EBD1230133694601A8039303F016FAE0
:1021380020B102280CBF01256FF0010503F08EF9CC
:10214800284605B0F0BD6FF00505F9E76FF0040506
:10215800F6E700BF0070FF1F00FCFF03014B18608B
:1021680000207047E00100202DE9F04F89B0B0F160
:10217800006F06460F460092C0F0C580DFF89881D0
:10218800664DD8F8E03505EA832303F10063013B87
:10219800984200F2B880002800F0B880002900F0CA
:1021A800B58040EA02035B0740F0B080FFF778FF94
:1021B8000446A0BB03F040F9002840F0AA80D8F8F4
:1021C800E01506F1784205EA8121B2FBF1F301FB43
:1021D8001322009B03F17843013B3344B3FBF1F036
:1021E80001FB1033DB0A01334FEAD22AA3EBD222D8
:1021F800012A039388BFC6F30A050AF58038C6F199
:10220800080398BF009D069388BFC5F500654FEA8F
:10221800C828B346039B9A4505D303F01FF9204607
:1022280009B0BDE8F08FA6F10803069A1A44954252
:1022380019D804950197CDF814B04FF00009059B03
:1022480009EB0301049B99453ED3009BAB442F4403
:102258005D1BB5F5006F28BF4FF400650AF1010A50
:1022680008F50068D6E753F8081F5A68B2F1FF3F2F
:1022780008BFB1F1FF3FD8D0294B186810B96FF0EB
:102288000504CAE7B8F1000F04D04FF400624146D4
:102298000EF03EFADFF88890D9F80030CBF30A0048
:1022A80039461844AAB20EF033FA4FF4006140469A
:1022B800FFF70CFF08BBD9F8003001934FF4006317
:1022C800CDF814800493B8E7019B07914B4402931F
:1022D8000120D3E9002303F0FBF888B90799019B93
:1022E800D1E9000259F80310029B5B689A4208BFC3
:1022F800884205D109F10809A1E76FF001048CE7CC
:102308006FF0030489E74FF0FF3488E76FF00504A6
:1023180085E76FF0040482E70070FF1F00FCFF03ED
:10232800E0010020B1F1006F70B511D30B4BD3F869
:10233800E0650B4B03EA862303F10063013B9942F6
:1023480006D840B139B192B20EF0E2F9002070BD62
:102358004FF0FF30FBE76FF00500F8E70070FF1F54
:1023680000FCFF03B0F1006F10B40DD3084BD3F895
:10237800E045084B03EA842303F10063013B9842DC
:1023880002D810BCFFF7A2BE4FF0FF3010BC704758
:102398000070FF1F00FCFF034FF0B04382B0DA6CFF
:1023A8000243DA64DB6C03400193019B02B070477F
:1023B80070B5012086B00024CDE90444FFF7ECFF96
:1023C8000220FFF7E9FF0420FFF7E6FF01250222BC
:1023D8000DEB00014FF404134FF09040CDE90123B9
:1023E800204E039503F008F94FF4441301A94FF068
:1023F8009040CDE90235019503F0FEF804230DEB7A
:1024080003013046CDE90135CDE9034403F0F4F882
:1024180022463046082103F015FA4FF4806301A9DB
:102428004FF09040CDE90134039403F0E5F8082318
:1024380001A93046CDE90135CDE9034403F0DCF8C4
:1024480022462146062002F07DFD062002F0ACFD62
:1024580022462146072002F075FD072002F0A4FD60
:1024680006B070BD0004004808B51248124A134B64
:10247800C0E9002300230122C0E90232C0E9043385
:10248800C0E90633036203F0EFF908B100F0EAF897
:102498000848002103F039FA08B100F0E3F80548CC
:1024A800002103F058FA18B1BDE8084000F0DAB886
:1024B80008BD00BFA4020020005800405D3E302047
:1024C80070B596B005461422002103A80EF058FDF9
:1024D8003822002108A80EF053FD2A68304B9A4292
:1024E8005BD18023089308A84FF440230E9303F090
:1024F8008DFF08B100F0B6F84FF0B0444FF4C0506B
:10250800E36C43F00103E364E36C03F0010302931B
:10251800029B12230026CDE903030323CDE90563BB
:102528004FF09040042303A9079303F065F8A36DC7
:10253800DFF870C043F48003A365A36D1A4C03F45D
:1025480080030193019B26620D23C4E900C3204642
:102558008023C4E90266C4E90436C4E9066602F0C9
:1025680083FD08B100F07EF8104AEC63A562104CB8
:102578000E23C4E900231021002380222046C4E949
:102588000213C4E90423C4E90633236202F06CFD94
:1025980008B100F067F8AC63A56216B070BD00BF63
:1025A8000058004044000240E40100205800024066
:1025B8004402002000B59BB04822002108A80EF074
:1025C800DFFC1822002102A80EF0DAFC03F0E8F97B
:1025D8004FF0B0420120D2F8903023F01803C2F82F
:1025E8009030D2F8003423F4C06343F40073C2F887
:1025F8000034D2F8003403F4C0630193019B242310
:10260800089381230B930023CDE91003B02208A877
:10261800CDE9122303F03CFB08B172B6FEE74F2365
:10262800CDE90230CDE90400CDE90600022102A877
:1026380003F0C8FD08B172B6FEE71BB05DF804FBF5
:1026480008B501F0F7FFFFF7B5FFFFF7B1FEFFF799
:10265800DAFC00F018FE40F6B83000F049FA00F055
:1026680019FEFCE772B6FEE700B58DB02C220021FA
:1026780001A80EF085FC1748174B03601F238360E1
:102688004FF080420023C0E90433C0E90723836187
:102698004FF48073436204F03FF808B1FFF7E2FF9C
:1026A8000C4804F065F908B1FFF7DCFF4FF0005360
:1026B80000220793074808924FF4807301A90292F9
:1026C80006920B9304F088F808B1FFF7CBFF0DB022
:1026D8005DF804FBF80200200028004010B504460D
:1026E80090B03822002102A80EF04AFC2268194B4B
:1026F8009A422CD14FF48033029302A84FF480738E
:102708000F9303F083FE08B1FFF7ACFF4FF0B0431F
:102718000220D3F8902042F40042C3F890209A6D2A
:1027280042F480629A659B6D002203F4806311462F
:102738000193019B02F006FC022002F035FC002206
:102748002A20114602F0FEFB2A2002F02DFC10B0D0
:1027580010BD00BF002800407047000008B501F018
:102768007FFF044B0120C3F88800BDE8084003F050
:102778006FB900BF0004005801F079BF08B501F037
:1027880076FF00F063FCFFF713FEFFF73CFCBDE8A3
:102798000840FFF769BE08B501F062FFBDE80840D0
:1027A8000121002003F004B970477047FEE7FEE7F7
:1027B800FEE7FEE7FEE77047704770477047000086
:1027C800014804F0FBB800BFF8020020012003F024
:1027D8003FB8022003F03CB870477047014802F048
:1027E800BDBD00BFE4010020014802F0B7BD00BF35
:1027F800D0030020014802F0B1BD00BF70030020E3
:10280800FFF7F2BF7047704770470000014804F0B7
:1028180099BC00BF30040020014803F001BF00BF8D
:10282800F8020020014804F0F4BA00BF5C0300205D
:102838002DE9F04389B080460020109E0790894614
:1028480015461F46FDF7ECFCF0B9104CCDE9009099
:10285800CDE9020407AB0E480593142304933A46C6
:10286800434629460068FDF7A5FD2346324604F194
:10287800140153F8044B42F8044B8B42F9D1079BDF
:10288800337509B0BDE8F0830120FAE73003002072
:10289800781101087FB5124C00253C2302A8637506
:1028A800CDE90255257500F0C5F8042303AA009464
:1028B80012210C48FFF7BCFF0B49142220460EF0EA
:1028C8004FFB0646B0FA80F0400960750090074B50
:1028D8002A46294602200DF013FE304604B070BD8A
:1028E80044030020BE110108EE060020A0110108D3
:1028F800054808B50823036004F0A6F818B1BDE838
:102908000840FFF7AFBE08BD5C0300204FF0B0439E
:1029180007B55A6E42F001025A665B6E002203F058
:102928000103019311463220019B02F00BFB322078
:1029380003B05DF804EB02F037BB00000CB407B538
:10294800054A05AB102101930EF0ECF903B05DF8D0
:1029580004EB02B0704700BFD011010830B585B054
:10296800044602A80D460EF009F8BDF90C30064AD7
:1029780000931021029B2046FFF7E0FF2046FEF758
:102988001BFD288005B030BDD01101084FF0B042C2
:1029980010B5936823F4004393600EF077F80F4B5B
:1029A80001241C7000F0B8F80DF040FD0C480DF043
:1029B80057FD0C4B4FF400421A6120460DF056FDAE
:1029C800FFF7A2FA00F014F900F050FC0DF04AFEEF
:1029D80021462046BDE810400DF064BE6803002083
:1029E80065290008004000580DF072BE08B5FFF7D1
:1029F80093FA40F6B83398420CD8B0F5E16F0BD390
:102A0800FE23A0F5E16058434FF49663B0FBF3F062
:102A1800C0B208BDFE20FCE70020FAE77FB5684693
:102A280000F0CAF80198FFF749F800B207B05DF85E
:102A380004FB0000194A38B5D2F88035591C044601
:102A480019D101F01BFE054601F024FE054401F0F2
:102A58001BFE2B0EE3712B0CA3712B0A6371030E63
:102A6800E370C0F30742C0F307232571C0B2A27018
:102A78006370207038BD190AC3718171190C1B0E5F
:102A880041710371D2F88435C370D2F88405C0F35C
:102A98000722C0F30743000EE9E700BF0070FF1FDD
:102AA80038B5094BD3F8803503600133054609D1A1
:102AB80001F0E4FD044601F0E7FD444001F0EAFDC1
:102AC80044402C6038BD00BF0070FF1F0121022068
:102AD8000DF0D2BD002102200DF0CEBD00207047C0
:102AE800024B187808B100F0BBB8704768030020A3
:102AF80082B00190019802B000F04EB94FF0B04397
:102B080082B0DA6C42F00202DA64DB6C03F0020392
:102B18000193019B02B070472DE9F043254C87B023
:102B280001F0BEFD01F0C4FD01F0CAFD012300253E
:102B380002934FF48059032301A9204604934FF4CC
:102B4800005803950595FFF7D9FFFFF7D7FFFFF763
:102B5800D5FFFFF7D3FFCDF8049002F04DFD01A992
:102B680020464FF40067CDF8048002F045FD01A926
:102B780020464FF40046019702F03EFD01A9204689
:102B8800019602F039FD2A464946204602F05AFECF
:102B98002A464146204602F055FE2A463946204636
:102BA80002F050FE2A463146204602F04BFE07B09E
:102BB800BDE8F0830004004810B50446FFF7C6F9E5
:102BC800074BA36040F30F20FEF724FF054B064A8E
:102BD8002360064B6060C4E90323002010BD00BFDA
:102BE8000000484200007A440D093E00AB0305008E
:102BF80000207047014B1868704700BF6C03002025
:102C08000320704708B501464FF47A72002380020A
:102C1800890DFEF779FF08BD4FF47A73A0FB030313
:102C2800800A40EA83507047034B98689A6890423C
:102C3800FBD1C043704700BF0028004008B5FFF72C
:102C4800F3FF014B186008BD6C03002008B5FFF7BF
:102C5800EBFF024B1B68C01A08BD00BF6C030020C5
:102C6800024B187808B1FFF7DFBF704769030020EF
:102C780010B5074B074C0122DA654FF480712046E6
:102C880003F094FC4FF0FF332363002010BD00BF16
:102C980000280040F802002002460021014803F005
:102CA8009EBE00BFF802002002460121014803F041
:102CB80096BE00BFF802002010B58CB02C2200216F
:102CC800044601A80EF05CF9FFF7D2FF0C4B0D4843
:102CD8001B681C440023089306934FF00053E443F9
:102CE800079301224FF4807301A902940B9303F018
:102CF80073FD08B1FFF7B6FC00200CB010BD00BF93
:102D08006C030020F802002038B50546FFF78CFF59
:102D180002210446074803F069FEC4F309024FF490
:102D28007A71A2FB0121920AA30A2A8043EA805001
:102D380038BD00BFF80200200148002103F056BE4C
:102D4800F80200200148012103F050BEF8020020DB
:102D5800F8B50F4D2E78CEB90E4C4FF0FF372763DC
:102D6800FFF782FCFFF784FF4FF48071204603F0E1
:102D78001DFC2046276303F0DDFD32462046022174
:102D880003F02DFEFFF75AFF01232B700020F8BD3A
:102D980069030020F8020020014610B54FF47A724A
:102DA80000238002890DFEF7AFFE0146FFF73CFFC6
:102DB8000446FFF739FF031B8B4200D310BD00BF49
:102DC800F7E70DF06BBF000010B5064C0221204656
:102DD80003F00CFE0221421C2046BDE8104003F01F
:102DE800FEBD00BFF80200201648174A08B54FF488
:102DF800E133C0E9002300230C22C0E90233C0E913
:102E08000523C0E90733C0E90933036104F07BFFF8
:102E180008B1FFF727FC0B48002105F0F0F808B1CE
:102E2800FFF720FC0748002105F009F908B1FFF772
:102E380019FC044805F0C3F818B1BDE80840FFF7CD
:102E480011BC08BD300400200044004070B596B0A5
:102E580005461422002103A80EF092F8382200211A
:102E680008A80EF08DF82A68334B9A4261D10223E4
:102E7800089308A8314B0A9303F0C8FA08B1FFF782
:102E8800F1FB4FF0B0430C219A6D2D4C42F4003207
:102E98009A659A6D02F400320292029ADA6C42F054
:102EA8000102DA64DB6C03F001030193019B022346
:102EB8000026CDE903130323CDE905634FF09040C5
:102EC800072303A9079302F097FB1E4826621423E1
:102ED800C4E900031023C4E9023620468023C4E96C
:102EE8000436C4E9066602F0BFF808B1FFF7BAFB7A
:102EF800154AEC67A562154C1323C4E90023204644
:102F080000238022C4E90233C4E90423C4E9063358
:102F1800236202F0A9F808B1FFF7A4FB2520C5F841
:102F2800804000220221A56202F00CF8252002F060
:102F38003BF816B070BD00BF0044004004000C0010
:102F4800D0030020800002406C0002407003002083
:102F580002680E4B9A4210B5044616D14FF0B042A3
:102F68000C21936D23F4003393654FF0904002F0E9
:102F7800EFFBE06F02F0ECF8D4F8800002F0E8F81C
:102F8800BDE81040252002F01DB810BD00440040E7
:102F980008B50A460146024804F038F8002008BD82
:102FA8003004002013B5114B114C18604FF4001376
:102FB800009302AB13E90600204604F0A4FF23683F
:102FC800DA69D103FCD4DA695202FCD59A68084858
:102FD80042F480029A6004F0DCFF064904480122AA
:102FE80004F04AFF002002B010BD00BFC404002056
:102FF80030040020CC04002008B5074B1860FFF708
:1030080002F8FFF7F1FE054AD2F8803043F000637A
:10301800C2F88030002008BDC8040020000800580D
:1030280008B54FF0B04308489A6B42F400329A63EF
:103038009A6B22F400329A63FFF78AFF0F2001F09F
:10304800C1FF002008BD00BF3004002008B50748B4
:1030580004F059FE08B1FFF705FB054802F004F833
:1030680018B1BDE80840FFF7FDBA08BD30040020DC
:10307800D00300200268044B9A4203D1034B00207E
:103088001B681847704700BF00440040C804002070
:1030980002680B4B9A4210B504460FD1094B1B68C6
:1030A8002BB1D0F8902012B9074801219847204643
:1030B8000549BDE81040012204F0DEBE10BD00BF86
:1030C80000440040C4040020CC04002013B5134C75
:1030D80023785BB9E37C03F0FF023BB9104B114640
:1030E800022002B0BDE810400DF00ABAFFF7D2FB8B
:1030F80000380C4B18BF0120400018701A78022ABB
:1031080002BF00222270E2741B7800930022064B53
:10311800114603200DF0F4F902B010BDEE060020B0
:103128002C120108E00400204812010838B5184C98
:1031380023785BBBE37C03F0FF023BBB154D2B6898
:10314800012B0CD92B68042B09D81146124B0220ED
:103158000DF0D6F9114A0421012000F0ADFB2B68CF
:10316800042B13D900220E4B114602200DF0C8F98A
:10317800FFF790FB00380B4B18BF01204000187078
:103188001B78022B02BF00232370E37438BD00BFF5
:10319800EE060020DC0400205F12010884120108FA
:1031A80089120108E0040020002213B5154B164CC3
:1031B800114603200DF0A4F901220821134802F05A
:1031C80041FB4FF47A70FFF793FC4FF480614FF0A6
:1031D800904002F031FB207021780D4A0D4B0029F8
:1031E80018BF13460022009311460B4B01200DF027
:1031F80087F906480022082102F024FB237802B050
:1032080010BD00BFE4120108E104002000040048DA
:10321800D3120108BC120108FC120108704770475C
:10322800022808B50ED801221021074802F00AFB2F
:103238003220FFF75DFCBDE808400348002210215A
:1032480002F000BB08BD00BF00040048054B1B7816
:10325800B3FA83F35B09037100234371024B012224
:103268001A707047E1040020ED060020034A00238D
:1032780013715371024A1370704700BFCE040020C7
:10328800ED060020704708B5FFF780FBBDE8084051
:1032980000F0D4BC4FF0FF300DF07EBA704700004C
:1032A800014BD870704700BF5C000020014B1874B8
:1032B800704700BF5C00002007B5064B00221B5C6E
:1032C80000931146044B02200DF01AF903B05DF883
:1032D80004FB00BF2C1301081213010808B50220D3
:1032E80000210DF021FABDE8084001480DF084BC2A
:1032F8003C060020002101200DF016BA13B50D4C34
:10330800A0B120600C480DF029FC21680A480DF096
:10331800ADFC09480DF070FC236800930022074BB0
:10332800114601200DF0ECF802B010BD42F2107306
:103338002360E7E7740000203C06002030130108F2
:1033480013B50D4C206023680BB90C4B23600C4857
:103358000DF004FC21680A480DF088FC08480DF0BF
:103368004BFC236800930022064B114601200DF008
:10337800C7F802B010BD00BF0C000020A0860100F5
:10338800540600205913010837B5044600283AD0DE
:1033980090F90650002D38D11F480DF0DFFB2A4662
:1033A80029461E4B02200DF0ABF8E379012B0CBF28
:1033B8001B4B1C4B2A46294602201B4D0DF0A0F83A
:1033C800E3792B70194B1868FFF7BAFF184B186888
:1033D800FFF794FF2978174A174B012918BF13469E
:1033E800002200931146154B01200DF089F894F93D
:1033F8000530019394F9043000930022104B1146D4
:1034080002200DF07DF803B030BD00220D4B1146AF
:1034180002200DF075F8EAE7D80500209E13010890
:10342800B3130108D0130108080600200C0000207F
:10343800740000209913010895130108ED13010881
:10344800251401080C14010838B504460D46074830
:103458004FF40061FEF786FF30B92A46214603483B
:10346800BDE83840FEF780BE38BD00BF00F0030855
:103478000A460149FEF756BF00F0030870B5164822
:103488000DF06CFB05F034FA044650B10022134BE2
:10349800114602200DF034F8BDE8704010480DF0D8
:1034A800ABBB104D104B0246014602200DF028F828
:1034B80001260E4B2E702246214602200DF020F8E0
:1034C8000B4805F0B9F82878314604F0E3FE0248C5
:1034D8000DF092FBE0E700BF3C0600204E14010807
:1034E8000C060020000000206C140108801401085C
:1034F8005C00002030B587B0FFF778FA0446FFF784
:1035080053FE02A8FFF7A2FE474B07221A70474A4C
:103518001178002943D00021117008221A70444AFA
:103528005968127862F07F020A705A6824B204EB74
:10353800440404EB4414FE21B4FBF1F45470022259
:103548003C493D4C0978012988BF00225A70637AAA
:1035580033B104F041FE012802D120460DF0FEFAF5
:10356800364B3148D978002204F022FF044600285F
:1035780044D10146324B012203200CF0C1FF3148EF
:103588000DF0ECFA304B2F481968A14238BF21469C
:103598000DF06CFB2B480DF02FFB07B030BD2B490D
:1035A8002B480A7822B9057805F0FF02002DC7D00C
:1035B800002202701E480A7059680078087059681D
:1035C8004A705A68562191705A680121D1705A6818
:1035D80024B204EB4404FE2104EB4414B4FBF1F4DC
:1035E80014715A68022151715A689DF80D10917131
:1035F8005A689DF80C10D1710822A1E7063410D141
:1036080004F0E4FD04460028B9D04FF47A7301228F
:10361800B0FBF3F30021009303200E4B0CF070FF76
:10362800ADE70024ABE700BF040000206C060020D3
:10363800D4050020E0040020D80500205C0000200C
:103648009F1401083C060020740000200307002096
:10365800ED060020AE14010800B503468DB0002821
:103668002CD0407802280AD003282AD0164B0022F2
:10367800114602200DB05DF804EB0CF041BFDA7E74
:103688000B929A7E0A925A7E09921A7E0892DA7DE5
:1036980007929A7D06925A7D05925A680492DA68D2
:1036A800039293F914200292B3F9122001921B7C21
:1036B80000930022054B11460CF022FF0DB05DF877
:1036C80004FB034BD3E700BFCC140108E314010843
:1036D8005515010801284FF000020CBF024B034B9F
:1036E800114602200CF00CBF74150108861501085C
:1036F8001FB50446002831D00378002B2ED01D4872
:103708000DF07AFA002211461B4B02200CF0F8FE4D
:1037180094F91830039394F90A300293237C0193A7
:10372800E368009300221146144B02200CF0E8FED7
:103738000022134B114603200CF0E2FE237A012BE2
:103748000ED1617A0F4A104B002908BF1346002298
:10375800009311460D4B02200CF0D2FE04B010BDB0
:1037680000220B4B1146022004B0BDE810400CF0BB
:10377800C7BE00BF240600209F150108D015010808
:10378800011601089A1501089B1501080E16010873
:103798001F16010808B5104B0122002102201A70DB
:1037A8000CF0C2FF0D480DF027FA0D4B1B788BB1BA
:1037B8000C4B1A7872B9DB7C63B90B4B1A68042A74
:1037C8009EBF1A6801321A600021BDE80840102027
:1037D8000CF0AABF08BD00BF6C06002054060020EC
:1037E80008060020EE060020DC040020044B1B78AD
:1037F800022B03D1002108200CF096BF704700BFB0
:103808000000002008B505F07CF880B904F0E4FC5D
:1038180001280CD1BFF34F8F0549064BCA6802F443
:10382800E0621343CB60BFF34F8F00BFFDE708BDD5
:1038380000ED00E00400FA0510B505F0F7F810F106
:10384800080F07D1064B0022BDE8104011460220A0
:103858000CF056BE013001D1024BF4E710BD00BF99
:103868002D1601084316010870477047704700007D
:10387800012837B5044603D0022817D003B030BD5D
:1038880001464FF0904001F0D7FF00220546009016
:10389800084B114620460CF033FE012DEED10021D5
:1038A800022003B0BDE830400CF03EBF00210820E4
:1038B800F7E700BF5B16010873B505460C461646C8
:1038C80004F058FD0346002838D0002426480DF09F
:1038D80045F9264B24481968A14238BF21460DF006
:1038E800C5F9214802B0BDE870400DF085B94A68B5
:1038F800F05CD0540133DAB2A242F8D31C4B0D70FD
:103908001B78012B88BF00244C701A4C637A33B1A2
:1039180004F062FC012802D120460DF01FF9164B75
:103928001648D978002204F043FD044640B9014600
:10393800134B012202200CF0E3FDC7E70F49DAE739
:103948000634C2D104F042FC04460028BED04FF42D
:103958007A730122B0FBF3F3002100930220094B94
:103968000CF0CEFDB2E700BF3C060020740000203A
:10397800E0040020D80500205C000020040000209E
:103988009F140108AE140108044B1B7823B9044A9C
:1039980005210120FFF790BF704700BFE004002019
:1039A8007916010810B5002490B03C22214601A8E0
:1039B80000940DF0E5FA2F4B2022DA7219788DF871
:1039C800001059788DF8011099788DF80210D9787F
:1039D8008DF8031019798DF8041059798DF80510B0
:1039E80099798DF80610D9798DF80710197A8DF81C
:1039F8000810597A8DF80910997A8DF80A108DF8FF
:103A08000B2021460DF10B0258180131007B02F8FA
:103A1800010F1C29F8D193F828208DF8282093F855
:103A280029208DF8292093F82A208DF82A2093F848
:103A38002B208DF82B2093F82C206AB193F83F2087
:103A480052B10DF12B0100229818013290F82C0088
:103A580001F8010F142AF7D107484FF40061FEF767
:103A680081FC20B9044840226946FEF77DFB10B06E
:103A780010BD00BF7800002000F80308014940226B
:103A88000CF046BE00F8030870B52A4D28796B790A
:103A98004D2BC0B233D1C0EB001080000A2838BFCC
:103AA8000A204FF47A735843234BAC791860EB79AA
:103AB8004D2BE4B22BD1C4EB0414A40095F82C30A0
:103AC8001E4E63BB95F83F304BBB42F21070FFF7B8
:103AD80015FC3068FFF734FC2B7A194A1949DBB218
:103AE80013706B7A184ADBB213700023EA1892F845
:103AF8002C20D2B2CA540133142BF7D170BD6B7984
:103B0800482B0ABF4FF461636B795843C6E7EB79DA
:103B1800482B0ABF4FF46163EB795C43CEE7FFF7AC
:103B2800EDFB012C38BF01244FF47A735C433460F9
:103B3800CFE700BF78000020740000200C000020B0
:103B480002070020EE060020E004002010B590B027
:103B580000213C2201A800910DF012FA40223449BC
:103B680068460CF0D5FD9DF800203AB99DF8010093
:103B7800562803D19DF8021001290FD000222D4BA1
:103B8800114601200CF0BCFCFFF70CFF4FF47A70D3
:103B9800FEF7AEFFFFF778FF10B010BD264B1A7086
:103BA800587099709DF80310D9709DF80410197118
:103BB8009DF8051059719DF8061099719DF8071028
:103BC800D9719DF8081019729DF8091059729DF85D
:103BD8000A1099729DF80B1001F03F01D972D87A3A
:103BE800D1B288421BD89DF8282083F828209DF858
:103BF800292083F829209DF82A2083F82A209DF877
:103C08002B2083F82B200DF12B010022981801326C
:103C180011F8014F80F82C40142AF7D1BAE701F1C6
:103C280040006844194410F8340C08730132D6E790
:103C380000F803087F16010878000020F0B50B2370
:103C48008BB00226002401250327CDE9063617226A
:103C58005623CDE9043221465E4B03942246CDE932
:103C680001550097284609940CF04AFC5A4B0095D8
:103C780022462146CDE9017430460CF041FC05236B
:103C8800CDE900632246554B0294214630460CF09C
:103C980037FC534B009522462146CDE90174304646
:103CA8000CF02EFC09A9204604F00EFE099BC3F374
:103CB80007220292C3F307421B0E01920093224689
:103CC800484B214630460CF01BFC09A9284604F055
:103CD800FBFD099BDAB20392C3F307220292C3F3F6
:103CE80007421B0E0192009322463F4B2146304665
:103CF8000CF006FC3D4B3E48009422464FF4FA7106
:103D08000CF0CEFE3B4B3C48009422464FF4FA712F
:103D18000CF0C6FE394B3A4800942A464FF4FA7123
:103D28000CF0BEFE2046FEF719FA08B1FEF79AFC21
:103D3800344B009400224FF4FA6133480CF0B0FE83
:103D4800324A002101200CF0ABFD314A002102204B
:103D58000CF0A6FD2F4A002104200CF0A1FD2E4AEC
:103D6800002108200CF09CFD00F0BCFB2B492C48DE
:103D780004F06CFD2B4804F05FFC21480CF03CFF7C
:103D8800294B0021187804F085FA28490094284B1B
:103D98000968284800220CF083FE26480CF02CFF06
:103DA800FFF7D4FE244A002110200CF079FD234AA5
:103DB80000214FF480600CF073FD214B21481968F5
:103DC800214B009400220CF06BFE1E480CF014FFEF
:103DD8000BB0F0BDC1160108081701082917010822
:103DE8004A1701086B1701088C170108A53200084B
:103DF8002406002073380008F005002071380008F8
:103E0800D8050020F53700080C0600209981000825
:103E1800FD3400084138000885340008000003011B
:103E2800100000205C00002000000020740000202A
:103E3800E53200083C06002035310008B1310008A1
:103E48000C000020540600209D37000830B50024DF
:103E5800A3B07C22214603A802940DF091F85323C5
:103E68008DF808304FF4AB73ADF80A3001238DF8A4
:103E78000C30ADF80440FEF7B9FD00B200EB40008D
:103E880000EB4010FE23B0FBF3F08DF80D0001A805
:103E980000F0CDFBC0B143000133DBB20B4C8DF811
:103EA8000E302C228021201D1D460DF069F8029845
:103EB800BDF80C302060A380A5712246072101209F
:103EC800FFF7FAFC23B030BD5823E7E76D06002062
:103ED800F0B50378592B95B0044640F0EF810529D9
:103EE8005FD84378443B162B5BD8DFE813F01E01FC
:103EF8005A000E015A0016015A005A005A005A0078
:103F080079005A00F9005A005A005A0093015A00E1
:103F18005A009D005A005A005A0017008578482D0B
:103F280017D1B14A14210120FFF7C6FC41F28830AD
:103F3800FEF7DEFD0022AD4B114601200CF0E0FA41
:103F480040F6B830FEF7D4FD15B0BDE8F040FFF7F5
:103F580059BC532D0ED130228021A5480DF010F800
:103F6800FFF774FF41F28830FEF7C2FDA04A152121
:103F780001206DE0432D16D1002404A88DF81040CF
:103F880004F0BEFA9A4A4C231370562393709DF896
:103F98001030547001204133D07013710521FFF7A0
:103FA8008BFC15B0F0BD442DFBD1914C2C22802107
:103FB800201D0CF0E5FF00232570637001255623B2
:103FC800A370E5702571FEF711FDFE23B0FBF3F039
:103FD80000EB400000EB4010607122460621C7E765
:103FE8008378303BDBB2092BDBD8824C824A2370C2
:103FF8002378DBB253727E4A592313704D235370D2
:1040080023783033937003210120FFF755FC237880
:1040180000930022794B114601200CF071FA15B07B
:10402800BDE8F040FFF7BEBC8578482D15D1704A31
:1040380056231370937003231371172353710B23A3
:1040480000210120937102235170D070D37108218F
:1040580015B0BDE8F040FFF72FBC432DA1D1644C4B
:1040680000213C2205A804910CF08AFF04A8FFF760
:1040780005FD2422802104F10C000CF081FF9DF83D
:10408800103063709DF81130A3709DF81230E37002
:104098009DF8133023719DF8143063719DF8153025
:1040A800A3719DF81630E3719DF8173023729DF8BF
:1040B8001830257063729DF81B509DF81930A37253
:1040C8009DF81A30E3722A4607A9257304F10D00FA
:1040D8000CF087FF05F10D012246C9B201205EE709
:1040E800807839280CD83038C0B2FFF797F8404AA2
:1040F8002378137063785370A3789370032137E79C
:1041080015B0BDE8F040FFF73FBC80783928F7D8F4
:104118003038C0B2FFF783F8E9E780783928EFD85C
:104128003038C0B2FFF77CF8E1E78378303BDAB289
:10413800092AE5D8C578303DEAB2092AE0D80179DC
:10414800A1F14802D2B20B2ADAD82D4840FA02F27D
:10415800D007D5D40A224D2902FB03553FD13C2371
:104168005D43284B4FF47A7068431860264B1860FB
:10417800FFF7C4F81E4A2378137063785370A37846
:104188009370E378D3702379137105210120FFF729
:1041980093FB194B5622012600271F705A709E70F8
:1041A800DE70A178303901EB8100E178303901EB1C
:1041B8004001C9B2197122795A71144A1278D2B2DF
:1041C8001A720C4A1278D2B25A72FFF7EBFB104BF4
:1041D80000953A46394630460CF092F9E1E648290E
:1041E800BFD14FF46163BBE7B0170108C5170108D9
:1041F8006D060020E004002078000020E717010881
:10420800DEF7FFFF740000200C00002002070020EA
:10421800101801088678A6F13007FBB2092B3FF683
:104228006FAFC078A0F13005EBB2092B3FF668AF4D
:104238002379A3F14802D2B20B2A3FF661AF6D4948
:1042480041FA02F2D2073FF55BAF0A224D2B02FB7F
:1042580007552ED13C225543674A592111705321E5
:1042680051709670D070137105210120FFF724FB5F
:10427800624B5622012600271F705A709E70DE700E
:10428800A178303901EB8100E178303901EB400148
:10429800C9B299712279DA71594A1278D2B21A726E
:1042A800584A1278D2B25A72FFF77CFB564B0095E7
:1042B8008FE7482BD0D14FF46162CCE7502B5DD10A
:1042C80002297FF66EAE4378303B012B3FF669AE8C
:1042D8008378312B7FF465AE0B2904D8FFF754FBA4
:1042E8000021454A44E6454D484F0234002614F85B
:1042F800012FA919303AD2B20A730B7BCDE90263B8
:1043080023780022CDE9006311463B46012001369F
:104318000CF0F6F80C2EEAD1FEF7B4FF364B50221B
:104328001A7056229A70002401225C70DA7003F821
:10433800042F2A190134127B0C2C02F1300203F8E5
:10434800012FF6D100225023114600930120304B53
:104358000CF0D6F800232B7056236B700123AB703A
:10436800EB70274B1B78DBB22B72264B1B78DBB22A
:104378006B72EC72FFF716FB1121B2E7412B7FF449
:1043880010AE4378432B7FF40CAE16297FF409AEA8
:10439800204D421C002312F8011FE9540133142B4D
:1043A800F9D1FEF793FE1C4B5B7D012B19D1134904
:1043B8000023EA5CC8180133D2B2142B80F82C20F1
:1043C800F7D1104B00221A701B78DBB24B72FFF743
:1043D800E9FA094A631E15349C4206D1064A162199
:1043E800C6E5084B02221A70F3E713F8011F02F81A
:1043F800011BF1E7DEF7FFFF6D06002078000020C3
:1044080002070020E004002047180108921801085C
:10441800BA180108EE0600204403002070B50546CE
:1044280086B00C4600293BD028480CF0E5FB2678DE
:10443800EEB1002D48D068682E78C0B1032E0BD09D
:10444800072E2FD0022E12D1697801290FD00B0622
:104458000DD4FFF73DFD0AE06B78012B07D10078FA
:10446800012802D0022800D008B903F0C9FE237C35
:10447800052B15D894F90A20059294F9092004927D
:10448800134A52F82330039394F90830CDE90163B5
:104498000022E368009311460E4B03200CF030F81D
:1044A80006B070BD6B78012BE1D102780A4B02F09F
:1044B80001021A702AB9094B114603200CF020F8A2
:1044C800D5E7074B0022F7E72E46D0E7F005002096
:1044D80040190108E8180108D4050020D51801087A
:1044E800DF180108034B0022C3E902220122C3E9B5
:1044F8000022704704070020004870470407002086
:104508004FF0B04382B0DA6C0243DA64DB6C0340EC
:104518000193019B02B070472DE9F04186B0002459
:104528000220154D0594FFF7EBFF0420FFF7E8FF85
:10453800124F03944FF4807601230DEB0001CDE96F
:1045480001632846032304934FF4005801F054F8FC
:1045580001A93846CDF8048001F04EF822464146BC
:10456800384601F06FF928462246314601F06AF9CB
:10457800204606B0BDE8F081000400480008004865
:10458800032810B50ED8012810D868B902460B4880
:104598004FF4807101F056F9002209484FF4005198
:1045A80001F050F9002010BD0122F0E70022034875
:1045B8004FF4807101F046F90122EEE7000400484B
:1045C800000800480220704700207047012070470B
:1045D80000280CBF0F201620704700000D488546A4
:1045E80000F027F80C480D490D4A002302E0D45882
:1045F800C4500433C4188C42F9D30A4A0A4C002325
:1046080001E013600432A242FBD30CF0C1FCFEF7B8
:1046180017F8FEE700000120000000205C010020E0
:10462800C02301085C0100200C260020FEE70020C2
:104638007047704710B5032000F072FC01F018FBBA
:10464800064B18600F20FEF749FA044618B9FEF722
:10465800ACF8204610BD0124FBE700BFB8000020DD
:104668004FF0E022136923F00203136170474FF003
:10467800E022136943F0020313617047014BD3F83A
:10468800900570470070FF1F014BD3F894057047E1
:104698000070FF1F014BD3F8980570470070FF1F8B
:1046A800024A536823F0010353607047002004E076
:1046B800024A536823F0020353607047002004E065
:1046C800024A536823F0040353607047002004E053
:1046D8008068C0F380007047F7B500230193044653
:1046E800002800F0E980856D25B9FDF7B7FBE56581
:1046F80084F8545023689A68D00040F1A1809A68E1
:10470800D10000F1B480A26D42F01002A265E26D02
:1047180042F00102E26501251846FFF7D9FFA26DB4
:1047280002F01002024340F0C980A26D206922F411
:10473800817242F00202A2659A68D2075DD4226BA8
:10474800A67E94F82CC0003A18BF01221703D4E9BA
:1047580002120A43217E42EA8132617E42EAC13274
:1047680042EA4632002842EA4C02B4BF20F0004137
:104778004FF400113A430A4394F82010012903D159
:10478800002E76D142F48032616A21B1A66A01F422
:10479800E07131430A43D968E66C21F4FE3121F413
:1047A800FF711143D96094F83C206168012A01F037
:1047B800404C4CEA060609D1D4E910273A43324363
:1047C800A66C324342EA0C0242F001061F693E4AD7
:1047D8003A4032431A6121F00042B2F1804F0CD0C6
:1047E800B1F1004F09D0394ED6F8082701F47011FD
:1047F80022F470120A43C6F808275A69666BA16B3F
:1048080022F0070232435A615A6922F0700242EAE2
:1048180001125A61002835D19A6A62F00F029A6231
:104828005B6903F007039E423CD10023E365A36D57
:1048380023F0030343F00103A365284603B0F0BD4A
:104848009A68234922F0104222F0170242F080525F
:104858009A60204A1268B2FBF1F2013252000192CA
:10486800019A002A3FF44BAF019A013AF7E7002575
:1048780052E7A16D41F02001A165E16D41F0010110
:10488800E16581E7B0F5001FCAD19A6AE269013A89
:1048980092006FF00F0102F01C0201FA02F2216E81
:1048A8000A43BCE7A36D23F0120343F01003A3658A
:1048B800E36D43F00103E3650125BEE7A36D43F013
:1048C8001003A365F8E700BF02FCFF1F00200140AA
:1048D800400D0300B8000020F8B54569082D0446CE
:1048E8000E460AD00368DB68D80705D5A36D43F0E8
:1048F8002003A3650120F8BD0425FEF7F1F807465B
:1049080023681A682A4221D0A26D42F40072A26577
:10491800DA6812F4406F14D1A27E92B91A681207AD
:104928000FD51846FFF7D4FE28BB5A6822F00C02B0
:104938005A60A26D22F4807222F0010242F0010254
:10494800A265207E00BB0C221A60D4E7711CD8D067
:10495800FEF7C6F8C01BB04201D8002ED0D123689C
:104968001B682B40CCD1A26D84F8543042F004026D
:10497800A2650320BFE7A26D42F02002A265E26DA6
:1049880042F00102E265DCE70020B4E70368186C36
:1049980070470000F7B50023019390F85430012BBD
:1049A800044600F0C58005680669012380F8543084
:1049B8002846FFF78DFE002840F0B480D1E900209A
:1049C800022826F0040300F08280B3F1004FC2F3FE
:1049D800110E13D1AB6A43EA0E03AB628B686869A8
:1049E80003EA022323F07C4323F0FF0320EA022199
:1049F8000B43002A6B6126DB002055E0236E00F094
:104A08001F074FF00F0C0CFA07FC6FEA0C0623EA9D
:104A18000C0CBEF1000F11D1C2F38463BB4043EA12
:104A28000C0323668008E36901309842D6D8A86A47
:104A3800C2F38363BB4006403343CEE792FAA2F346
:104A4800B3FA83F3EAE73B493B48D1F80837824297
:104A580003F0E07519D11B02CED4D1F8083723F042
:104A6800E0732B4343F40003C1F80837334B1A684B
:104A7800334BB2FBF3F20C2302FB03330193019B8C
:104A8800002BB9D0019B013BF8E72E48824210D198
:104A980013F08070B0D1D1F8083723F0E0732B43BE
:104AA80043F08073C1F80837002384F8543003B00A
:104AB800F0BD254882429FD113F480009CD1D1F8E3
:104AC800083723F0E0732B4343F48003EAE7B3F19C
:104AD800004F01BFAB6AC2F311018B43AB62002ADE
:104AE8008ADA154813498242D1F8083709D1D1F832
:104AF800082703F0A07322F0E0721343C1F80837C7
:104B08007AE71048824204D1D1F8082703F4400319
:104B1800F1E70D4882427FF46FAFD1F8082703F020
:104B2800C073E8E7A26D42F02002A2651846BBE711
:104B38000220BCE700200140001000B0B8000020AF
:104B4800400D0300004000B8002000B4026838B5EA
:104B580004461046FFF7BCFD08B9002038BD93682D
:104B6800990707D4936823F0004323F0170343F011
:104B780010039360FDF7B4FF054623689B685B0745
:104B8800EBD5FDF7ADFF401B0228F6D923689B68DB
:104B98005A07F2D5A36D43F01003A365E36D43F004
:104BA8000103E3650120D9E773B500230268019387
:104BB8009368DD07044602D5002002B070BD9168F5
:104BC800214B194209D0A36D43F01003A365E36D8F
:104BD80043F00103E3650120EFE7936823F0004306
:104BE80023F0170343F001039360184BD3F80837F9
:104BF80018021CD4637E012BDED0FDF771FF144E22
:104C0800054622681368DB07D6D49368D9075FBFC7
:104C18009368334043F001039360FDF761FF401B45
:104C28000228EED923681B68DA07EAD4CBE7094BD8
:104C3800094A1B68B3FBF2F301330193019B002B74
:104C4800D8D0019B013BF8E7170000800020014005
:104C5800E8FFFF7FB8000020400D030038B5044688
:104C68000068FFF735FD054620BB94F85430012B4A
:104C780020D0012384F854302046FFF795FFB0B9BF
:104C8800A36D226823F4706323F0010343F4807357
:104C9800A3651C23E065136084F85400936823F02F
:104CA800004323F0170343F00403936038BD84F8EE
:104CB8005450FBE70220F9E7026838B59368916819
:104CC8000446C80701D4002038BD9907FBD493686F
:104CD80003F00503012B19D1936823F0004323F057
:104CE800170343F00203936003231360FDF7F8FEF4
:104CF800054623689B68DB07E5D5FDF7F1FE401BF9
:104D08000228F6D923689B68DA07F2D5A36D43F029
:104D18001003A365E36D43F00103E3650120D3E7C6
:104D280070B5044600284BD0836D43F002038365B9
:104D3800FFF70CFF054668B92046FFF7BDFF05469B
:104D480008B90123A3652268936823F0104323F070
:104D58001703936023685A6822F4677222F00302EB
:104D68005A6040F29F321A60D968164A0A40DA60DF
:104D78001A6922F040421A615A6922F007025A6100
:104D88001A6A02F0F0221A625A6A02F0F0225A6293
:104D9800DA6A02F0F022DA629A6A0B4A00269E6208
:104DA800D2F8083723F0FE73C2F808372046FDF71B
:104DB80069F8E6652666A66584F85460284670BDDD
:104DC8000125FBE700023E830020014010B590F862
:104DD8005430012B044615D0012380F85430FFF7D6
:104DE800B5FE58B92046FFF767FF38B9A36D23F41D
:104DF800807323F0010343F00103A365002384F8C3
:104E0800543010BD0220FCE7F7B50023019390F859
:104E18005430012B04467FD0012380F85430FFF72B
:104E28004BFF23689A6812F00102054607D0A36D6C
:104E380043F01003A365002384F854302DE0A16DDE
:104E4800364F21F4817141F00201A165DE68D9680D
:104E580026F4FF4626F07C0621F40041360421F0B2
:104E68000301360CD96008209968394041F00041A7
:104E780099609968002913DA019901310191019922
:104E8800B1F52E3FF5D3A36D23F0120343F01003C1
:104E9800A365002384F854300125284603B0F0BDEB
:104EA800D3F8B410013801F07F010A44DCD19968C5
:104EB8001A48014041F001019960D3F8B41021F07B
:104EC8007F0141EAD202C3F8B4209A68024042F056
:104ED80002029A60FDF704FE074623689A68D20723
:104EE80008D4DA683243DA60A36D23F0030343F091
:104EF80001039FE7FDF7F4FDC01B0228EDD92368E5
:104F08009B68D907E9D5A36D43F01003A365E36D4A
:104F180043F00103E365BFE70225BEE7E8FFFF7F33
:104F28000749CA6822F4E0620302120403F4E0634A
:104F3800120C134343F0BF6343F40033CB60704754
:104F480000ED00E0164B30B5DC68C4F30224C4F170
:104F58000703251D042B28BF0423062D4FF0FF351A
:104F68008CBF033C002405FA03F321EA0303A540A0
:104F780022EA0502A340002843EA0203ACBF00F17D
:104F88006040084A4FEA0313B8BF00F00F00DBB2D5
:104F9800AABF00F56140135480F8003330BD00BF4C
:104FA80000ED00E014ED00E0002807DB044A4109A9
:104FB800012300F01F00834042F82130704700BFF2
:104FC80000E100E000280CDB4309064900F01F005F
:104FD80020330122824041F82320BFF34F8FBFF3D3
:104FE8006F8F704700E100E070B5D0E91345656048
:104FF800446D14B1D0E916456560D0E9105404F049
:105008001C060124B4406C60046863608368102B3C
:105018000BBFA260A160E160E26070BD0268416CF4
:10502800D3B210B5083B1424B3FBF4F30B4CA242E3
:1050380088BF0B4A21F0030199BF01F1804202F5B4
:105048000232521807338264064AC26403F01F030F
:10505800012202FA03F3036510BD00BF07040240F2
:105068001C0802408008024038B500285ED002685B
:105078002F4B9A424FF014014CD82E4B1344B3FBDC
:10508800F1F32D499B00C0E91013022380F8253065
:105098001368056923F4FF4323F070031360D0E914
:1050A800024323432B43456911682B4385692B43EE
:1050B800C5692B43056A2B430B431360FFF7AEFF0B
:1050C800B4F5804F04BF002343604268816C02F04E
:1050D8007F030B60D0E91314013A032A4C6020D8EF
:1050E800164A174981651A44013B9200012103F0D1
:1050F800030301FA03F300214265C3651160114AF5
:10510800536400230122C36380F8243080F82520EB
:10511800184638BD0C4B1344B3FBF1F30B499B0005
:10512800B1E70023C0E91533C365EAE70120F0E7DA
:1051380007040240F8FFFDBF000002403F82001054
:105148004009024000090240F8FBFDBF000402408C
:1051580038B5002841D00268136823F001031360B2
:105168001F4B9A424FF0140130D81E4B1344B3FB27
:10517800F1F31D499B00C0E91013012403F01C033F
:1051880004FA03F3002515604B60FFF747FF836CB3
:1051980041681D60D0E913325A604A1E032A06D8B6
:1051A800124B0B449B0094401D60114B5C64002320
:1051B800C363C0E91533C0E90B33C0E90D33C365D8
:1051C80080F8253080F82430184638BD094B134440
:1051D800B3FBF1F308499B00CDE70120F5E700BFD9
:1051E80007040240F8FFFDBF000002403F820010A4
:1051F80000090240F8FBFDBF0004024070B590F8BA
:105208002450012D04463BD090F825600125AE427C
:1052180080F824504FF000062CD1022580F8255044
:105228000568C6632E6826F001062E60FFF7DCFECF
:10523800036BBBB12B6843F00E032B60A36C1A6899
:10524800D20342BF1A6842F480721A60636D1BB1C0
:105258001A6842F480721A602B6843F001032B60CD
:10526800002070BD2B6823F004032B602B6843F0EB
:105278000A03E2E78023C36380F824602846F0E746
:105288000220EEE7034640B190F82520022A06D016
:105298000422C263002280F824200120704702689B
:1052A800806C116821F00E011160016821F4807191
:1052B8000160116821F001011160D3E9100202F0C8
:1052C8001C0101228A404260D3E9132151605A6DC2
:1052D80032B1116821F480711160D3E9162151604F
:1052E8000122002083F8252083F82400704710B598
:1052F80090F82530022B03D00423C363012010BD8E
:1053080003681A6822F00E021A601A6822F0010275
:105318001A60826C136823F480731360D0E9101349
:1053280003F01C02012393404B60D0E913325A600A
:10533800436D33B11A6822F480721A60D0E91632CC
:105348005A60012380F82530836B002480F82440BC
:1053580013B198472046D2E71846D0E770B4426C9C
:10536800046C036826681D6802F01C020421914041
:1053780031420FD015F0040F0CD01A6892065EBFA8
:105388001A6822F004021A60036B6160002B33D0A4
:1053980070BC184702219140314217D015F0020F16
:1053A80014D01A68940606D41A6822F00A021A6001
:1053B800012280F82520114A93428CBF104B114BD3
:1053C8005960002380F82430C36ADFE70821914040
:1053D800314211D029070FD5196821F00E01196043
:1053E800012303FA02F26260C36380F825300023C8
:1053F80080F82430436BC9E770BC704780000240D6
:1054080000040240000002400A4A536943F4802322
:1054180030B55361EFF3108472B60023CD58C550F0
:105428000433B3F5807FF9D11369DB03FCD484F32B
:10543800108830BD00400058064B5A69002ABFBF8B
:10544800054A9A6002F188329A60BABF5869C00F5B
:10545800002070470040005823016745044B5A69F3
:1054680042F000425A615869C043C00F704700BFFC
:105478000040005870B50546FDF732FB124E044651
:105488003369D90313D43369DA0744BF012232617F
:105498004CF2FA32134011D10B4E306910F48020CF
:1054A8000BD0FDF71DFB001BA842F6D304E0FDF767
:1054B80017FB001BA842E3D3032070BD024A136107
:1054C800024A01205360F8E7004000581407002002
:1054D8002DE9F041184D98462B78012B06460C46CD
:1054E800174626D001232B704FF47A7000236B6087
:1054F800FFF7C0FFA0B9012E16D1104A536943F037
:10550800010353612760BFF36F8FC4F804804FF421
:105518007A70FFF7AFFF094A536923EA060353611C
:1055280000232B70BDE8F08139462046FFF76CFF59
:10553800EDE70220F6E700BF1407002000400058FE
:10554800054A536923F47E7343EAC00040F480306F
:1055580040F0020050617047004000582DE9F041CA
:10556800234F3B78012B054688463FD001233B70EB
:105578004FF47A7000237B60FFF77CFF044688B9FC
:105588002B68042B13D11B4A536943F4803343F02F
:10559800040353614FF47A70FFF76CFF0446154B10
:1055A8001A681B6800233B702046BDE8F0814FF065
:1055B800FF33C8F800306E68D5E901321344B342AE
:1055C8000AD93046FFF7BCFF4FF47A70FFF752FF55
:1055D80050B1C8F800600446064A536923F47E7344
:1055E80023F002035361DAE70136E5E70224DBE73B
:1055F80014070020004000582DE9F04F524C0023BA
:105608004FF00F090A6832FA03F501D1BDE8F08FAF
:10561800012505FA03F818EA020200F08E804E68A8
:10562800032706F003054FEA430E07FA0EFC6F1E28
:10563800012F6FEA0C0C32D8876807EA0C0ACF688A
:1056480007FA0EF747EA0A078760476827EA080853
:10565800C6F300179F4047EA08074760C76807EA8C
:105668000C088F6807FA0EF747EA0807022DC7608B
:1056780017D14FEAD30800EB880803F0070AD8F8D7
:1056880020704FEA8A0A09FA0AFB27EA0B0B0F690E
:1056980007FA0AF747EA0B07C8F8207001E0032D5C
:1056A800DCD1076805FA0EF507EA0C073D4316F446
:1056B800403F056041D023F0030707F1804707F515
:1056C800803703F0030CBD684FEA8C0C4FF0070ECF
:1056D8000EFA0CFEB0F1904F25EA0E0E2FD01B4D9E
:1056E800A8422ED005F58065A8420CBF02250725E3
:1056F80005FA0CF545EA0E05BD602568D74316F492
:10570800801F0CBF3D4015432560656816F4001FD7
:105718000CBF3D4015436560D4F8805016F4803FB7
:105728000CBF3D401543C4F88050D4F88450B603EC
:1057380054BF3D401543C4F88450013362E7002547
:10574800D6E70125D4E700BF000800580004004848
:10575800374A2DE9F04F00234FF0010A4FF0070BAD
:105768004FF00F0931FA03F401D1BDE8F08F0AFABE
:1057780003FC1CEA010654D023F0030404F180441E
:1057880004F5803403F00307A568BF000BFA07F897
:10579800B0F1904F08EA050E45D0264DA84244D0F6
:1057A80005F58065A8420CBF02250725BD40754553
:1057B80017D1D2F8805025EA0605C2F88050D2F8F1
:1057C800845025EA0605C2F88450156825EA0605BE
:1057D8001560556825EA06055560A56825EA080597
:1057E800A560056803265C0006FA04F423FA06F6A9
:1057F800254300EB8606056003F00705376AAD0010
:1058080009FA05F527EA05073762856825EA0405D8
:105818008560456825EA0C054560C56825EA0404E5
:10582800C46001339EE70025C0E70125BEE700BF3D
:1058380000080058000400480369194214BF0120F9
:10584800002070470AB1816170478162704700008B
:10585800044AD168014208B502D0D060FEF708F8C2
:1058680008BD00BF0008005810B5044600284AD0FB
:1058780090F8413003F0FF021BB980F84020FCF794
:105888001FFE242384F8413023681A6822F001029D
:105898001A60626822F070621A619A6822F4004203
:1058A8009A60D4E90221012924D142F400429A6085
:1058B8005A6842F0007242F400425A60DA6822F4F0
:1058C8000042DA60D4E904210A43A16942EA0122CC
:1058D800DA60D4E907210A431A601A6842F0010223
:1058E8001A6000202023606484F84130206384F823
:1058F800420010BD42F4044202299A6004BF4FF4EA
:1059080000625A60D4E70120F3E710B590F841200F
:10591800202A0346D4B21CD190F84020012A18D07E
:10592800242280F841200268106820F001001060ED
:10593800106820F4805010601068014311601168ED
:10594800002041F00101116083F8414083F84000D4
:1059580010BD0220FCE710B590F84120202A03462C
:10596800D4B21BD190F84020012A17D0242280F805
:1059780041200268106820F001001060106820F4CF
:10598800706040EA012111601168002041F00101B6
:10599800116083F8414083F8400010BD0220FCE705
:1059A800024A136843F48073136070470004005878
:1059B8000D4B10B55B690C4628B99A0507D500F060
:1059C80027F820B110BD9B0501D400F019F8074A4B
:1059D8001369012C23F00403136101D130BFF1E7EF
:1059E80040BF20BF20BFEDE70004005800ED00E0F5
:1059F800024B186800F4C060704700BF00040058EC
:105A0800024A136843F48043136070470004005847
:105A18000C4A136823F4804313600B4B1B68322134
:105A28004B430A49B3FBF1F35169890500D533B9F2
:105A3800536913F4007F14BF032000207047013B13
:105A4800F2E700BF00040058B800002040420F00F1
:105A58000B4A136823F0070343F002031360094B52
:105A68001A69012842F004021A6105D130BF1A6987
:105A780022F004021A61704740BF20BF20BFF6E73A
:105A88000004005800ED00E04FF0B0431868C0F380
:105A9800404070474FF0B0431868C0F3400070476B
:105AA8004FF0B042536823F47F4343EA0023536026
:105AB80070474FF0B0431868C0F34060704700006B
:105AC8007FB54FF0B0432C4AD3F80831C0F3031028
:105AD80003F00F0352F82040284A52F82330B4FB51
:105AE800F3F4FFF785FF264B054693E80700B5F565
:105AF800007F04AB03E9070010D0224B9C4218D367
:105B080003F5B70303F67F539C4229D903F57413B1
:105B180003F510639C4225D802230BE01A4B9C42E4
:105B280007D91A4B9C421BD903F5370303F5D85301
:105B3800F0E7002304AA02EB830353F80C4C144D3E
:105B48002B6823F0070323432B60FCF7C9FF0646A5
:105B58002B6803F007039C4206D1002004B070BDF7
:105B68000123E7E70024EAE7FCF7BAFF801B0228D5
:105B7800EED90320F2E700BFB81901085819010847
:105B880028110108C0CF6A00BFEA21013F933402FF
:105B9800004000584FF0B04310B59A68D96812F029
:105BA8000C0205D00C2A4AD101F00303012B50D175
:105BB8004FF0B0412B480B6813F0080306D00B6870
:105BC80013F0080337D1D1F8941007E00C682407C4
:105BD80056BFD1F894300968C3F3032350F8233033
:105BE800002A0CBF184600204FF0B0418A6802F026
:105BF8000C020C2A1ED1CA6802F00302022A2ED017
:105C0800032A06D10B68184A13F4801F174B18BFD4
:105C180013464FF0B042D068D168D268C0F306206E
:105C28005843C1F302130133B0FBF3F0530F0133B0
:105C3800B0FBF3F010BD0B68C3F30313CEE7042ADF
:105C48000AD0082A05D11B6813F4801304D1074829
:105C5800CAE700231846C7E703480023C4E7024BF6
:105C6800D7E700BFB81901080024F4000048E8018C
:105C780008B5FFF78FFF4FF0B043044A9B68C3F3A2
:105C8800031352F82330B0FBF3F008BD581901088C
:105C98002DE9F0410446002853D04FF0B0439D68E9
:105CA800DE6803689B0605F00C0506F0030668D558
:105CB800026A1DB10C2D46D1012E44D1002A40D0D4
:105CC8004FF0B043A16A1A68170756BFD3F894304B
:105CD8001B681B0903F0F00399421FD90846FFF718
:105CE800EFFE00282DD14FF0B042136843F00803AF
:105CF80013601368A16A23F0F0030B431360606A12
:105D0800FFF7CEFEFFF7B4FFAB4B1860AB4B18683C
:105D1800FCF7E4FE002834D0BDE8F0814FF0B04233
:105D2800136843F008031360136823F0F0030B4370
:105D38001360606AFFF7B4FE0846FFF7C1FE00284B
:105D4800E0D00120E8E74FF0B043002A54D01A68A9
:105D580042F001021A60FCF7C3FE0746FFF79AFEFD
:105D6800002842D04FF0B042136843F00803136094
:105D78001368A16A23F0F0030B431360606AFFF70E
:105D88008FFE2368D80748D42368990700F18C80D0
:105D980023681E0740F1FA80A3694FF0B046002B34
:105DA80000F0E180D6F89430E16903F010029142E6
:105DB80000F0C48003F00302022AC2D0D80740F1E1
:105DC800B380D6F8943023F00103C6F89430FCF77A
:105DD80087FE0746D6F89430990740F1A580FCF76E
:105DE8007FFEC31B112BF5D904E0FCF779FEC01B1D
:105DF8000228B3D903208FE71A6822F001021A603B
:105E0800FCF76EFE0746FFF745FE0028B9D0FCF701
:105E180067FEC01B0228F6D9ECE7082D03D00C2D2D
:105E280005D1032E03D16368002BADD189E74FF06C
:105E3800B043A1681A6822F480120A431A606268A3
:105E4800B2F5803F10D11A6842F480321A60FCF72C
:105E580047FE0746FFF718FE002895D1FCF740FEDD
:105E6800C01B6428F6D9C5E7B2F5041F04D11A6827
:105E780042F400121A60E6E7196821F480311960CB
:105E8800196821F400111960002AE0D1FCF728FEF6
:105E98000746FFF7F9FD00283FF476AFFCF720FE30
:105EA800C01B6428F5D9A5E7042D236903D00C2D60
:105EB8000ED1022E0CD1002B3FF443AF4FF0B0426D
:105EC8006169536823F0FE4343EA016353605FE767
:105ED8004FF0B046BBB1336843F480733360FCF7CE
:105EE800FFFD074633685A0507D57368626923F0D2
:105EF800FE4343EA026373604AE7FCF7F1FDC31B04
:105F0800022BEFD976E7336823F480733360FCF70C
:105F1800E7FD074633685B057FF53AAFFCF7E0FD20
:105F2800C31B022BF6D965E74FF0B042E169D2F8FE
:105F3800943023F010030B43C2F894304FF0B0476D
:105F4800D7F8943043F00103C7F89430FCF7C8FD44
:105F58000646D7F894309A0718D4FCF7C1FD831B7E
:105F6800112BF6D946E7D6F8943023F00103C6F88A
:105F78009430FCF7B5FD0746D6F894309B0705D555
:105F8800FCF7AEFDC31B112BF6D933E7236858077E
:105F980054D50B4F3B68D90514D4FFF701FDFCF726
:105FA8009FFD06463B68DA050CD4FCF799FD831B78
:105FB800022BF7D91EE700BFB8000020BC00002064
:105FC80000040058E3684FF0B046002B58D023F087
:105FD8008003052B02BFD6F8903043F00403C6F8BF
:105FE80090304FF0B046FCF77BFDD6F8903043F088
:105FF80001030746C6F8903041F28838D6F8903049
:106008009B0705D4FCF76CFDC31B4345F6D9F1E6A5
:10601800E36823F00403812B1BD1FCF761FDD6F85C
:10602800903043F08003C6F8903007464FF0B046F2
:1060380041F28838D6F89030180504D5E06A00286F
:106048004AD1002068E6FCF74BFDC01B4045F1D95A
:10605800D0E6FCF745FDD6F8903023F08003C6F86B
:10606800903007464FF0B04641F28838D6F8903065
:106078001905E3D5FCF734FDC01B4045F6D9B9E650
:10608800FCF72EFDD6F8903023F080030746C6F8BB
:10609800903041F28838D6F890301A0516D4FCF7BB
:1060A8001FFDD6F8903023F00103C6F8903007465C
:1060B8004FF0B04841F28836D8F890309B07BDD5EC
:1060C800FCF70EFDC31BB342F6D993E6FCF708FDB7
:1060D800C01B4045DFD98DE60C2D4ED04FF0B043A4
:1060E80002281A6822F080721A6033D1FCF7F8FC93
:1060F8000546FFF7DEFC38BBD4E90C314FF0B0425F
:106108000B43D0682D4901400B43E16B0B43216CD5
:106118000B43616C0B43A16B43EA0123D360136803
:1061280043F080731360D36843F08053D360FCF767
:10613800D7FC0446FFF7BDFC002882D1FCF7D0FC51
:10614800001B0A28F6D955E6FCF7CAFC401B0A28AA
:10615800CFD94FE6FCF7C4FC0446FFF7AAFC30B9D8
:106168004FF0B042164BD1680B40D360D4E5FCF732
:10617800B7FC001B0A28F0D93CE601283FF4CCAD57
:106188004FF0B043226BDB6803F0030191427FF4C8
:10619800D8AD616B03F070028A427FF4D2ADA16B77
:1061A80003F4FE42B2EB012F7FF4CBAD626C03F037
:1061B800604393423FF445AFC3E500BF8C80C111F3
:1061C800FCFFFEEE2DE9F0410D46044610B9012012
:1061D800BDE8F081684E336803F007038B4216D39D
:1061E80023689A0727D54FF0B047A268BB6823F009
:1061F800F0031343BB60FCF773FC0646BB68DB0384
:1062080019D4FCF76DFC831B022BF7D911E0336816
:1062180023F007030B433360FCF762FC074633683F
:1062280003F00703AB42DBD0FCF75AFCC01B022883
:10623800F5D90320CCE72368580617D54FF0B047A7
:106248006269D7F8083123F00F0343EA1213C7F83D
:106258000831FCF745FC0646D7F80831D90305D4C0
:10626800FCF73EFC831B022BF6D9E2E723685A07AA
:1062780013D54FF0B047E268BB6823F4E0631343DB
:10628800BB60FCF72DFC0646BB689B0305D4FCF7F6
:1062980027FC831B022BF7D9CBE72368180714D5F3
:1062A8004FF0B0472269BB6823F4605343EAC20346
:1062B800BB60FCF715FC0646BB68590305D4FCF720
:1062C8000FFC831B022BF7D9B3E72368DA070FD437
:1062D800294C236803F00703AB4239D8FFF7C8FC01
:1062E800264B1860264BBDE8F0411868FCF7F6BB52
:1062F8006268022A1DD1FFF7C7FB00283FF467AF89
:106308004FF0B04641F28838B36823F003031343D3
:10631800B360FCF7E5FB0746B368626803F00C035B
:10632800B3EB820FD4D0FCF7DBFBC01B4045F3D99D
:106338007FE7032A02D1FFF7BCFBDEE712B9FFF7BC
:10634800A9FBDAE74FF0B0431B685B05D8D43EE7FA
:10635800236823F007032B432360FCF7C1FB0646A1
:10636800236803F00703AB42B8D0FCF7B9FB801BE6
:106378000228F5D95DE700BF00400058B8000020AA
:10638800BC00002008B5FFF773FC4FF0B043044A87
:106398009B68C3F3022352F82330D84008BD00BFDE
:1063A8009819010808B5FFF763FC4FF0B043044A99
:1063B8009B68C3F3C22352F82330D84008BD00BFFE
:1063C800981901084FF0B043D3F89000C0F340008B
:1063D80070474FF0B0410209D1F8883002F47F22AB
:1063E800000123EA020300F47F200343C1F8883048
:1063F80070474FF0B041020CD1F88830120423EAFC
:10640800020343EA0040C1F88800704770B5066887
:1064180016F48036044638D0FFF7C2FAFCF760FB62
:10642800614E05463368DB0529D54FF0B043616BF3
:10643800D3F8902002F44072914214D0D3F890100F
:10644800D3F8902042F48032C3F89020D3F89020FB
:1064580021F4407022F480328D07C3F89020C3F8ED
:10646800900000F190804FF0B042616BD2F890300C
:1064780023F440730B43C2F89030002605E0FCF784
:106488002FFB401B0228CDD903262568E8070AD52B
:106498004FF0B0416268D1F8883023EA124392B2D3
:1064A8001343C1F88830A9070AD54FF0B041A26854
:1064B800D1F8883023EA124392B21343C1F88830E6
:1064C800AA0609D54FF0B0422169D2F8883023F4E2
:1064D80040630B43C2F88830AB0502D5206AFFF74A
:1064E80088FF680502D5606AFFF783FF290502D592
:1064F800A06AFFF77EFF6A0602D56069FFF769FFA9
:106508002B0602D5A069FFF764FFE80502D5E0690C
:10651800FFF75FFFE90610D54FF0B042E168D2F807
:10652800883023F440730B43C2F88830B1F5807F7C
:1065380002BFD36843F08073D3602A040ED54FF0AE
:10654800B042216BD2F8883023F040430B43C2F8A5
:10655800883019B9D36843F08073D3606B0410D5C1
:106568004FF0B042E16AD2F8883023F040530B4331
:10657800B1F1005FC2F8883003D1D36843F48033A7
:10658800D360304670BDFCF7ABFA41F28836054659
:10659800FFF718FF01283FF466AFFCF7A1FA401B8C
:1065A800B042F5D970E700BF0004005830B590F844
:1065B8002C30012B02464FF0020022D0174B82F8F4
:1065C8002D00CA24012582F82C505C6253245C6299
:1065D800B1F5807F146B996914D121F488519961C0
:1065E800596C24F0010421F0004159641463DD65FD
:1065F8000A4BFF2159620020012382F82D3082F8CE
:106608002C0030BD21F408519961D96C24F00204A2
:1066180021F00041D9641463D865E9E700280040F7
:1066280070B50B4E036B756D1D40EA07044603D524
:106638000123F365FCF7C5FBAB0704D50223F3651B
:10664800204600F0CBF9012384F82D3070BD00BF3F
:106658000028004038B50A4CE36823F02003E360C3
:10666800FCF73EFA0546E3689B0601D5002038BDD5
:10667800FCF736FA401BB0F57A7FF4D90320F6E729
:10668800002800402DE9F041114DEC6814F0400459
:1066980007461AD1EB6843F08003EB60FCF720FA59
:1066A8004FF003080646EB685B0601D4032C02D1C1
:1066B8002046BDE8F081FCF713FA801BB0F57A7F1D
:1066C80084BF87F82D800324EDE70024F0E700BF9E
:1066D8000028004038B50F4CE36823F08003E360DE
:1066E800A3699B06054606D4FFF7B4FF10B1032043
:1066F80085F82D0038BDA36923F02003A361FFF7B7
:10670800A9FF10B1032085F82D00A36943F02003E9
:10671800A361EFE70028004038B5044600284BD0B5
:1067280090F82D3003F0FF021BB980F82C20FBF7FE
:10673800D5FF0223214D84F82D30EB68DB0632D4D7
:10674800CA236B6253236B622046FFF79BFF78BB1B
:10675800AB6923F08E6323F04003AB612169636862
:10676800AA690B431343A2691343AB61D4E902231B
:1067780043EA02432B61D4E90931EA680B4322F466
:10678800F8521343EB602046FFF7A4FF80B9D4E921
:106798000713AA690B4322F060421343626913434B
:1067A800AB61FF236B62012384F82D30002002E0E7
:1067B800024BFF225A6238BD0120FCE70028004046
:1067C8000023092803D840EA0310C0B270470A38EA
:1067D8000133C0B2F5E700002DE9F04790F82C30FE
:1067E800012B05464FF0020069D0012385F82C30B3
:1067F8004E4B85F82D00DE6806F44076B6F5807FAE
:1068080078D04C69087891F8019091F802A091F835
:106818002470002A55D19B6913F0400308BFCB7040
:10682800FFF7CEFF80464846FFF7CAFF02465046AC
:10683800FFF7C6FF81463846FFF7C2FF0B6ACF78DD
:10684800234343EA875343EA090343EA084343EAF5
:10685800022343EA0063354ACA205062532050623B
:106868008C6A8869B4F5807F946945D124F488548A
:1068780094610124D465B6F5807F09BFCB691364A0
:106888000343536418BF5064284B4A681A672A6B3D
:1068980042F001022A639A6942F488529A61244AB2
:1068A800D2F8803043F40033C2F880301F4BFF2207
:1068B8005A620020012385F82D3085F82C00BDE8A8
:1068C800F087B4F1803F07D0B4F5000F04D09B697E
:1068D80013F0400308BFCB700B6ACA781C4344EA24
:1068E8000A0444EA004343EA092343EA825343EA99
:1068F8000763B0E70023AEE724F408549461022448
:10690800D465B6F5807F09BFCB6993640343D3642C
:1069180018BFD064054B4A685A672A6B42F00202D6
:106928002A639A6942F40852B8E700BF0028004079
:106938000008005890F82C20012A03464FF0020066
:1069480012D00A4A83F82D00CA215162532151629C
:10695800916941F020019161FF21516200200122DB
:1069680083F82D2083F82C00704700BF00280040D2
:1069780090F82C20012A03464FF0020019D00D4A46
:1069880083F82D00CA2151625321516291690A4846
:1069980041F080019161D0F8801041F48021C0F865
:1069A8008010FF2151620020012283F82D2083F8F6
:1069B8002C0070470028004000080058064B5A6D0C
:1069C800520610B5044603D54022DA65FCF7FCF9F7
:1069D800012384F82D3010BD00280040704789003D
:1069E80001F1804101F531410A607047890001F1E8
:1069F800804101F53141086870470000034AD2F828
:106A0800903043F40043C2F89030704700040058B7
:106A1800034AD2F8903023F40043C2F8903070470C
:106A280000040058074B1A6822F040021A6040F42C
:106A380041704FF4B85218605A601A6842F0400228
:106A48001A6070470000015837B5054600284ED037
:106A5800837903F0FF046BB1032C0BD0254B4FF463
:106A680000629A612868FFF7DDFF002401232B717B
:106A7800AC602FE000236B712846FBF747FF1E4AE6
:106A8800D2F8903043F48053C2F89030002CE5D10E
:106A980002234FF0B042AB71D2F8943023F4004394
:106AA800C2F89430154B1B681C214B43DB0C642146
:106AB8004B430193019B93B90124AC60FFF79EFF00
:106AC8000C4B9A6842F400629A604FF400629A6133
:106AD800002CC7D00123AB71204603B030BD019B09
:106AE800013B0193D2F894305B04E3D4E6E7012438
:106AF800F2E700BF0004005800080058B800002062
:106B080037B5174D2B6802461C204343DB0C642025
:106B1800434314480193019B93B901209060114CA1
:106B280021732B681C214B43DB0C64214B430193DD
:106B3800019B6BB9012090600A4BDB6803B030BD44
:106B4800019B013B019383689C07E4D50020E6E79D
:106B5800019B013B0193A368DB07E9D5ECE700BF84
:106B6800B80000200000015837B5184D2B680246C0
:106B78001C204343DB0C6420434315480193019BCD
:106B8800A3B901209060124CFF2323732B681C25A6
:106B98006B43DB0C64256B430193019B73B90120A4
:106BA80090600B4BDB680B7003B030BD019B013B61
:106BB800019383689C07E2D50020E4E7019B013B31
:106BC8000193A368DB07E8D5EBE700BFB800002016
:106BD800000001580F4B13B51B680F4C1822534384
:106BE8001B0D64225343014601936269019B02F025
:106BF800040223B902238B60012002B010BD019B5F
:106C0800013B0193606910F00200F6D0002AECD134
:106C18001046F2E7B80000200004005807B50379D1
:106C2800012B0FD10A4B1B68182253431B0C0193ED
:106C3800FFF7EEFE019B013B0193019B002BF9D16D
:106C4800FFF7DCFE03B05DF804EBFFF7C3BF00BF3E
:106C5800B8000020F8B51E468379012B1546044676
:106C68000F46DAB22DD14379012B2AD00223427183
:106C78008371FFF7D3FF0D212046FFF7C9FEFFF709
:106C88003FFF390A2046FFF73BFFF9B22046FFF7DE
:106C980037FF2E44B5420ED12046FFF7AFFEFFF76F
:106CA80099FFA06801230038A3714FF0000318BFB3
:106CB80001206371F8BD15F8011B2046FFF720FF7E
:106CC800E8E70220F6E7F8B51E468379012B15465A
:106CD80004460F46DAB22FD14379012B2CD04271EA
:106CE800FFF79CFF1D212046FFF792FEFFF708FFE4
:106CF800390A2046FFF704FFF9B22046FFF700FFE4
:106D080000212046FFF7FCFE2E44B5420ED1204656
:106D1800FFF774FEFFF75EFFA06801230038A37138
:106D28004FF0000318BF01206371F8BD29462046C3
:106D3800FFF71AFF0135E8E70220F6E7F8B51F4626
:106D48008379012B154604460E46DAB22CD14379D5
:106D5800012B29D04271FFF761FF06F0EF03A3F181
:106D6800840253425341237131462046FFF750FEB7
:106D7800FFF7C6FE2F44AF4210D1FFF73FFE842E27
:106D880002D02046FFF726FFA06801230038A37130
:106D98004FF0000318BF01206371F8BD15F8011BFF
:106DA8002046FFF7ADFEE6E70220F6E7F8B51E46F7
:106DB8008379012B154604460F46DAB227D1437969
:106DC800012B24D04271FFF729FF39462046FFF7EF
:106DD8001FFEFFF795FE00212046FFF791FE2E4487
:106DE800B5420ED12046FFF709FEFFF7F3FEA06873
:106DF80001230038A3714FF0000318BF012063710D
:106E0800F8BD29462046FFF7AFFE0135E8E7022026
:106E1800F6E737B50023ADF8043001AA02231221A2
:106E28000546FFF7C3FFBDF80440022364BA01AA70
:106E3800A4B219462846FFF781FFE20702D5284683
:106E480009F0F6F9A30702D5284609F0F7F9600713
:106E580002D5284609F01CFA210702D5284609F070
:106E68001DFAE20602D5284609F01EFAA30602D545
:106E7800284609F007FA600602D5284609F0E4F921
:106E8800210606D514F4807118BF0121284609F09F
:106E9800E1F9A20502D5284609F0ECF9630402D508
:106EA800284609F007FA03B030BDF8B51E468379C5
:106EB800012B154604460F46DAB227D14379012B38
:106EC80024D04271FFF7AAFE0E212046FFF7A0FD4D
:106ED800FFF716FE39462046FFF712FE2E44B5424C
:106EE8000ED12046FFF78AFDFFF774FEA068012344
:106EF8000038A3714FF0000318BF01206371F8BD7B
:106F080015F8011B2046FFF7FBFDE8E70220F6E72E
:106F1800F8B51E468379012B154604460F46DAB2AA
:106F28002BD14379012B28D04271FFF777FE1E2120
:106F38002046FFF76DFDFFF7E3FD39462046FFF7D2
:106F4800DFFD00212046FFF7DBFD2E44B5420ED1C0
:106F58002046FFF753FDFFF73DFEA06801230038E8
:106F6800A3714FF0000318BF01206371F8BD2946D3
:106F78002046FFF7F9FD0135E8E70220F6E7026849
:106F880052E8003F23F0C00342E8003102680029BC
:106F9800F5D102F1080353E8003F23F4000302F19E
:106FA800080C4CE800310029F3D12023C0F88830C0
:106FB8007047000010B5026852E8003F23F4907350
:106FC80042E8003102680029F5D10F4C02F10803AC
:106FD80053E8003F234002F1080C4CE80031002937
:106FE800F4D1C36E012B07D152E8003F23F0100300
:106FF80042E800310029F7D12023C0F88C30002363
:10700800C366436710BD00BFFEFFFFEFF8B5044637
:107018001346D4F88850202D32D1F1B1EAB1E06F8F
:10702800A4F85620A4F8542000262122C4F8906021
:107038002165C4F88820226888B1124FC762124FB0
:107048000763124F2832C0E90D76FEF7D7F830B142
:107058001023C4F89030C4F8885001200FE023684A
:1070680040221A62226802F1080353E8003F43F005
:10707800800302F1080141E800300028F3D1F8BD8F
:107088000220FCE799700008E1700008ED70000824
:1070980008B50346806A1B681B6813F0200317D1E4
:1070A800A0F85630026802F1080353E8003F23F0C5
:1070B8008003083242E8003102680029F2D152E820
:1070C800003F43F0400342E800310029F7D108BDF2
:1070D800FBF7D0FFFBE7704708B5806AFFF7FBFFB7
:1070E80008BD7047806A38B50468D0F88830D0F891
:1070F8008C50A268120606D5212B04D10023A0F8D3
:107108005630FFF73CFFA3685B0606D5222D04D155
:107118000023A0F85E30FFF74DFFD0F8903043F021
:107128001003C0F89030FFF7DCFF38BD08B5806A5F
:107138000023A0F85E30A0F85630FFF7D2FF08BD54
:10714800704700000368D9691A682DE9F04140F6D4
:107158000F0631429D68044610D18E0640F1978093
:1071680002F0200605F080573E4300F09080436F00
:10717800002B00F08580BDE8F0411847AB4EAC48C5
:107188002E401040304300F08280CF0709D5D0054B
:1071980007D501201862D4F8900040F00100C4F827
:1071A80090008F0709D5E80707D502201862D4F8A0
:1071B800900040F00400C4F890004F0709D5E80794
:1071C80007D504201862D4F8900040F00200C4F8F3
:1071D80090000F070BD502F02000304307D008209D
:1071E8001862D4F8900040F00800C4F890000E052A
:1071F8000AD5500108D54FF400601862D4F89030D1
:1072080043F02003C4F89030D4F89030002B37D0E6
:107218008B0609D502F0200205F080552A4303D0D9
:10722800636F0BB1204698472668D4F89020B3685E
:1072380002F0280203F0400353EA0205204621D059
:10724800FFF7B8FEB3685F0617D5226802F1080396
:1072580053E8003F23F04003083242E80031002998
:10726800F3D1D4F8800040B1724B8363FEF73FF846
:1072780030B1D4F88000836B7DE72046FFF731FFFB
:10728800BDE8F081FFF72DFFC4F89050F8E7E06EF5
:10729800012840F08980CE0640F18680D00640F172
:1072A800838010221A629A6851064BD5D4F8802040
:1072B80011684A6892B2002AE2D0B4F85C009042A1
:1072C800DED9A4F85E200A6892062FD453E8002F6E
:1072D80022F4807243E800210029F7D103F1080263
:1072E80052E8002F22F0010203F1080040E80021D3
:1072F8000029F3D103F1080252E8002F22F04002DE
:1073080003F1080040E800210029F3D12022C4F845
:107318008C20E16653E8002F22F0100243E8002198
:107328000029F7D1D4F88000FDF7ACFF02232367CA
:10733800B4F85E30B4F85C10C91A89B22046FFF779
:10734800FFFE9DE7B4F85E20B4F85E00B4F85C1068
:1073580080B292B2002893D0891A89B200298FD0BE
:1073680053E8002F22F4907243E800200028F7D158
:10737800314D03F1080252E8002F2A4003F10806B4
:1073880046E800200028F4D12022C4F88C20606749
:10739800E06653E8002F22F0100243E8002000289E
:1073A800F7D102232367C9E7CF0209D56E0207D5B3
:1073B8004FF4801220461A62BDE8F04100F0A0BDEB
:1073C80008060BD502F0800005F40005284305D017
:1073D800A36F002B3FF454AF2046CCE64F0611D5DF
:1073E80056060FD553E8002F22F0400243E800214B
:1073F8000029F7D12023C4F88830A1672046FBF77D
:1074080039FE3DE70D0206D5500004D52046BDE8FB
:10741800F04100F077BDCB017FF532AF002ABFF60F
:107428002FAF2046BDE8F04100F06BBD0100001011
:107438002001000435710008FEFFFFEFD0F88C2012
:10744800B0F86010222A08B5036855D15B6A826DCE
:107458000B401370836D01338365B0F85E30013BD8
:107468009BB2A0F85E30B0F85E309BB2002B42D1E0
:10747800026852E8003F23F4907342E80031036841
:107488000029F5D103F1080252E8002F22F0010289
:1074980003F1080C4CE800210029F3D12022C0F8A0
:1074A8008C20184A41679342016705D1C26E012AB0
:1074B8000ED0FBF7EDFD1EE05A681102F6D553E831
:1074C800002F22F0806243E800210029F7D1EDE780
:1074D8000022C26653E8002F22F0100243E8002180
:1074E8000029F7D1DA69B0F85C10D20644BF10223F
:1074F8001A62FFF725FE08BD9A6942F008029A61F0
:10750800F9E700BF00800040D0F88C20B0F8601088
:10751800222A08B5036852D15A6A1140826D22F8AE
:10752800021B8265B0F85E20013A92B2A0F85E2094
:10753800B0F85E2092B2002A40D153E8002F22F41E
:10754800907243E800210029F7D103F1080252E8BC
:10755800002F22F0010203F1080C4CE80021002959
:10756800F3D12022C0F88C20174A41679342016763
:1075780005D1C26E012A0ED0FBF78AFD1EE05A68BB
:107588001102F6D553E8002F22F0806243E800216B
:107598000029F7D1EDE70022C26653E8002F22F058
:1075A800100243E800210029F7D1DA69B0F85C102D
:1075B800D20644BF10221A62FFF7C2FD08BD9A69BD
:1075C80042F008029A61F9E7008000402DE9F74F80
:1075D8000368B0F86080DF691A689D68D0F88C107D
:1075E80001922229044640F0B480B0F86890DFF890
:1075F8006CA1DFF86CB10026B9F1000F01D0BB0611
:1076080021D4B4F85E309BB2D3B1B4F868209A4262
:1076180016D9226802F1080353E8003F23F080538B
:10762800083242E8003122680029F2D14D4B6367E5
:1076380052E8003F43F0200342E800310029F7D127
:1076480003B0BDE8F08F2368A26D5B6A03EA080304
:107658001370A36D0133A365B4F85E30013B9BB290
:10766800A4F85E302368DF6978072CD0F9070AD5BB
:10767800019AD20507D501211962D4F8901041F07A
:107688000101C4F89010B80709D5E90707D5022108
:107698001962D4F8901041F00401C4F890107A07E8
:1076A80009D5E80707D504211962D4F8903043F0CA
:1076B8000203C4F89030D4F8903023B12046FFF785
:1076C80010FDC4F89060B4F85E309BB2002B93D1E3
:1076D800216851E8003F23F4807341E800302368B3
:1076E8000028F5D103F1080252E8001F01EA0A0157
:1076F80042E800100028F5D120215B45C4F88C1021
:10770800606720670AD05968090207D553E8001F47
:1077180021F0806143E800100028F7D1E16E0129CB
:1077280013D1E66653E8001F21F0100143E800106A
:107738000028F7D1D969CA0644BF1021196220462A
:10774800B4F85C10FFF7FCFC56E72046FBF7A0FCFA
:1077580052E79A6942F008029A6171E7FEFFFFEF6B
:1077680000800040457400082DE9F74F0368B0F821
:107778006080DF691A689D68D0F88C100192222910
:10778800044640F0B280B0F86890DFF868A1DFF8EE
:1077980068B10026B9F1000F01D0BB0621D4B4F8B6
:1077A8005E309BB2D3B1B4F868209A4216D92268E9
:1077B80002F1080353E8003F23F08053083242E8FF
:1077C800003122680029F2D14C4B636752E8003F30
:1077D80043F0200342E800310029F7D103B0BDE8A7
:1077E800F08F2368A26D596A08EA010122F8021B8A
:1077F800A265B4F85E20013A92B2A4F85E20DF696F
:1078080078072CD0F9070AD5019AD20507D50121A6
:107818001962D4F8901041F00101C4F89010B8072B
:1078280009D5E90707D502211962D4F8901041F06B
:107838000401C4F890107A0709D5E80707D5042190
:107848001962D4F8903043F00203C4F89030D4F8A9
:10785800903023B12046FFF744FCC4F89060B4F898
:107868005E309BB2002B95D1216851E8003F23F48C
:10787800807341E8003023680028F5D103F108023D
:1078880052E8001F01EA0A0142E800100028F5D179
:1078980020215B45C4F88C10606720670AD05968BE
:1078A800090207D553E8001F21F0806143E8001062
:1078B8000028F7D1E16E012913D1E66653E8001FCD
:1078C80021F0100143E800100028F7D1D969CA0651
:1078D80044BF102119622046B4F85C10FFF730FC51
:1078E80058E72046FBF7D4FB54E79A6942F00802B0
:1078F8009A6173E7FEFFFFEF0080004011750008F2
:1079080038B5044603682169A2681D68C0690A433E
:1079180061690A437D49024329400A431A605A684B
:10792800E16822F440520A435A60794AA1699342B5
:107938001CBF226A11439A6822F06E4222F4306218
:107948000A439A60DA6A616A22F00F020A43DA622D
:10795800704A93421CD14FF0B043D3F8883003F0FB
:10796800030343F44033A3F54033013B022B00F2F9
:10797800C780694A9B5CB0F5004F40F08980082BAE
:1079880024D8DFE803F061C0832380232323650024
:10799800624A934209D14FF0B043614AD3F8883024
:1079A80003F00C0343F44023E4E7594A93420DD112
:1079B8004FF0B043D3F8883003F44063B3F5006F59
:1079C8001AD005D853B1B3F5806F12D0012009E061
:1079D800B3F5406FFAD14FF400400EE0FEF7D2FC49
:1079E80058B900204FF00113A3660023C4E91D33E2
:1079F80038BDFEF7CFF8F3E74A4865684A4B626A34
:107A080005EB450133F81220B0FBF2F39942DDD8BB
:107A1800B3EB053FDAD800231946FAF775F80902DF
:107A280041EA10616B080002C0182A464FF00003B3
:107A380041F10001FAF768F83C4BA0F540729A4210
:107A4800C4D82368D860CCE7FEF79CFC0028C8D0CF
:107A58006168354B626A33F81220B0FBF2F24B08CA
:107A680003EB42034FF6EF72B3FBF1F3A3F11001FE
:107A78009142ABD823F00F02216892B2C3F34203BC
:107A88001343CB60ADE7FEF785F8DFE72548DFE76E
:107A9800082B9BD801A252F823F000BFED7A00080A
:107AA800F97A0008057B0008D5790008FF7A0008F4
:107AB800D5790008D5790008D5790008C97A000871
:107AC8004FF400406368616A174A32F81120B0FB2E
:107AD800F2F000EB5300B0FBF3F04FF6EF73A0F1B8
:107AE8001002ACE7FEF74EFC00283FF47AAFE9E756
:107AF800FEF758FCF8E7FEF74DF8F5E70948E1E727
:107B0800B0F5004FF4D1FEF74DFC9FE7F369FFCFC6
:107B18000080004000380140F81901080044004086
:107B2800FB19F5070024F400081A0108FFFC0F00F0
:107B3800836ADA0710B506D50168C46A4A6822F470
:107B4800003222434A609C0706D50168046B4A68E4
:107B580022F4803222434A60590706D50168446BF3
:107B68004A6822F4802222434A601A0706D501682F
:107B7800846B4A6822F4004222434A60DC0606D538
:107B88000168C46B8A6822F4805222438A6099068D
:107B980006D50168046C8A6822F4005222438A6080
:107BA8005A060FD50168446C4A6822F480122243B1
:107BB800B4F5801F4A6005D14A68846C22F4C0027B
:107BC80022434A601B0606D50268C16C536823F439
:107BD80000230B43536010BD2DE9F041DDF81880F8
:107BE80004460E4615461F462268D36936EA030343
:107BF8000CBF01230023AB4201D0002027E0B8F1DD
:107C0800FF3FF2D0FAF76CFFC01B4045206802D84E
:107C1800B8F1000F1DD150E8003F23F4D07340E8BD
:107C28000032002AF7D100F1080353E8003F23F09F
:107C3800010300F1080141E80032002AF3D12023B2
:107C4800C4F88830C4F88C3084F884200320BDE858
:107C5800F08103685A07C7D5C3691B05C4D54FF41B
:107C68000063036250E8003F23F4D07340E8003219
:107C7800002AF7D100F1080353E8003F23F001037D
:107C880000F1080141E80032002AF3D12023C4F8AA
:107C98008830C4F88C30C4F89030D5E773B5044602
:107CA8000026C0F89060FAF71BFF23681B681A07C4
:107CB800054619D423681B685B070AD56FF07E4315
:107CC800009300222B464FF480012046FFF784FFE3
:107CD800B0B900202023C4F8883084F88400C4F8A0
:107CE8008C30E06620670CE06FF07E4300933246EC
:107CF80003464FF400112046FFF76EFF0028D9D045
:107D0800032002B070BD10B5044650B3D0F88830D7
:107D18001BB980F88430FBF799F822682423C4F84B
:107D28008830136823F0010313602046FFF7E8FD4D
:107D3800012816D0A36A13B12046FFF7F9FE23687D
:107D48005A6822F490425A609A6822F02A029A608D
:107D58001A6842F0010220461A60BDE81040FFF799
:107D68009DBF012010BD000030B581658168A0F875
:107D78005C200023B1F5805FA0F85E20436735D111
:107D88000369002B40F2FF1318BFFF23A0F86030EF
:107D98000023C0F890302223C0F88C30016801F12C
:107DA800080353E8003F43F00103083141E8003479
:107DB8000368002CF2D1456E84680169B5F1005F53
:107DC80034D1B0F86850954230D8B4F5805F1DD1F1
:107DD800254A264C002918BF22464267C1B153E8FC
:107DE800002F42F4807243E80021F7E729B90369BC
:107DF800002B14BF7F23FF23C8E7B1F1805FC5D1F3
:107E08000369002B0CBF7F233F23BFE7174AE4E732
:107E180003F1080252E8002F42F0805203F10800F3
:107E280040E800210029F3D1002030BDB4F5805F7F
:107E38000FD10F4A0F4C002918BF2246426751B193
:107E480053E8002F42F4907243E800210029F7D14B
:107E5800EAE7084AF2E753E8002F42F0200243E835
:107E680000210029F7D1DFE771770008D5750008F0
:107E78001175000845740008D0F88C30202B30B4F8
:107E880015D1B9B1B2B100230468C3660A4B9C424C
:107E98000AD063681B0207D554E8003F43F08063AB
:107EA80044E80035002DF7D130BCFFF75DBF022054
:107EB80030BC70470120FBE700800040436E30B5BE
:107EC8002BB90123A0F86A30A0F8683030BD0368E8
:107ED800094D9A689968094C490FC2F342626B5C74
:107EE800615CDB00B3FBF1F3A0F86A30AB5CA25C29
:107EF800DB00B3FBF2F3E7E7281A0108201A0108B0
:107F08007047704770471FB504AB03E9060090F847
:107F18008430012B04463AD0012380F8843024238E
:107F2800C0F8883003681A6822F001021A609A685B
:107F380022F440120A439A6071B95A68BDF80C00DD
:107F48009DF80E1022F0100202435A605A6822F07F
:107F58007F4242EA01625A601A6842F001021A60DE
:107F6800FAF7BEFD6FF07E42034600924FF480019F
:107F780000222046FFF730FE38B92023C4F88830A5
:107F8800002384F8843004B010BD0320F8E70220F1
:107F9800F9E790F88430012B0FD0012380F8843062
:107FA800016851E8002F42F0020241E80023002B4B
:107FB800F6D180F88430184670470220704710B513
:107FC80090F88430012B044617D02423C0F8883059
:107FD80003681A68196821F00101196042F000521B
:107FE8004FF0005141661A60FFF768FF2023C0F880
:107FF8008830002084F8840010BD0220FCE770B5AA
:1080080090F88430012B044617D005682423C0F863
:1080180088302E682B6823F001032B60AB6823F0AF
:1080280060431943A960FFF749FF20232E60C0F879
:108038008830002084F8840070BD0220FCE770B509
:1080480090F88430012B044617D005682423C0F823
:1080580088302E682B6823F001032B60AB6823F06F
:1080680060631943A960FFF729FF20232E60C0F839
:108078008830002084F8840070BD0220FCE70000EE
:1080880038B5094D002455F8043B33B90134E3B23F
:10809800052B64B2F7D1002038BD002CF6D01B693F
:1080A80098470028F2D0F7E7440800207FB50A2354
:1080B80001A88DF8043003F0D9F80038044B059A6C
:1080C8001A6018BF0120404207B05DF804FB00BFEA
:1080D8003C08002070B504460B46144962784A7083
:1080E8000020A2780A7208701A884A729A788A72EE
:1080F800DB780B746368CB600D4B1B68DA6A2AB1B6
:10810800237803F0FB030B2B00D09047094E002582
:1081180056F8043B1BB19B6A0BB1204698470135C2
:10812800EBB2052B6DB2F3D170BD00BFD8000020B3
:10813800400800204408002070B504461148012377
:10814800037063784370A3788372E368C360E3784D
:10815800037623694376237943720B4B1B689B6A2A
:1081680003B19847094E002556F8043B1BB1DB695B
:108178000BB1204698470135EBB2052B6DB2F3D110
:1081880070BD00BFEC00002040080020440800201B
:1081980038B501F011FE0C4D052455F8043B5BB1D0
:1081A8005B694BB155F8043C9B682BB1984718B1F3
:1081B80055F8043C5B699847013C14F0FF04ECD186
:1081C800BDE83840FFF75CBF44080020014B186841
:1081D800704700BF3C08002000B58BB001236846FB
:1081E8008DF8003002F0BCFC38B99DF80400003866
:1081F80018BF01200BB05DF804FB0020FAE700006F
:1082080030B58BB0054601F0BBFD0446002839D1D6
:10821800FFF7E2FF012838D168468DF8004002F0E8
:108228009FFC10B14FF0FF3004E09DF80430AB42E2
:1082380002D100200BB030BD012DF3D0022D11D09A
:10824800002DF7D1002BF4D068468DF8045002F0C9
:1082580099FD0028E6D10E4B1B681B6B002BE8D05C
:108268009847E6E7002BDDD168468DF8045002F008
:1082780089FD0028D6D1064B1B681B6B002BD8D074
:108288002846EDE76FF00100D4E76FF00200D1E770
:108298004008002070B5324C324B94F9042094F910
:1082A800055090B0012602288DF804608DF8092049
:1082B8008DF80A500AD18DF80800D871197202F0A9
:1082C8009FFB01A802F0D2FF10B070BD4FF4807080
:1082D8001A715D71D8801972234B8DF808601B786C
:1082E80053BB1E2306A88DF81C208DF8183002F009
:1082F80049FD1F238DF8183006A823798DF81C3006
:1083080002F040FD21238DF8183006A863798DF816
:108318001C3002F037FD20238DF8183006A8637949
:108328008DF81C3002F02EFD28238DF8183006A891
:108338000E4B079302F026FD02F062FB012306A80C
:108348008DF818308DF81C3002F01CFD084B1B68A6
:108358005B6A0BB1034898476078FFF751FFB3E7B2
:1083680058080020C0000020380800200003000141
:108378004008002008B501F003FD40B9FFF72CFFC5
:10838800012806D0084B197AD879FFF783FF012016
:1083980008BD064B1B68DB6898470028F7D1BDE885
:1083A8000840FFF76DBE00BFC00000204408002051
:1083B8002DE9F04186B005460C46164601F0E0FC72
:1083C800002840F08D8001F0EDFC40B9FFF704FF74
:1083D800012807D0444B197AD879FFF75BFF6FF073
:1083E80002046DE0414F3B68DB68984730B13A685A
:1083F8002B7812789A4201D0002B6ED13C4FDFF8CF
:10840800F4803C72003C18BF012498F80430687866
:108418008DF8044069468DF8123002F049FB0028B7
:1084280040D000238DF804300393ADF810306FF07E
:10843800060495E80300304B83E8030098F80430FD
:10844800BB72314601A803F009F82C4B059A1A6053
:1084580011283FD801A353F820F000BFC3840008B7
:10846800E9840008DD840008DD840008DD84000854
:10847800DD840008DD840008E7830008DD84000847
:10848800DD840008DD840008D7840008DD84000846
:10849800DD840008E9840008E9840008E98400080C
:1084A800D18400082B788DF808306B78ADF810303F
:1084B8006B6803934FF0FF34BBE7E31D18BF00243C
:1084C800204606B0BDE8F0816FF00404F8E76FF0CD
:1084D8000504F5E74FF0FF34F2E76FF00304EFE728
:1084E8006FF00104ECE700BFC00000204408002042
:1084F800EC00002058080020FC0000203C08002068
:1085080010B504468AB018B94FF0FF300AB010BD54
:10851800002368468DF8003002F022FB0028F3D1D2
:108528009DF804302370F1E7F0B587B000220B46C0
:108538002A498DF8072001220A7042784A700446B9
:10854800002A41D102790A721A884A729A788A7284
:10855800DB780B740369CB60C378214D8DF8083044
:10856800037B8DF80930836803932B68DB6A0BB1B2
:1085780002A898472B689B6B13B1227E02B19847DB
:10858800184E0025374656F8043B53B11A6A42B1D3
:108598001A78E3789A4219D156F8043C20461B6AA7
:1085A80098470135EBB2052B6DB2ECD10DF1070000
:1085B800FFF7A6FF63793BB10021012204A8ADF8BB
:1085C80010100591FFF7F4FE07B0F0BD002DE8D1BB
:1085D8003B68DB6898470028DED1E2E7D800002036
:1085E800400800204408002010B504468AB018B995
:1085F8004FF0FF300AB010BD1F2368468DF80030D9
:1086080002F0AEFA0028F3D1024A9DF90430237033
:108618001371EFE75808002000B58BB022230190B2
:1086280068468DF8003002F0ADFB003818BF012015
:1086380040420BB05DF804FB70B5634C014618224C
:108648008EB0204605F066FFFBF756FF237840689A
:10865800012202FA03F1014004D15C4B084607F0FD
:108668004FFFFEE75A495B481A4602F011F818B165
:108678004FF0FF300EB070BD262304A88DF81030DF
:1086880002F080FB544E554D002870D10123337001
:108698002B68DB690BB100209847262304A88DF8C6
:1086A800103002F05DFA059B93F84820227093F889
:1086B800182193F81A316270A370454BD3E902016F
:1086C80005F01AFE05460028D2D1454E062304A817
:1086D8008DF8103002F044FA059B736104A802F08B
:1086E80051FB022304A88DF81030059602F038FAE1
:1086F8000836032304A88DF81030059602F030FAE6
:108708000F2605F0BDFE012304A88DF814308DF85E
:10871800106002F037FB10230DEB03008DF81030CA
:108728008DF8145002F02EFB04238DF8103004A8A5
:10873800A3788DF8143002F025FB39238DF810301A
:1087480004A86369059302F01DFB02A920788DF83F
:10875800086003F051FF003818BF0120E0711420B1
:10876800FFF75AFFE07903F003F8284682E727234A
:108778008DF810302B681B6943B104A802F0F0F99A
:108788002B6805981B694FF4EE619847262304A8C7
:108798008DF8103002F0F6FA50B9012304A88DF8CC
:1087A800103002F0DDF99DF81430002B7FF46EAF25
:1087B8003378002B7FF46CAF052204A88DF81020C5
:1087C800059302F0DFFA78E758080020301A01080C
:1087D8007008002088080020380800204008002081
:1087E8002008002037B500230D4601930446C0B980
:1087F80000F0D0FA0190019BC3B10E4A0E4942F82D
:1088080024300E4ADA620E4A1A630E4A5A630E4A36
:10881800126892699A6128465B68F222984700209C
:1088280006E001A900F0BCFA0028E4D04FF0FF30C0
:1088380003B030BD440800202C0700209D820008AA
:10884800B9830008B580000840080020154B07B51B
:108858001860154B154A1A60154A5A60154A9A60ED
:10886800154ADA60154B02681A6042685A608268D5
:108878009A60C268DA60124A01911A6111498269E4
:108888005A610020FFF7AEFF48B901A800F086FA48
:10889800003818BF0120404203B05DF804FB4FF0D8
:1088A800FF30F9E7400800208808002041810008CF
:1088B800318500084D890008DD8000087008002017
:1088C800B1C50008CC00002051B118B1012804D06E
:1088D80000207047044B0B607047044B0B60F7E7B0
:1088E8004FF0FF30704700BF000300010300010193
:1088F80008B502F059FF002814BF6FF001000020EE
:1089080008BD08B502F0A4F8002814BF6FF00100F4
:10891800002008BD10B504468AB018B94FF0FF30E2
:108928000AB010BD202368468DF8003002F018F90F
:108938000028F3D1024A9DF9043023705371EFE700
:10894800580800202DE9F0412F4D304F00232B709F
:1089580043786B703B689B6A8AB004460BB1284623
:108968009847DFF8AC80002658F8043B1BB15B6AD7
:108978000BB1204698470136F3B2052B76B2F3D1F6
:108988002378052B2FD00C2B35D0012B25D1214C4A
:10899800062368468DF8003002F0E2F80199E07984
:1089A80005F0F0FC10B91C4B019A5A611B48FFF7FF
:1089B8001BFE1B48FFF7AEFF6B788BB9A371194BF1
:1089C8005878FFF71DFC3B685B6A0BB11148984764
:1089D8006B7813B9E07905F065FD0AB0BDE8F08160
:1089E800FF23A371EFE7104B01225A74227A9A747D
:1089F800627ADA74F1E76378002BEED00AB0BDE84A
:108A0800F041FFF753BB00BFEC00002040080020F6
:108A180044080020C000002020080020C4000020D6
:108A2800C500002058080020D800002030B58BB0C1
:108A3800FFF767FF0446F0B903F0BEFD831C1DD0A5
:108A4800F8B9134D2B685B69DBB1262368468DF8AE
:108A5800003002F085F82B6801985B694FF4EE61ED
:108A6800984703F0BBFD78B92CB9094B1B68DB6943
:108A78000BB10120984720460BB030BD6FF00704BA
:108A8800EFE74FF0FF34ECE74FF0FF34F3E700BFB8
:108A98004008002030B5064D064C30B129B1286099
:108AA800A16062710123237030BD00232B60FAE7B7
:108AB800C408002098080020014B1878704700BFB0
:108AC80098080020024B187800B15878704700BF0A
:108AD8009808002070470000064B1A784AB15A7867
:108AE8003AB10278012A04D1027912B19A89013285
:108AF8009A81704798080020074B1A7852B15A7823
:108B080042B10278052A05D1017A427AD973012047
:108B180098731A74704700BF9808002013B51A4C50
:108B280023783BB363782BB3A27BA36862B100229E
:108B3800A2730322A27105221A70E27B5A70227C6A
:108B48009A700122A27004E0A278012A14D0042AA3
:108B5800F7D0E0228DF800200C48A27901938DF817
:108B6800012008F049F80A4B1B6B1BB1E178012280
:108B78006846984702B010BD0222A271A2895A70B5
:108B8800110A1970E5E700BF98080020AC0800201A
:108B980008010020FFF7C2BF30B5794C23788DB0AB
:108BA800002B43D0437B002B40D0657825B1837BD5
:108BB80013B9A3890133A381C178E02936D1002DE7
:108BC80036D1027B042A31D18368187801282DD147
:108BD800587801282AD19878012827D1DB78012BE9
:108BE80024D102206380A071E56002A863708DF82B
:108BF8000C3021718DF80820257402F0C3F828463E
:108C080002F0B6FD5F4B1B685B6803B19847002212
:108C18005D4B00924FF0FF315C4807F041FF41F295
:108C280088315A4808F022F8FFF778FF0DB030BDB8
:108C380083681A78A2700A2AF8D8DFE802F00621B9
:108C480024282A3D44658D8F9900504807F086FFF7
:108C580000236370A3814B4C04238DF808302368EC
:108C680002A81B788DF80C3002F08CF8236858782D
:108C780002F07EFD23689B68002BD7D09847D5E784
:108C88000223A371D2E740F201136380CEE70123E8
:108C9800FBE7A568037BA37104222A7062799A42D4
:108CA80028BF1A4600230133D9B28A42BED9816847
:108CB800C95C0131E954F6E705238DF8083002A8AC
:108CC80002F0D4FAB2E7314807F048FF0023637096
:108CD800A3812C4C04238DF80830236802A81B7844
:108CE8008DF80C3002F04EF82368587802F040FDF9
:108CF80023689B6803B19847254BDB6A002B95D006
:108D080001210220984791E7027B032A0DD1062210
:108D18008DF80820B3F801305BBAADF80C3002A822
:108D280002F0A4FA0123A37080E7072AF7D18DF88F
:108D38000820B3F8012052BAADF80C201A79D97876
:108D4800120242EA014259790A4364214A430492D1
:108D58009B798DF81430E2E70A23AEE700228DF8FC
:108D680008205B788DF80C3002A802F00BF85DE75C
:108D78000D228DF808205B788DF80C309FE700BF36
:108D880098080020C40800209D8B0008AC0800202B
:108D980008010020004870470801002000207047A3
:108DA8004FF0FF3070470000044B054A93F8183124
:108DB800022B18BF062382F8803470473810002031
:108DC800AC170020034BD3F8483313B15B6903B1E8
:108DD80018477047AC170020034A137843F0020382
:108DE8001370FFF7EFBF00BFA81700201FB50A4B8D
:108DF8008DF8090093F87C208DF80A2093F88C20D0
:108E080093F848000D3202A98DF8082003F0F4FB0E
:108E1800C0B205B05DF804FB3810002010B50D4C49
:108E280004F57D7007F09AFE94F8103413B101230D
:108E380084F80F34084B93F81831022B02BF94F8CA
:108E4800813443F0100384F88134BDE81040FFF703
:108E5800B9BF00BFAC1700203810002010B50C4C6B
:108E6800D4F8403343F08003C4F8403394F8103406
:108E780013B10020FFF7D2FF94F8813423F01203D6
:108E880043F0120384F88134BDE81040FFF78CBF2B
:108E9800AC1700202DE9F0412C4D95F81831022B24
:108EA80007460E4602D02A4BDB6A984702F01BFDA4
:108EB800044628B1022002F00CFD002002F00EFD4D
:108EC80095F81831012B17D102F00FFD804630B10B
:108ED800002002F0FFFC002002F001FD444602F0F1
:108EE80006FD48B1002002F0F6FC002002F0F8FC74
:108EF800BDE8F041FFF758BF002CF9D1154C94F8A4
:108F0800802494F81034B2B90BB184F8357438461B
:108F180002F090FEE86A07F0E7FDD4F8B43398420F
:108F2800E6D30D4807F01AFE94F8813443F0100395
:108F380084F88134DCE70BB184F83564304602F0FC
:108F480079FE95F81831022BEED1D1E738100020C0
:108F580038210108AC170020441B0020074A10B52F
:108F6800137843F001031370FFF72CFFBDE810409E
:108F7800034B01220021022007F0C2BAA8170020E3
:108F8800791A0108074A10B5137843F004031370DF
:108F9800FFF718FFBDE81040034B01220021022013
:108FA80007F0AEBAA8170020891A01082DE9F04188
:108FB8000F4616461D46804607F08CFD0A4A0B4CA4
:108FC8001378278143F00803C4E900081370668109
:108FD8002573FFF7F7FEBDE8F041054B012200219C
:108FE800022007F08DBA00BFA8170020B41C00208B
:108FF800991A010813B507F06DFD0D4B6C46186002
:10900800204607F0BBFC94E803000A4A0A4B83E8B1
:109018000300137843F010031370FFF7D3FE074BD8
:1090280001220021022002B0BDE8104007F068BA12
:10903800C41C0020A8170020E41A0020A61A010862
:109048002DE9F04192B0064602F04DFC002840F0B0
:109058005681AC4D95F81831012B09D02B6BAA4CD1
:1090680093B194F80431BBB1042B6FD0032003E013
:1090780002F03BFC18B10F2012B0BDE8F08102F0FD
:1090880036FC0028EAD0F6E7B5F81E31D4F81424E7
:10909800013B53432B63E4E79C4803F0E4F90028C1
:1090A80040F0298194F80C3123802B6B0C930DF13F
:1090B800180895F839308DF83830404695F81C3145
:1090C8008DF83A3007F080FCD5F82431009302AFD0
:1090D80098E80600D5F82031384607F00CFC97E8E8
:1090E80003000FAB83E80300EB6A0D9300238DF8B0
:1090F80044302388ADF8463095F82C3101228DF89C
:1091080039201BB98DF844208DF83930804B0093F5
:10911800804B95F84800A3F173020CA903F0E1FA1B
:10912800C0B10B28A8D1D4F8841499B1002EA3D0CB
:10913800D4F84033784843F02003C4F8403307F0AC
:1091480095FD754807F058FD002095E76F4803F036
:10915800BEF9A4E795F8487095F9693095F9392072
:1091680095F87D106D4E384603F0CDFA009641B261
:10917800EB6C95F850203846143603F063FA0096E5
:10918800EB6C95F8502095F9701095F8480003F0AD
:1091980059FAD4F8C413AB6DD4F8D8230B44C4F8E7
:1091A800B033EB6D1344C4F8B43394F80431042B92
:1091B80007D02B6E0B44C4F8B0336B6E1344C4F85D
:1091C800B4330023089395F82C3183B108A802F032
:1091D80061FC00284AD195F9390094F837629DF866
:1091E8002070FFF703FE3E4480B2B0423CD3002318
:1091F8008DF8133095F839308DF8213095F83830DE
:109208008DF82230D5F880300993D5F884300A9348
:10921800238894F81164ADF82C3095F84800404B39
:109228008DF820600DF1130208A903F01FFA01233D
:1092380084F8353495F8393084F836349DF813308D
:1092480084F83734D4F81434C4F84464C4F83C348B
:10925800C4F84C3402F04DFB50B1D4F8140402F0B9
:109268005AFB28B1102007E7082005E7132003E779
:1092780095F81831012B01D102F04FFB02F03CFBAD
:109288000023059394F8043195F9395094F8116442
:10929800BBB1042B7FF4EAAE05A802F037FE60BB31
:1092A80094F80C341BB994F80E34012B02D9059BA1
:1092B800013B0593154B05983246E9B202F098FE3A
:1092C80002E0124802F06CFEA8B9D4F8403394F8D2
:1092D8000C11218043F00203C4F8403394F8103491
:1092E80023B994F80C34013384F80C340D4B0E4830
:1092F8009B6A984728E71120BEE61220BCE60E209C
:10930800BAE600BF38100020AC170020B4180020BF
:1093180068100020301C0020141B0020641B002053
:10932800C01B002038210108AE17002073B5144C6B
:10933800144D04F57876EB6C95F8502095F9781073
:1093480095F84800009603F07DF940F2012395F85E
:109358004800A4F8F23304F21C42314603F07EF9C7
:1093680058B194F81C3484F85E34074B00205B6BCA
:10937800984794F8F33384F8803402B070BD00BF86
:10938800AC1700203810002038210108F8B5334DFB
:1093980095F81841012C06464BD0022C51D064B9DF
:1093A80038B9D5E91B0105F1740383E803002046A9
:1093B800F8BD01283DD0022801D00324F7E7284F43
:1093C80085F8180107F5737EBEE80F0007F5787C6D
:1093D800ACE80F00DEF80030CCF8003095F8E93042
:1093E80087F8F363E3B195F80031022B18D1D5F86B
:1093F80004316B67C7F8E43395F87D3095F8082198
:1094080087F8F03395F88C3085F8782087F8F133B1
:1094180097F8112487F8E02340F20133A7F8F233D4
:10942800002387F810340F4BDB6A9847FFF77EFF5D
:10943800BDE702F063FA04460028B8D185F8186140
:10944800B5E70028B9D1064B85F81801062283F83C
:109458008024044BDB6A98473446A8E7381000207C
:10946800AC17002038210108F0B5484C484EB4F834
:10947800DC202287D4E92D0194F8B12084F86920F2
:1094880004F16C0282E80300D4E92F0104F17402AC
:1094980082E80300B4F8C420A4F87C20D4F8CC20D7
:1094A800C4F884208FB0D4F8D020D4F8C810C4F8F9
:1094B80088200025374AC4F880100123A4F81E31FB
:1094C800C6F80C24C4E94E5584F82C51A56284F8DA
:1094D8001B5184F83A50C4F83051A4F8345186F836
:1094E800105484F841518DF8143004F5087394F839
:1094F8004800A4F84251039303A904F52D7304937B
:1095080003F088F8E36EC6F8D03394F87D3086F817
:10951800DC3394F88C3086F8DD334FF48073A6F88A
:10952800DE3386F8CC5306F573770FCF06F57874DB
:109538000FC43B68236040F20123A6F8F233D6F843
:10954800483386F81154CDE901551BB15A685B6957
:1095580001920293104B0693A3F144020792A3F1E0
:10956800140208920D4A0A9225330993A2F19C032A
:109578000B93A2F198030C9301A9131D06A802F2FC
:1095880074620D9302F0A4F90FB0F0BD38100020FA
:10959800AC17002000010100081C00201C1100204D
:1095A800F8B50D4F0D4C0E4E0D4607F0D7FA3B6B34
:1095B800984796F8480004F21C42294603F04EF8F2
:1095C80048B194F81C3484F85E34706D7B6B98470E
:1095D800EB7C84F88034F8BD38210108AC170020F2
:1095E800381000200D4890F8113480F8B8330C4B2F
:1095F80093F8692080F8BB2393F87D2093F88C308A
:1096080080F8C933002380F8C823A0F8CA3300F5CE
:109618006E7100F56070FFF7C3BF00BFAC17002084
:10962800381000200F4890F88034CBB190F81134EE
:1096380080F8CC330C4BDA6EC0F8D02393F87D2039
:1096480093F88C3080F8DD334FF4807380F8DC2396
:10965800A0F8DE3300F5737100F56670FFF7A0BF60
:10966800704700BFAC1700203810002070B5344C8C
:109678002421204604F064FF636A984218BF6062A0
:109688004FF01C012F4814BF0125002504F058FF96
:10969800636C984218BF60644FF0FC012A4818BFF9
:1096A80045F0020504F04CFFD4F84431984218BF45
:1096B800C4F844014FF0D401244818BF45F004050C
:1096C80004F03EFFD4F81C32984218BFC4F81C02BC
:1096D8004FF090011E4818BF45F0080504F030FF10
:1096E800D4F8B032984218BFC4F8B0024FF494616D
:1096F800184818BF45F0100504F022FFD4F8543775
:10970800984218BFC4F854074FF01401124818BF04
:1097180045F0200504F014FFD4F86C3798420F4B3D
:1097280018BFC4F86C07D3F8483318BF45F0400594
:109738002BB11B691BB12846BDE87040184770BDA6
:1097480038100020601000208010002080110020B8
:1097580058120020EC12002090170020AC170020AF
:109768002DE9F04F91B00026BD4F8DF815600546E4
:1097780088469346ADF81860B146C14502D311B08A
:10978800BDE8F08F15F8090002F0C2F948444045D9
:10979800F5DC15F8093009F10104023BE4B2112B9C
:1097A800EDD801A252F823F0F9970008299800088B
:1097B800E998000815990008A5990008C9990008B2
:1097C8003D9A0008719A0008EF9A000887970008E8
:1097D800879700084F9B000887970008879700081D
:1097E800059C00082B9C00086F9C0008AD9C000895
:1097F800052002F039FA88B10521002002F0F8F9B5
:109808002B5D87F8503409F1030409F102095FFA66
:1098180089F9E4B215F8093087F85134A146ACE764
:1098280000238DF816308DF817308DF81C308DF820
:109838002030002E52D18B4E631E2B440D9396F888
:109848001A318DF83A3096F87C308DF8393096F820
:1098580039308DF83B3096F838308DF83C3096F832
:1098680068308DF83D30D6F828310C9308AB019359
:1098780007AB009396F84800A8EB09090DF1170308
:109888000DF116020CA98DF8389002F0FBFE8DF848
:10989800150000F0070007280BD19DF8163086F850
:1098A80039309DF8173086F838309DF81C3086F826
:1098B800683000264FF0050906E001220DF1150178
:1098C800032002F03BF80136F2B29DF82030B3FBDA
:1098D800F9F19142F1D8013B2344DCB201269DE71E
:1098E8002B5D604903F00F03012281F81B3109F158
:1098F800020902FA03F3A1F81E315FFA89F900227E
:1099080006A9042002F01AF84C4687E707238DF8C9
:1099180015302B5DC3F3021203F00F038DF83030BE
:1099280009F10303DBB28DF83120EA5C09F1040385
:10993800DBB209F10504EB5C09F102095FFA89F968
:109948001B0443EA022315F80920DFF81891134392
:109958006422534399F848000D930CA902F0A1FE24
:1099680000F00703072BE4B28DF815000ED19DF81F
:10997800303089F8703089F878300D9BC9F86C3030
:10998800C9F874309DF8313089F869308DF81800BD
:10999800012206A9052001F0D1FF3FE7D7F8483397
:1099A80063B11B6853B198470BF03F038DF818005B
:1099B8008DF81930022206A90620ECE7FF20F3E70C
:1099C80003238DF815302B5D8DF824300CAB0893EC
:1099D80009F10303DBB209F10604EA5C09F10403A7
:1099E800DBB208A9EB5C1B0443EA022309F102027B
:1099F800D2B209F10509AA5C1343642253435FFA02
:109A080089F90C9300230D9315F809308DF8383037
:109A1800144B93F8480002F04AFEC3B20028E4B29F
:109A28008DF81530FFF6FAAE8DF81830012206A928
:109A38000720B0E72B5D03F00F03012B4FF47A7278
:109A480038BF01235343074A09F10209936503F517
:109A58007A73D3655FFA89F9002206A9082051E7CD
:109A6800AC170020381000202B5D9C4CC3F340122B
:109A78008DF81D2094F84800C3F3001207A903F0DD
:109A88000F038DF81C208DF81E3002F016FE09F128
:109A9800020901305FFA89F93FF436AFBDF81C308E
:109AA8008F4AA4F87C309DF81E309DF81CA0D05C2D
:109AB800F7F7ACFF0223C4F880000CA994F848001B
:109AC8008DF830308DF832A002F096FD94F93930D7
:109AD800089040B29842B8BF184684F8390000226E
:109AE80006A909200EE703238DF815302B5D8DF8A4
:109AF800303009F10303DBB209F10504EA5C09F12E
:109B08000403DBB209F10209EB5C5FFA89F91B0473
:109B180043EA022315F809201343642253430D93A3
:109B28006E4B0CA993F8480002F0CDFDC3B2002893
:109B3800E4B28DF81530FFF671AE8DF818300122B9
:109B480006A90A2027E70A2002F08EF800283FF429
:109B580065AE0A21002002F04BF80023ADF826304C
:109B680009F10203DBB24FF47A71EA5C09F10303ED
:109B7800DBB20DF1300AEB5C1B0443EA02232A5DD9
:109B8800134309F10402D2B209F1060409F10509E7
:109B9800AA5C5FFA89F943EA026315F8092003937E
:109BA8004A4312125046ADF8242006F0E7FE039B04
:109BB80003F1965303F5A91303F5EC530893D7F86B
:109BC8003C3300930DF1200999E80600D7F83833A3
:109BD8000AA806F090FE0B9B00939AE806000A9BE1
:109BE800484606F06DFE99E8030006F09FFE01F076
:109BF8008FFE0123E4B287F830340FE60D2002F01F
:109C080033F800283FF40AAE0D21002001F0F0FFE0
:109C180097F88034043B012B7FF600AE01F074FE08
:109C2800FCE509F10203DBB22A5DE95C09F10303F3
:109C3800DBB209F10504EB5C09F104095FFA89F963
:109C48001B0415F8090043EA01231343642159430F
:109C580000F00F0001F059FEE4B28DF8180001225F
:109C680006A9112097E60E2001F0FEFF00283FF418
:109C7800D5AD0E21002001F0BBFF09F10203DBB2D4
:109C8800184AE85C2B5D126809F1040409F103091C
:109C98005FFA89F943EA002015F80910E4B201F0E7
:109CA80036FEBBE52A5D09F1020309F1040409F156
:109CB8000309DBB25FFA89F9E95C15F809301B047E
:109CC80043EA012313436420584301F022FEE4B21F
:109CD8008DF81800012206A913205CE63810002030
:109CE800B31A0108B41C00200E4B93F88124920784
:109CF80003D593F87F24012A06D90B4A92F81A1142
:109D080011B1916A01319162002283F80C2483F821
:109D1800102483F80F24D3F8402322F00202C3F85A
:109D280040237047AC1700203810002010B5124CA3
:109D380004F55A7006F012FFD4F84033012023F0DE
:109D48002003C4F84033FFF77BF998B10B2811D0F2
:109D58000A4B93F8393084F83634092094F80E34D5
:109D680084F8393484F8350401F064FFBDE8104004
:109D7800FFF7BABF10BD00BFAC1700203810002095
:109D8800074BD3F84023012A06D03AB993F8820446
:109D9800013818BF01207047002070470120704724
:109DA800AC170020034BD3F84003431E58425841D8
:109DB800704700BFAC1700202DE9F04FA5B0EFF3B6
:109DC800108172B6C04A00201368106081F31088B1
:109DD800BE4C002B00F0DA80D9065FFA83FB6BD506
:109DE800BB4D95F81831022B02D0BA4BDB6A984765
:109DF800EFF3108872B6B84F06F06CFE3E68D4F8E0
:109E0800B013361A3144B54806F030FFB34806F0AF
:109E1800F3FED4F8B413B248314406F027FFB04833
:109E280006F0EAFE88F3108895F81831022B02D064
:109E380094F810348BB116230EA995F848008DF8C4
:109E4800383002F0D9FBD4F8B4130C900144A5487B
:109E580006F00CFFA34806F0CFFE3B6894F81124E7
:109E6800EB620AAF38468DF86020199306F0ACFD16
:109E7800D5F82431009304AE97E80600D5F82031D0
:109E8800304606F038FD96E803001BAB83E8030074
:109E9800D4F814341A9395F82C3195F84800003BFF
:109EA80018BF012318A98DF8613002F0AEFB94F8B1
:109EB80010340BB984F835341BF0080F3AD08A4BAC
:109EC800834D5F681E89B3F90A8093F90C90D5F821
:109ED800E42003920023079384F83834A4F81A3452
:109EE80084F81D34C4F82034A4F8243484F82634C3
:109EF800C4F8283484F81834C4F82C3484F830347E
:109F0800744B94F88024DB6A84F87F24A4F87C845A
:109F180084F87E949847724806F020FE3146384609
:109F280001F0DFFC8246002800F0E680A4F8728485
:109F380084F874941BF0040F1AD0654B93F8183109
:109F4800022B02D0634BDB6A98470220FEF72CFFF6
:109F580084F8350401F06EFE94F8103413B101232F
:109F680084F80F3494F8813443F0100384F8813472
:109F78001BF0020F03D006210520FEF78BFF1BF014
:109F8800010F03D004210320FEF784FF01F0C6FC73
:109F980094F88124D0065FD5002384F88234D4F85D
:109FA8004033190644BF23F08203C4F8403312F04B
:109FB800050F00F0C5820C2001F056FE002800F0C5
:109FC800BF8294F88134DF0700F1BA825E0740F15E
:109FD800CB82D4F8403323F00203C4F84033D4F8DA
:109FE800402382BB94F8815415F001011EBF2B4613
:109FF80062F3000384F8813494F881345E0744BF27
:10A008006FF3820384F88134012384F8823421B108
:10A01800D4F8443335481B6898476D070BD5344846
:10A0280001F02EFE01F05CFE28B194F8813443F073
:10A03800040384F8813401F060FC94F881346FF3F0
:10A04800041384F88134012384F8823494F8813429
:10A0580043F0200384F8813494F8813418070AD532
:10A068006FF3C303234984F88134D4F84433A1F14E
:10A078002000DB68984794F8813499070AD56FF374
:10A0880041031C4984F88134D4F84433A1F16400B5
:10A098005B68984794F88034022B01D1FFF746F9A2
:10A0A80094F881349A0640F1EC826FF3451384F8F2
:10A0B8008134D4F84033002B40F0E38225B0BDE86A
:10A0C800F04FFFF7D3BA00BFA8170020AC17002045
:10A0D8003810002038210108C41C00202C1B002047
:10A0E800441B0020A01B0020B41C0020E01B002003
:10A0F800F41B0020281C002095F81831012B0CD1E6
:10A1080001F0F3FB804668B1504601F0E3FB50468E
:10A1180001F0E5FB042384F87F347EB9012384F839
:10A1280019344AE101F0E3FB0028F6D0404601F07B
:10A13800D2FB404601F0D4FB0523ECE73B780293C1
:10A148005B09013B062B00F2ED81DFE813F0070005
:10A15800EB019200EB018F00EB01DB01102EDDD942
:10A1680095F82C310E97F6B28DF83C60002BD5D1BE
:10A1780018A804F0F9F80EAA18A9FF2002F04CF864
:10A188009DF84830C3F3030307468DF8203095F84F
:10A19800480095F87D308DF82130072208A902F093
:10A1A8003EFA002F5AD1002858D09DF843309DF828
:10A1B80042201199C5F8E4101B0443EA02239DF8D4
:10A1C800412002201343C5F8E03004F0DBF89DF885
:10A1D800483095F8480085F82A71C3F30212C3F392
:10A1E800030385F8703085F878309DF8493085F894
:10A1F8006920012B38BF01234FF47A725343AB65B2
:10A208001344EB654FF001080DF14A03113E0CA908
:10A218000C9385F868808DF8346002F008FA022300
:10A22800404685F82C3101F01FFD18B141463846EB
:10A2380001F0DEFC94F81034002B00F0798194F8DA
:10A24800383413B10020FEF7E9FD94F8813443F067
:10A25800100384F88134FEF7A7FD6BE6012001F0B6
:10A2680003FD0028E6D001210720E1E7012384F857
:10A27800183495F87D308DF8223094F81C348DF818
:10A28800213095F88C3095F848000D3308A98DF8E1
:10A29800203002F0B1F9A6F10D031BB2069023EAB3
:10A2A800E37300B283423FF739AF0B2E7FF636AF28
:10A2B800A24B219318A8FF2318978DF864608DF896
:10A2C800883002F075F8804600287FF427AF9DF8A3
:10A2D8006C301A99C4F82C1413F00F0203D09DF8AF
:10A2E800800000286CD19DF8880000286AD0002AD8
:10A2F8007FF414AF9DF88020002A0CBF02270327A3
:10A3080000220792D5F8EC2091425DD195F8E9102A
:10A31800002959D0D5F80C1195F8EAA009680791D9
:10A3280095F81811022902D1032184F87F14032F0C
:10A338007FF4F4AE13F0600F7FF4F0AE03924FF0A9
:10A348000108152395F848008DF8203008A902F077
:10A3580053F995F82A310690BAF1000F37D0BAF1BF
:10A36800010F3ED1012B34D16FF009063E4106F0B2
:10A378000106C6F10206F6B281B2BDF86E2007AB3F
:10A38800304601F0CFFD70B3072824D1082384F8A4
:10A39800193495F82A315BB9029B03F0E003A02B2E
:10A3A80006D16A6B239B9A4202D1012385F83A3081
:10A3B800079BC4F82834C4F86034FEF74FFDB9E5AC
:10A3C80047469DE701279BE74FF0010AB9E70426B6
:10A3D800D2E70326D0E7082803D10A2384F81934E2
:10A3E800E6E70123FAE718AB00930399079B324687
:10A3F800504601F063FE20B102280CBF0B230C234A
:10A408008DE6079BC4F82834C4F860349DF86C3096
:10A4180084F81904C3F3401384F8263484F83834D4
:10A4280094F87F3484F81A84012B98BFA862B8F195
:10A43800010FC4F8200484F8240484F8350433D1C7
:10A44800022284F8182495F83A20002A3BD19DF876
:10A458006C20D20637D4012B94F834149DF86C2064
:10A4680005D8012901D1960601D501F001FB022F7B
:10A4780037D0032F09D09DF86C10012F4A4601F000
:10A488000F011CA831D0FFF76BF99DF8803084F8D4
:10A498001B34219BC4F820349DF8883084F8243478
:10A4A800012384F8253426E0029A02F0E002A02A6B
:10A4B80011D195F82A11012285F83A2009B9239972
:10A4C800696384F8182495F81821002AC3D1012259
:10A4D80084F81D24BFE7002285F83A2084F8182460
:10A4E800B5E79DF8881021984A46FFF739F99DF895
:10A4F800803084F81B3494F8813443F0020384F8E4
:10A50800813497E6DFF83480013EB2B2791C4046C8
:10A5180004F000F80323A4F81834C4F8208484F85D
:10A528002464E8E7012384F81934FEF797FC81E6F0
:10A5380095F81831022B7FF488AE83E6E4190020E1
:10A5480094F881345D070FD5012001F08DFB88B3A5
:10A55800012001F05FFB08B984F80C04D4F84033FB
:10A5680023F00203C4F8403394F88114C8077FF538
:10A5780036AD94F834340BB1032B26D1424B94F802
:10A588000C0493F86820904208D28A0750D593F8B3
:10A5980018311BB194F87F34002B49D13B4806F0A1
:10A5A800DDFAD4F8403323F02003C4F84033FFF732
:10A5B8009BFB14E5062001F057FB0028CED10720AD
:10A5C80001F052FB0028C9D1CEE7012B30D194F815
:10A5D8000F24002A3FF403AD94F80E3494F80D04C8
:10A5E800834204D211F0020218BF94F83824264D91
:10A5F80095F82A11002941D132BB834218D2013380
:10A60800DBB2DF0784F80E3412D522238DF86030D0
:10A6180095F87C308DF8623095F8480095F8393017
:10A628008DF8613018A901F0E7FF0E9085F8390020
:10A6380094F8813400206FF3041384F8813484F88B
:10A648000F04FFF773FBCAE494F838648EB9022349
:10A658008DF8683005F50873189395F8480005F5E6
:10A668002D7318A9199301F0D5FF84F8106484F8A4
:10A67800386494F80E3484F839348FE7002AD7D038
:10A688008CE725B0BDE8F08F38100020141B00209F
:10A698002DE9F04F8A468BB091460746002800F016
:10A6A8008D81002900F08A810368002B00F08681E3
:10A6B8004368002B00F082818368002B00F07E81C4
:10A6C800C368002B00F07A81104601F091FF002842
:10A6D80000F07681BC4CBD4D384601F03FFA4FF48E
:10A6E800EE620021204603F029FF4FF4A162002109
:10A6F800284603F023FFB64BC4F8283100264FF054
:10A7080001080F2305A948468DF8143084F84890AD
:10A7180084F8186184F88C6085F80E8485F80D84B7
:10A7280001F06AFF801B18BF01204FF00A0B84F864
:10A738001C0105A994F848008DF814B001F05CFFDD
:10A748004FF0060984F8DC0005A994F848008DF854
:10A75800149001F051FF102384F8DD0005A994F846
:10A7680048008DF8143001F047FF1123C4F89C000D
:10A7780005A994F848008DF8143001F03DFF122324
:10A78800C4F8A00005A994F848008DF8143001F029
:10A7980033FF1323C4F8A40005A994F848008DF8E2
:10A7A800143001F029FF14230DEB0301C4F8A800AD
:10A7B80094F848008DF8143001F01EFF1723C4F8F0
:10A7C800AC0005A994F848008DF8143001F014FF86
:10A7D800182384F8B10005A994F848008DF81430BE
:10A7E80001F00AFF1923C4F8B400C4F8BC0005A995
:10A7F80094F848008DF8143001F0FEFEC0B21E2314
:10A8080084F8B80084F8C00005A994F848008DF8C9
:10A81800143001F0F1FE1F2384F8C40005A994F850
:10A8280048008DF8143001F0E7FE202384F8C500B5
:10A8380005A994F848008DF8143001F0DDFE2123B5
:10A84800C4F8C80005A994F848008DF8143001F040
:10A85800D3FE0B23C4F8CC0005A994F848008DF862
:10A86800143001F0C9FE0C23A4F8D00005A994F80F
:10A8780048008DF8143001F0BFFED4F89C306365B1
:10A88800D4F8A030A365D4F8A430E365D4F8A83090
:10A898002366D4F8AC30636604F5087307A90490FE
:10A8A800A4F8D200079394F848008DF8246004F5C2
:10A8B8002D73089384F8B080C4F894B084F8989005
:10A8C800C4F84CB084F8509084F8688001F0A2FE77
:10A8D800C5F848A3FEF7C8FD32463E4B00964FF038
:10A8E800FF3105F55A70C4E90B66C5F8447385F85D
:10A8F800816484F81981C5F8408306F0D1F832469E
:10A90800354B00964FF0FF3105F5607006F0C8F83A
:10A918003246324B00964FF0FF3105F5667006F06F
:10A92800BFF832462E4B00964FF0FF3102AE05F5C8
:10A938007D7006F0B5F8304606F046F896E8030054
:10A9480004F5907383E80300264BC5F84C33264B77
:10A95800C5F85433254BC5F85C33254F254BC5F84E
:10A968005033254BC5F8583305F553703B68984765
:10A9780004F5A47003F016FB20B1112630460BB085
:10A98800BDE8F08F204601F09DFA0028F5D100F0CF
:10A99800C7FFB8B9194801F0F7FA06460028ECD104
:10A9A8007B69984703F094FDBB6D94F819019847AB
:10A9B800FB6A9847012385F88234DFE70326DDE741
:10A9C8000926DBE71326D9E738100020AC1700204A
:10A9D80000030001359D0008ED9500082D9600083C
:10A9E800258E0008FD8F0008B58F0008E18D00084E
:10A9F800382101088D8F0008658F0008201100207C
:10AA080008B5034B0020C3F84003FEF7CDF908BD95
:10AA1800AC17002010B5FFF7B3F90A4C60B90A4B20
:10AA280093F81831022B02D1084BDB6A98470123AF
:10AA3800C4F84033002010BDD4F84003013818BFD3
:10AA48000120F8E7AC170020381000203821010851
:10AA580038B5134C04F55A7006F080F804F56070A8
:10AA680006F07CF804F5667006F078F804F57D7059
:10AA780006F074F800F040FF0A4B0025DB6A98479F
:10AA8800C4F84053FEF7F2FD074908484FF4EE6258
:10AA980003F040FD0123C4F84033284638BD00BF09
:10AAA800AC1700203821010838100020C808002001
:10AAB80030B52A4B89B0054693F8DD008DF80200C1
:10AAC80093F8DC009A6A8DF8030000200192029046
:10AAD8000C4600293ED00592D3F8882006921A8F9A
:10AAE800D3F82811039152BA93F81A11ADF81C2023
:10AAF80093F87C2093F848308DF810008DF81110E9
:10AB08008DF81E208DF81F300DF1030201AB0DF1F9
:10AB1800020103A800F06EFE9DF90200FEF766F937
:10AB2800607002A800F0B6FFB0B9029A0F2A0DD8DB
:10AB380063789A420AD81544AB42A3EB02012CBFB2
:10AB4800002001202170C00009B030BD002323700F
:10AB58000820F9E70320F7E71320F5E7381000206D
:10AB68001FB50446002800F0FD8000783F2800F259
:10AB7800F380DFE810F0400046004B00500054001E
:10AB880058005D00F100F100F100F100F100F10062
:10AB9800F100F100640068006C0077007E0081001D
:10ABA8008400890087008B008F0092009500980030
:10ABB8009B009E00A200AA00A600AE00B100B5004E
:10ABC800BE00BA00BC00F100C200F100F100F100C3
:10ABD800F100F100F100F100F100F100F100F100E5
:10ABE800F100F100F100F100CA00CE00D300D70057
:10ABF800DB00DF00E8005D4B93F81831237104B0E7
:10AC080010BD5A4B93F82C31237102E0606803F0B1
:10AC180065FB0020F3E7606803F0A6FBF9E7534BF8
:10AC280093F81A31F0E7514BD3F8E0306360F0E75E
:10AC38004E4B211D93F82C0103F0AEFBE9E74B4B7B
:10AC480093F81931E0E7494B93F88C30DCE71D2382
:10AC58008DF80830454B02A993F8480001F0CCFC68
:10AC68006060D6E7424B043493E8030084E80300AD
:10AC7800CFE7404B0434F7E73F4B0434F4E73F4B4E
:10AC88000434F1E71B23E3E71A23E1E7374B93F892
:10AC98006830B9E7354B5B6DC8E7344B9B6DC5E74A
:10ACA800324BDB6DC2E7314B1B6EBFE72F4B5B6E40
:10ACB800BCE72E4B93F8DD30A6E72C4B93F83930E0
:10ACC800A2E72A4B93F8DC309EE7284B93F83830FC
:10ACD8009AE7264BDB6CA9E7244B93F8503093E7AF
:10ACE800224BD3F88430636093E7204B9EE7244BD4
:10ACF8009CE71E4BD3F8CC30F5E71C4BD3F8283132
:10AD0800636001F00DFDA06083E7184BD3F8903025
:10AD18008CE7164BB3F88830A3807AE7134BB3F867
:10AD28008A30F9E7114BB3F8D030F5E70F4BB3F899
:10AD3800D230F1E70D4B93F848200AB1062A13D117
:10AD4800B3F84C37E8E7094B93F848200AB1062ACC
:10AD58000AD1D3F8503769E7204604B0BDE810405F
:10AD680000F0CEBD03204AE7182048E7381000203D
:10AD7800A4100020EC100020AC100020F4100020DB
:10AD8800C808002073B5044600285ED0A04DD5F849
:10AD980040339A0700F15F8202783F2A00F2568218
:10ADA800DFE812F0400046004E0056005A005F00EF
:10ADB800640070007A007F00840089008E00930090
:10ADC80098009D00A7005402AC00CC00DF000601EB
:10ADD800280119012C013C014001440148014C01A2
:10ADE800500162018A0178019C01A201A901AE010A
:10ADF800B301540218025402540254025402540279
:10AE0800540254025402540254025402540254028A
:10AE180054025402540227022C02310236023B0229
:10AE280040024A02007902B0BDE87040FEF7AEBAAF
:10AE38000379022B09D0774A82F82C31002005E0EB
:10AE4800406803F03DFA0028F8D0032002B070BD36
:10AE5800406803F079FAF6E76E4B027983F81A2115
:10AE6800ECE76C4B4268C3F8E020E7E7694D4168BE
:10AE780095F82C0103F086FA0028E6D16368C5F836
:10AE8800E430E3E741680029DFD0002001F0A8F9A9
:10AE98000028D3D01120D9E741680029D5D0012056
:10AEA800F4E741680029D0D00820EFE7416800297D
:10AEB800CBD00920EAE741680029C6D00C20E5E795
:10AEC80041680029C1D00D20E0E741680029BCD0C5
:10AED8000E20DBE741680029B7D00F20D6E74E4C9B
:10AEE8004C4B007983F81901A36D9847E36A98479A
:10AEF800A4E7484B027983F88C209FE7454D037AF5
:10AF08008DF8003095F8480095F87D308DF80130BF
:10AF18000722694601F083FB002896D0636895F8FC
:10AF2800480000930022694601F079FB00288CD084
:10AF38006C35D4E9010185E803007FE7354D037AD4
:10AF48008DF8003095F8480095F87D308DF801307F
:10AF58000722694601F063FB00283FF476AFB43559
:10AF6800E7E72C4D037A8DF8003095F8480095F8FE
:10AF78007D308DF801300722694601F050FB00282A
:10AF88003FF463AFD4E9010105F1740383E80300DA
:10AF980095F81831022B7FF451AF95F82C31002B1E
:10AFA8003FF44CAF1C4BDB6A9847FEF7BFF945E707
:10AFB800184D037A8DF8003095F8480095F87D30E3
:10AFC8008DF801300722694601F029FB00283FF47B
:10AFD8003CAFBC35ADE74368009301238DF80430DE
:10AFE8000C4B694693F8480001F026FB00287FF4D3
:10AFF80025AF2AE7436800930023EFE703795A1E39
:10B008000E2A3FF622AF034A82F8683016E700BFDF
:10B01800AC1700203810002038210108904B4268F6
:10B028005A650BE78E4B42689A6507E78C4B426876
:10B03800DA6503E78A4B42681A66FFE6884B42687E
:10B048005A66FBE6864C037994F848008DF8003080
:10B058000622694601F0E3FA00283FF4F6AE9DF8AF
:10B06800003084F8DD30E9E67D4C03798DF8003056
:10B0780094F8480094F87C308DF80230052269462F
:10B0880001F0CDFA00283FF4E0AE9DF8003084F8D6
:10B098003930D3E6724C037994F848008DF80030C3
:10B0A8000A22694601F0BBFA00283FF4CEAE9DF8AB
:10B0B800003084F8DC30C1E6694C037994F8480024
:10B0C8008DF800300922694601F0A9FA00283FF4FA
:10B0D800BCAE9DF8003084F83830AFE6604B42686B
:10B0E800C3F89420DA64A9E65D4B027983F89820C6
:10B0F80083F85020A2E65A4B4268C3F884209DE6A4
:10B10800574B4268C3F8CC2098E6012B40F0A38047
:10B11800544C2421204603F013FA636A984201D064
:10B12800172093E61C2104F1280003F009FA636C48
:10B138009842F5D1FC2104F1480003F001FAD4F853
:10B1480044319842ECD1D42104F5A47003F0F8F905
:10B15800D4F81C329842E3D1902104F5087003F02A
:10B16800EFF9D4F8B0329842DAD14FF4946104F58B
:10B178002D7003F0E5F9D4F854379842D0D1142152
:10B1880004F5EB6003F0DCF9D4F86C379842C7D1CA
:10B19800334E214630464FF4EE6203F0BBF92046A9
:10B1A8004FF4EE62002103F0C9F995F8113485F8DF
:10B1B800E033736FC5F8E43396F87D3085F8F033E3
:10B1C80040F20123A5F8F233274B96F819019B6D3D
:10B1D800984733E68379012B3FF637AE204B426818
:10B1E8004068C3F8282100F089FE00283FF42EAEFD
:10B1F80050E61B4B4268C3F890201FE6184B828824
:10B20800A3F888201AE6164B8288A3F88A2015E648
:10B21800134B8288A3F8D02010E6114B8288A3F83C
:10B22800D2200BE60E4B93F848200AB1062A14D117
:10B23800A288A3F84C2701E6094B93F848200AB1E5
:10B24800062A0AD16268C3F85027F7E502B0BDE8BC
:10B25800704000F057BB0120F8E51820F6E500BF64
:10B2680038100020C8080020382101082DE9F041D5
:10B2780086B00023ADF800300646002800F0E280D2
:10B28800FEF77EFD20B10124204606B0BDE8F0811E
:10B2980000F02CFD0028F6D100F022FD014618B977
:10B2A8006948142203F04AF9684D95F8813401225F
:10B2B80043F0040385F8492485F8813433788DF800
:10B2C80004300021013B8DF805208DF807100D2B67
:10B2D80000F2B080DFE803F007AEAEAE525A7DAEA2
:10B2E800AE85AEA28F9ED5F8404314F02004CAD193
:10B2F800DFF85C81574FFEF7B7F8224696F905103C
:10B3080098F8480001F0E5F988F83900B37988F829
:10B318003830204607238DF80530FEF737F8FF232D
:10B3280007F58670A5F80C3185F80441C5F8087151
:10B3380003F01AF807F58A7002F0D0FF2046FDF7EF
:10B348007FFE044640B196F9051098F8480001229E
:10B3580001F0BFF988F83900D5F884343361002C3E
:10B368006CD000F0BDFC00288ED195F8813485F8AA
:10B37800100460F3820385F8813485E7002269466A
:10B38800022000F0DBFA10B31324E5E795F8113436
:10B398008DF808302E4BB28893F839108DF80910C3
:10B3A80093F838108DF80A10D3F880100391D3F869
:10B3B8008410049193F84800ADF8142002A901F014
:10B3C8009DF9D5F8403343F00203C5F84033002413
:10B3D800C2E7214BB28896F90C10B068DB6B98472E
:10B3E800EFE702A90D2000F027FB0028EFD000228C
:10B3F80069460D20C5E7164B93F81831D3B934794F
:10B4080004F0070000F077FA8DF800400122694641
:10B418001020B6E7002269461220B2E78DF807200F
:10B4280000F05AFA044638B900F053FA204600F002
:10B4380055FA91E702248FE701248DE701A800F06F
:10B44800A1FB21E703241FE7F41B0020AC17002011
:10B4580038100020AE170020382101082DE9F04FE0
:10B4680091B000260391054618B9032011B0BDE834
:10B47800F08FFEF785FC8246002840F06481B84CC6
:10B4880014220146074604F2344003F057F801231A
:10B4980084F8353484F80E342A789A4200F0B08063
:10B4A800032A00F0BF80002A40F0C98084F80D34D8
:10B4B800022295F80490D5F80880AE8995F90EB067
:10B4C80062F347179A46A74B022493F87C2093F817
:10B4D80048008DF8244009A98DF8262001F08CF841
:10B4E800BAF1000F00F02D819E4B93F81A21B2B9E2
:10B4F80040B25845B8BF584693F87C208DF81400E0
:10B508008DF8162093F84800052205A901F087F860
:10B518000028AAD0934B9DF8142083F83920198F5E
:10B528001A8F93F82C010291996A069152BA002851
:10B5380000F0058193F81B0100B9186393F818010E
:10B54800ADF83C20013893F87C208DF83E20D0F1EE
:10B55800000B93F848208DF83F204BEB000B824AF4
:10B5680093F83A0093F81A4101900D914FF00100B9
:10B57800D3F88810D3F828318DF830000E910B934A
:10B58800511C06AB0BA88DF8314000F033F9019B34
:10B598004FEA0B1B4BEA431B4FF0000A4BEA801B98
:10B5A8004BEAC413D0456E4C019308BF5646324649
:10B5B800414604F59C709B46CDE907AAA4F800A073
:10B5C80084F810A402F0A6FFF9B2A770C7F34217D7
:10B5D800F2B2042F634E019B84F8372233D0072F31
:10B5E80000F09D80022F32D00220029B33875C4BF3
:10B5F800002283F810245A4BD3F884342B6135E7A2
:10B60800EB7B082B28BF082384F80D34042395F816
:10B618000490D5F80880AE8995F90EB063F3471702
:10B62800924650E784F80D34D5F804802E8995F9B0
:10B638000AB067F01F079A464FF0000943E7D34660
:10B64800D046D1463FE74FF0010084F81004474F39
:10B6580084F80D11042084F80401FF20D6F8E410C2
:10B6680084F80C0184F8143107A807F59B73C4F813
:10B67800087184F82891C4F8101184F83021C4F8AE
:10B688002C3100F043FC002857D1079BA4F838045C
:10B6980008A8A4F81631C4F8403400F0FBF960BBE0
:10B6A800089BABB196F93900FDF7A0FB94F8373247
:10B6B8002BB3089B0F2B19D807F58B7208A90F20FD
:10B6C80000F0F4F9C8B9089B63F3030B84F814B1CC
:10B6D8000398FDF7B5FC002887D1069B86F83A0049
:10B6E800B36200F0B7F980B3132080E707F286420F
:10B6F80008A900F0DBF90028EAD0132075E707F263
:10B7080086473A4608A900F0D1F90028F5D1089BE8
:10B7180084F82801C4F82C7184F83031D8E7B8F1DE
:10B72800000FD5D0002AD3D04146E01C02F0F2FE2B
:10B7380094F8373201332380CAE7122055E70720EF
:10B7480055E7204657E7012090E62B7884F83434F3
:10B7580094F8813443F0010384F881344BE700BF47
:10B76800AC1700203810002070100020AE17002001
:10B7780037B50B4D8DF8040004460F2295F84800A4
:10B7880001A900F04CFF40B1064A85F81C4192F827
:10B79800813443F0200382F8813403B030BD00BF08
:10B7A80038100020AC17002010B5FFF733F9044615
:10B7B800A0B90B4805F0D2F90A4805F0CFF90A48B4
:10B7C80005F0CCF9094805F0C9F900F095F8FDF73E
:10B7D8004BFE074BDB6A9847204610BD0124FBE768
:10B7E800141B00202C1B0020441B0020A01B002041
:10B7F800382101082DE9F04F90F802908BB00446EB
:10B808008A460192B9F1000F60D14579816890F9B3
:10B81800102090F911801960002D55D0817C8DF889
:10B828001610C07C4FF0020B05A9CDE902238DF854
:10B8380014B000F0E1FE029A47B2BA421646B8BF09
:10B848003E46BA420CDC039BC3F800904D46019B70
:10B858008AF8006083F8008028460BB0BDE8F08FB6
:10B86800A268A189E3898A420B4434BF00250125D7
:10B878009A42ECD3082305A9E07C8DF8143000F037
:10B88800BBFEE289A368B3FBF2F102FB1133012B83
:10B898004FFA80F8DBD122238DF81430E07CA37CAA
:10B8A8008DF8156005A98DF8163000F0A5FE46B292
:10B8B800B742CCD12579002DC9D0E07C8DF824B0D1
:10B8C80007A900F0A7FEC1E71646C0E70025C3E7B1
:10B8D800704770477047704700207047704770473F
:10B8E80070470020704700207047002070470020F4
:10B8F80070470020704770477047704702207047B4
:10B908000220704702207047704700207047704738
:10B91800704700207047002070477047704700004C
:10B9280010B5054CFC222046002102F007FE00203D
:10B93800C4E9000010BD00BFC81C00202DE9F0417B
:10B9480080461546002942D0244B002403F1010CFF
:10B958001A462001103312F8016F002E39D19A428D
:10B96800F9D11F4F3B680BB9C7F800C07B680BB112
:10B97800C3F800C03B18002201349A6083F80C8099
:10B988000D302301AAB23844FD50C7F804C002F0B4
:10B99800C1FDB8F1050F17D0A8F10808B8F1020FDA
:10B9A8008CBF4FF000084FF0010807EB0414002388
:10B9B8006371D7F8F83084F8048001332B44C7F852
:10B9C800F8303046BDE8F0814FF00108EDE7012678
:10B9D800F7E701340F2CB9D10226F2E7CF1C00207B
:10B9E800C81C002010B510B3124A1368984204D13D
:10B9F80003681360002304E00B4613B119688842FA
:10BA0800FAD15168884208BF53600BB101681960C8
:10BA1800D2F8F8308168013B00245B1A04602146A3
:10BA2800C2F8F830102202F089FD204610BD01202E
:10BA3800FCE700BFC81C0020054B1B6813B11A792E
:10BA48008242FAD1002B0B600CBF03200020704704
:10BA5800C81C002010B5054B186800B910BD037B41
:10BA680004680BB9FFF7BEFF2046F6E7C81C0020A4
:10BA780010B5074B186800B910BD03790468052B89
:10BA880002D0083B022B01D8FFF7ACFF2046F2E7B3
:10BA9800C81C002028B1044BD3F8F83003600020FC
:10BAA80070470120704700BFC81C00202DE9F041F5
:10BAB80007460E4615463AB331B3144B1C680023AB
:10BAC8002CB93046FFF7E6FF0020BDE8F081A268F8
:10BAD800F91A0132914210D32279EA54581C22896A
:10BAE8005FFA80F8611D55FA80F002F013FDA36833
:10BAF800246898445FFA88F3E2E720462468FFF751
:10BB080071FF002CF9D1DCE70120DEE7C81C00201A
:10BB18000238C0B211289ABF014B185C0020704748
:10BB2800C31A010830B50B4B93F820200446084689
:10BB380072B100211C330578A54208D00131984222
:10BB4800CDB20CBF04480430AA42F4D8002030BD5E
:10BB58001046FCE7C41D0020D01D002010B5084C7D
:10BB680000232060142204F10C00FF2184F8203007
:10BB7800C4E9010002F0E2FC012384F8213010BD81
:10BB8800C41D002010B50E4A92F82010042915D8BB
:10BB9800936804781C7044785C70C078D870013160
:10BBA8000020987082F8201002F11C018B4214BF0B
:10BBB800043302F10C039360012010BD0020FCE760
:10BBC800C41D0020094B93F8200068B15A6803F19E
:10BBD8001C018A4200F1FF3014BF043203F10C0249
:10BBE80083F820005A600120704700BFC41D002060
:10BBF80010B5074B93F820200446084632B159681F
:10BC0800FFF790FF10B101234470837010BD00BF8F
:10BC1800C41D002008B5064B93F820202AB15968A6
:10BC2800FFF780FF08B1407808BD0120FCE700BF9E
:10BC3800C41D002030B50A4A92F82010536882F8D3
:10BC4800210061B1916801241C32DD78587005B972
:10BC58009C7093420CBF034B04339942F5D130BD1D
:10BC6800C41D0020D01D002008B5044B5968FFF7FB
:10BC780059FF003818BF012008BD00BFC41D0020AF
:10BC88002DE9F3410422154E044600210DEB020074
:10BC980096F8208002F052FC0025EBB2984502D8B5
:10BCA80002B0BDE8F0817368197821705A78627023
:10BCB8009F785FB1336820469B689847FFF782FFFB
:10BCC80017B901A8FFF75EFF0135E6E7DB788DF8C5
:10BCD80004108DF805208DF80730EFE7C41D00200B
:10BCE800014B93F820007047C41D0020034B93F8C4
:10BCF8002000042894BF002001207047C41D0020A4
:10BD08001FB50024CDE90244C41F8DF800408DF80A
:10BD180001100C0AADF80420090C120C8DF8031060
:10BD28008DF806208DF8073002461B0A0121684667
:10BD38008DF802408DF8083002F05DFA002818BF2F
:10BD48000F2004B010BD2DE9F04188B017460D460C
:10BD58000F9A064600284DD000240121CDE904445D
:10BD68008DF810109DF838108DF81510ADF81630B4
:10BD7800190CCDE900441B0ECDE902448DF81930A9
:10BD8800ADF81A20130C120E07948DF818108DF8C0
:10BD98001C308DF81D20E3B24FEA0318002D5FFA1E
:10BDA80088F803DC002008B0BDE8F08101331021D9
:10BDB8008DF81F303A466B460DEB010002F0B1F9E1
:10BDC8000346C8B9102DAC46A8BF4FF0100CDAB224
:10BDD800624503F1010303DB103D2DB20134DAE7BC
:10BDE80008EB020020326A44315C12F8202C4A40E9
:10BDF8003254ECE70A20D6E70F20D4E701380328AD
:10BE080015D8DFE800F002080C100A4B1B681B6904
:10BE18000B6000207047074B1B685B69F8E7054B10
:10BE28001B689B69F4E7034B1B68DB69F0E7052097
:10BE3800704700BFE81D00202DE9F041C4B00C4652
:10BE48004A9E17461D468046B8B3B1F5807F36D85E
:10BE58004FF488720021684602F070FB4923009372
:10BE68004FF48073ADF804302B0C8DF80830330C88
:10BE7800ADF80650ADF80A608DF80C302246002364
:10BE8800414604A82D0E360E8DF80E308DF8095057
:10BE98008DF80D608DF80F4002F03CFB04F11001A5
:10BEA8004B9A3B4689B2684602F025F910B1012841
:10BEB80018BF0F2044B0BDE8F0810A20FAE70E2031
:10BEC800F8E7000010B590B10A4C28220021206044
:10BED80002F034FB2368084A1A6000204FF0FF3252
:10BEE800C3E90302C3E90522C3E9072210BD0920FB
:10BEF800FCE700BFE81D002000010101024B1B68A0
:10BF080018600020704700BFE81D002030B1044BC6
:10BF18001B68DB6801330360002070470A20704704
:10BF2800E81D002073B50E46002101911D4633B36C
:10BF380001A9FFF763FFD0B9019C631C04D0A3B229
:10BF4800D31A002B10DDE2180E4B2A601B689B7871
:10BF58006BB9121B63EB0303B24273F10003ACBF6E
:10BF680001200020C00002E003D12C60072002B0AD
:10BF780070BD230C1B0403F580331A44E4E70A2040
:10BF8800F5E700BFE81D002028B1044B1B681C33EF
:10BF98004362002070470A20704700BFE81D002058
:10BFA8001FB50446F0B1002303A8039302F07AF901
:10BFB8000E4ABDF80C30126820469380E38200F0E8
:10BFC80052FA60B904F1180300932168012313227F
:10BFD80002F088F840B9204600F045FA00B1112077
:10BFE80004B010BD0A20FBE70F20F9E7E81D002088
:10BFF800F0B5054687B01C463BB32F4E3368DB6867
:10C00800834257D894F82020002A14BF0922082216
:10C01800834205D3204600F05AFA70B111200AE095
:10C02800002301900093A36894F82810606AFFF732
:10C038008AFE0028EED007B0F0BD23792168B4F855
:10C0480008C0A768043B9AB209B90A20F3E7B2F519
:10C05800807F2DD8ADF80EC08DF817304FEA174CF9
:10C0680004F12C033F0E8DF8117000932F0C082358
:10C078004FF0490EADF80C008DF814708DF81600CD
:10C088002F0E0DEB0300CDF808E08DF810C0ADF8C9
:10C0980012508DF8157002F025F808B10F20CAE784
:10C0A800204600F014FA0028B8D13368DD60C2E7F2
:10C0B8000E20C0E70620BEE7E81D00202DE9FF415D
:10C0C8000A9D80460F4616461C46002D5AD000236E
:10C0D80003A910460393FFF791FE18B1062004B098
:10C0E800BDE8F081039B9C4201D80133F6D1284674
:10C0F80000F05EF9002847D1264B1A78424503D054
:10C108001A79424542D10120AA68BA4240D103EBCC
:10C118008002EB6A92F801802979CDE9004304395D
:10C12800927828683B4689B2FFF786FE0028D6D168
:10C1380095F820300194002B4FF00103009314BFB1
:10C148004246082295F82810686A3B46FFF7FBFD2F
:10C158000028C4D1013E032EC1D8DFE806F002074B
:10C168000B0F0D4B1B681C611C62B8E70A4B1B6860
:10C178005C61F9E7084B1B689C61F5E7064B1B6897
:10C18800DC61ACE70A20AAE71020A8E70C20A6E7A4
:10C198000220A4E744010020E81D00201FB50A463C
:10C1A8000B2A4FF00001CDE90011CDE9021107D0AB
:10C1B8000C2A13D00A2A0FD00B2005B05DF804FB17
:10C1C800012802D120238DF80030684602F013F8C8
:10C1D800002818BF0F20F0E73023F4E70B21F4E71D
:10C1E80038B5054602F002F8044678B97DB9094B1E
:10C1F8001B680B219878FFF7D1FF38B90C21FFF79E
:10C20800CDFF18B90A21FFF7C9FF00B10F24204656
:10C2180038BD00BFE81D00202DE9F04380468FB0EF
:10C228000C461746002A6BD0002969D000252946FC
:10C238001D2206A8059504F0A3FE8DF81350344D71
:10C248002B680DF114099E88CDF804900DF11303A5
:10C2580002933B7900933B6832462146404601F001
:10C26800E6FF00284ED138683A79494602F052F97B
:10C27800384600F04FF8002846D13C7AFA79BB7965
:10C28800240444EA02241C432B689A6894423DD94A
:10C298009C609DF813000B21FFF780FF034658BBF5
:10C2A8000C21FFF77BFF034630BB0A21FFF776FF1F
:10C2B800034608BB7B7ABA7AFF7A3F0447EA02272B
:10C2C8001F433A46334621460920FFF719FD034626
:10C2D80090B933463A4621460820FFF711FD034638
:10C2E80050B92A689DF8131091700021D1604FF061
:10C2F800FF31C2E90411916118460FB0BDE8F0831F
:10C308000A23F9E70F23F7E71023F5E70323F3E7F9
:10C31800E81D002010B50446002845D00168002912
:10C3280042D011F8013B43710322063002F0F2F8C3
:10C338002046032250F8091B043102F0EBF821686B
:10C34800CB79E3600A7A43EA0223E3604A7A43EA54
:10C358000243E3608A7A43EA0263E360CB7A237498
:10C368000B7B63742379212B1AD110220D3104F130
:10C37800120002F0CFF81D222168501C8B5C63620A
:10C38800085C43EA0023901C6362085C033243EABA
:10C39800004363628A5C43EA02636362002010BD63
:10C3A800112B03DC0D22E7E70220F8E70120F6E76E
:10C3B80010B50446002854D00168002951D00B78E4
:10C3C80043714B7883608A7843EA02238360CA7892
:10C3D80043EA024383600A7943EA026383604B7944
:10C3E80003738B79C381CA7943EA0223027BC38131
:10C3F80002F00F020831103002F08CF8237B002283
:10C4080003F00F0384F8202084F82820227903F110
:10C418000800111A04290DDD21680933043AD21ADB
:10C42800085C84F82000D2B2606A84F82820194495
:10C4380002F070F8237922681A44002012F8043CAC
:10C44800E36212F8031C43EA0123E36212F8021CB8
:10C4580043EA0143E36212F8012C43EA0263E36210
:10C4680010BD0220FCE710B5044660B3036853B35F
:10C478000279162A29D942791A700146082251F8F8
:10C48800060B013002F050F82146082251F80E0B35
:10C49800093002F049F82368E28A5A74E38A22686C
:10C4A8001B0A93742368A269DA74A36922681B0AB9
:10C4B80013752368628B5A752368E27E9A75172371
:10C4C8002371002010BD0120FCE70220FAE738B5EF
:10C4D8000446002863D00168002960D0037B90F8E7
:10C4E800282003F00F03002A57D10833207904329B
:10C4F8001344984255D363790B702368A2685A7025
:10C50800A36822681B0A937023686289DA7023681B
:10C51800E27A1A712368227B5A712368E2899A7138
:10C52800E38922681B0A2146D371227B51F8100B3C
:10C5380002F00F02083001F0EDFF237B94F8282069
:10C5480003F00F0303F108052AB1226894F82010BC
:10C55800515503F10905206894F82820616A284498
:10C5680001F0D8FF94F828302268E16A2B44D154AE
:10C578005A1CE16A206892B2090A81549A1C2168FF
:10C58800E08D92B28854DA1C216894F82F0092B298
:10C59800043388542371002038BD0933A6E70120ED
:10C5A800FAE70220F8E70000024B1A8810431880C7
:10C5B800704700BFEC1D002008B5074B1B883BB136
:10C5C800FEF728FA00280CBF00206FF0020008BD13
:10C5D8006FF00100FBE700BFEC1D002010B5034B16
:10C5E80000241C80FEF70CFA204610BDEC1D00202C
:10C5F800B0FA80F04009704782B018B9084602B016
:10C6080000F0D0B8002002B0704710B9084600F01A
:10C6180083B9704710B9084600F09AB970470346C5
:10C62800084611460BB900F0E7B90020704710B969
:10C63800084600F045BD704710B9084600F008BA32
:10C648000020704710B40446084611461A46019B5C
:10C6580014B910BC00F01ABA10BC7047034608465B
:10C6680011460BB900F044BA0020704710B40446D4
:10C67800084611461A4614B910BC00F0B1BA002099
:10C6880010BC704730B40546084611461A46DDE925
:10C6980002341DB9029430BC00F02EBB002030BC1F
:10C6A800704710B9084600F0DFBB0020704710B98A
:10C6B800084600F043BD0020704710B9084600F056
:10C6C800EEBB0020704710B9084600F0EBBB002015
:10C6D80070470346084611460BB900F005BC002018
:10C6E800704710B40446084611461A46019B14B90F
:10C6F80010BC00F0FBBB092010BC704710B90846FD
:10C7080000F03CBD704710B40446084611461A466E
:10C7180014B910BC00F05CBDC8B210BC7047000072
:10C728000048704703000101064B10B51B6A044618
:10C73800984730B10448054B204498428CBF0020EC
:10C74800012010BD38210108403576C9405DC6007A
:10C75800F0B5114B85B00C4610491F56054601F03F
:10C7680045F80F4BE4B25E6A072D4FF00103CDE99F
:10C77800024301460AD105220023CDE900234FF4E4
:10C788007A727A431846B04705B0F0BD08220020F7
:10C79800CDE900203A46F5E7FF1A0108D81A010842
:10C7A800382101081FB5002300930378013B382B7B
:10C7B80000F28580DFE803F01D23838383208383D1
:10C7C80083834042444B835356595C5F6265836D53
:10C7D800206F74797B7E7E80872583838383838320
:10C7E80083838383838383898B90838389908392D4
:10C7F8009600C378002B62D0022300935FE0837811
:10C80800F8E743788DF8043007238DF805308378EE
:10C81800003B18BF01235B008DF8063010238DF80C
:10C828000730334B1B6801A803F59062CDE902235A
:10C8380000F0BCFF009042E04023DEE72023DCE765
:10C84800827890F9013042B92A4AD35CD5E78278D8
:10C8580090F901300AB9284AF7E7284AF5E740F67F
:10C86800B833CAE74FF47A73C7E74FF4FA63C4E7FB
:10C8780041F28833C1E741F27073BEE74FF4804359
:10C88800BBE71F484FF47A7101F028FE00F5FA6003
:10C89800D0E71C4BB1E7164B1B6803F59063ACE778
:10C8A800134B1B6803F28C43A7E71023A5E7104B33
:10C8B8001B68A2E70123A0E74FF083430093009889
:10C8C80005B05DF804FB104BF8E7104B95E740F214
:10C8D8001123ADF80030F2E703238EE790F9013019
:10C8E8000B4AB2E70B4990F9010000F07FFFA1E77E
:10C8F800F41D00200F1B01081F1B0108171B01084E
:10C9080018FCFFFF00EA06379A99094040F70937F3
:10C91800FF1A0108D81A010837B50B4B02781B68B3
:10C928000C2101FB02335B7A03EB4304074B1D68C0
:10C9380003690093C3684278816805EBC40000F07E
:10C94800D5FC03B030BD00BFF41D0020F01D002051
:10C9580030B587B0027A6423ADF80030012A4FF071
:10C968000003CDE90133CDE9033301468DF80230E8
:10C978008DF8143027D0022A2ED012BB006800B3DD
:10C988004B68F3B1194A1A4C1060694618222360A3
:10C9980001F0C0FD174B246893E807000C3384E8C6
:10C9A800070093E8070004F10C05032385E8070056
:10C9B800A4F88C34012204F28C4104F5906000F054
:10C9C80086FC07B030BD0A4908684360036100F27D
:10C9D8008C4100F59060F2E7054B1B68B3F88024A2
:10C9E800B3F88C140A43A3F88024EAE7F01D00206A
:10C9F800F41D00203411010808B503460A2924D87B
:10CA0800DFE801F006232323230B161B2321210033
:10CA1800BDE808400068FFF787BE90F900009978E4
:10CA2800072271B900F013FC003818BF012008BDB7
:10CA3800052293F900000021F4E790F900005978E5
:10CA4800EEE70221EEE70722F3E70020EFE7000018
:10CA580010B504791CB1012C0BD0002010BD0A4B75
:10CA680001681B68012203F5906000F030FC01208A
:10CA7800F4E7054B01681B68224603F28C4000F07E
:10CA880026FC2046EAE700BFF41D0020F7B507287A
:10CA9800144D1C46A8BF072058700E462946174655
:10CAA80000F0A4FE94F90130A070072B13D13220B6
:10CAB80000F09CFD0C4BDB6D0546984704F10C0219
:10CAC80008340346019200943A463146284600F05D
:10CAD80092FD03B0F0BD054A55F82310D05C00F074
:10CAE8007DFDE7E7D81A010838210108FF1A010877
:10CAF8002DE9F04F344F90F901607B68D0F804902D
:10CB08008BB00446884698470546002859D1E37CEF
:10CB180073B92E4A2378126803EB4303990002EB9A
:10CB28008303D3F80490B9F1000F01D152F80190B2
:10CB3800274B484613F906B0FB689847A37CD7F8FB
:10CB480018A022890993072E28D100230121CDE9B5
:10CB58000223204A0693CDE90431CDE907330521A4
:10CB6800CDE900214FF47A7202FB0BF24CF25031FE
:10CB78001846D047637C13B3174B995D7B6D0D3115
:10CB8800C9B228469847E07C3246494600F040FE44
:10CB980088F8006001200BB0BDE8F08F0021012566
:10CBA8000823CDE90013CDE90715CDE90511CDE935
:10CBB80003110292A1782B465A462846D9E7074B1B
:10CBC800DBE70020E7E700BF38210108F41D00205B
:10CBD800FF1A0108854501001F1B01080F1B0108EA
:10CBE8002DE9F04F8DB090F90130DFF8F8A0DFF8AB
:10CBF800F890CDE90A123D4A017812F903B0DAF843
:10CC080000203B4B0C2505FB01221B68527A18219A
:10CC180001FB0233044693F9021090F9020000F078
:10CC2800E0FD3449064694F9010000F0DFFDA268F2
:10CC380061688046304600F006FD2178DAF8002069
:10CC4800D9F80C306943074650589847D9F81C3032
:10CC58009C4694F901300025072B4FF47A63CDE9FF
:10CC68000753CDE905552DD10123CDE903530523FC
:10CC7800CDE901534FF47A7303FB0BF30093394664
:10CC8800434646F2A81228466746B8472378DAF89A
:10CC980000200C214B4394F90110D05800F0DAFD24
:10CCA800A18994F90100FFF753FD0B9B217B1860C4
:10CCB800D9F85430284698470A9B01201E700DB0B9
:10CCC800BDE8F08F01200823CDE90350CDE9010329
:10CCD8002A46CDF800B0654643463946A8470120A4
:10CCE8000546D3E7F41D002038210108FF1A010882
:10CCF800F01D0020D81A01082DE9F04F8FB000244C
:10CD080005468A46914698460494ADF81440ADF815
:10CD1800024007264FF0010B2B7AA34206D9686818
:10CD280004A9204400F0F4FB00285DD102238DF80B
:10CD3800083002A86B7A8DF80A30FFF733FDAB7A1A
:10CD48008DF81D309DF811308DF81E309DF8123089
:10CD58008DF81F309DF810308DF82030EB7A8DF863
:10CD680021302B7B8DF822306B7B8DF823301023FC
:10CD78008DF81C608DF824303A4E8DF82C000DF19A
:10CD880002030A93072332688DF82D30ADF834304A
:10CD98002B680C9206930DF1120204AB0DF11101F0
:10CDA80006A800F0CFFB072805460BD130680C22F7
:10CDB800002100F5906001F0C1FB3368BDF8022046
:10CDC800A3F880249DF811308AF800309DF81230BD
:10CDD80089F800309DF8103088F80030189B2846F4
:10CDE8001C700FB0BDE8F08F9DF81330BDF81470BB
:10CDF800ADF802702044C4B2F3B917B3194A002041
:10CE08001168072602464FF00C0C062B1BD10CFBB1
:10CE180000FE51F80EE0BEF1000F04D00BFA00F24C
:10CE28003A4397B2012201301028EED1002A3FF48C
:10CE380073AFADF802706FE75A1E042A01D9062BAA
:10CE4800DCD0062668E747FA00FE1EF0010FEAD09C
:10CE58000CFB00FE51F80EE0BEF1000F08BF0626DD
:10CE6800E1E700BFF41D002038B505464068FFF72C
:10CE78005BFC0722841D002195F90000E4B200F054
:10CE8800E6F908B904F0FD0495F90100072200212C
:10CE980000F0DDF908B904F0FB04204638BD002095
:10CEA8007047000010B503780F2B044618D8406867
:10CEB800FFF73AFC22780B4902EB42020968831C0F
:10CEC80001EB820051F82220DBB21AB903F0FD030E
:10CED80058B210BD032B06BF626842600223F7E711
:10CEE8000020F6E7F41D0020022070472DE9F041EC
:10CEF8003A4D0446286896B00E46904600211F46D3
:10CF08000122032300F59060CDE90411CDE9061153
:10CF18008DF80C108DF80D10ADF80E3000F0B9F941
:10CF280030B92A68B2F8803443F00303A2F8803499
:10CF38002A68637A8DF8203002F59061CDE90912EC
:10CF4800274A94F9083012680B921022ADF8302065
:10CF58000DF10E020D9222680E9262680F92D4E9CA
:10CF68000301A27A8DF8402001228DF8412011AAF0
:10CF780082E80300227DE18A8DF8213018468DF879
:10CF88004C20FFF7E5FB08AB15930DF10D0314904A
:10CF98000093CDF8048003AB04AA39460EA800F02C
:10CFA800C1FB044678B99DF80C10013901F096FAD6
:10CFB80000F158030DEB030010F8483C337020468D
:10CFC80016B0BDE8F0810C2801BF2A68B2F8803499
:10CFD80043F00303A2F88034F1E700BFF41D0020FA
:10CFE800F01D0020F8B50679012E054601D8062067
:10CFF800F8BD0F2E2BD80368187A40F303000722D8
:10D00800002140B200F023F92B680446187A40F357
:10D0180003100722002140B200F019F9A8B1B4FAB0
:10D0280084F4640929680B7A086843F3030243F31C
:10D03800031352B25BB29A42C8BF0124FFF774FBD4
:10D0480048B9002CD3D10420D2E70124EAE7032011
:10D05800CEE70520CCE7002CFBD10C4F29683B68B4
:10D0680006EB460003EB80000C2201F053FA3A6805
:10D078000C2303FB062320465C72B2F880140123BC
:10D08800B3400B43A2F88034B2E700BFF41D002080
:10D0980010B4017801290ED9084B18680C234B43AA
:10D0A800C4180022C250C4E9012200F5906010BCE7
:10D0B800102200F0D5B8002010BC7047F41D0020E5
:10D0C8002DE9F04186B050238DF814300379102BE8
:10D0D800074630D10368DD7B6DBB0224A846642671
:10D0E800062C14D83A68535D03932A44517843EACE
:10D0F80001230393927843EA02437343CDE903384B
:10D1080063B968468DF80040FFF7C2FF0DE0CDF81F
:10D118000C808DF81480CDF81080F2E703AB01A8DD
:10D1280001938DF80840FFF75DFF0134E4B2102C3D
:10D1380005F10305D4D106B0BDE8F0811FB502683A
:10D148000379116851B901A88DF80430FFF7A0FFE1
:10D1580078B9002040B205B05DF804FB02A802923D
:10D168008DF80C30FFF73EFF0628F2D8024B185C0A
:10D17800F0E70320EEE700BFF81A010870B5114E7A
:10D1880001783268104B0C2505FB01221B68527A86
:10D19800182101FB0233044693F9021090F90200AA
:10D1A80000F01FFB2378326861686B43D558A2688A
:10D1B80000F049FA054BA289DB6B01462846BDE819
:10D1C80070401847F41D0020F01D00203821010888
:10D1D800074B9B56C91A431E584258414000884283
:10D1E800B8BF08460528A8BF0520C0B2704700BFD1
:10D1F800071B0108F0B59A42069D03DB9DF9143020
:10D208009A4220DD0020F0BD03EB430331F814C03F
:10D2180005EB830300264CFA06F7FF0707D51F7AAC
:10D2280007F00F0E724502DBB2EB171F0DDD01365A
:10D23800102E03F10C03EED10134E4B22301DBB26A
:10D248009842E1D8DEE70024F8E70120DBE78842CE
:10D2580004DB9042CCBF00200120704700207047BB
:10D2680010B51409B4EB111F03464FEA11100ED381
:10D2780091420CD202B201F00F0133F812400120A2
:10D2880000FA01F124EA010123F8121010BD002070
:10D29800FCE7F0B528B100EB4105012700209142D9
:10D2A80000D3F0BD002435F802CB234607FA04F674
:10D2B80036EA0C0608BF013304F1010408BFDBB2EB
:10D2C800102CF3D118440131C0B2C9B2E7E710B548
:10D2D80000B149B910BD31F8134020F813400133AB
:10D2E800DCB2A242F7D8F5E70023F9E782B030B5FF
:10D2F800048804936AB9B3F5616F18D349F6AF256A
:10D3080042F21072AB4298BF4FF47A72944238BF1F
:10D318001446012C38BF01246143BDE83040C3687E
:10D328008B428CBF5B1A0023C36002B07047642233
:10D33800ECE700002DE9F04F91B01546DDF86C8060
:10D3480004939DF8683009930C46064603F0C2FB27
:10D35800684ADFF8A4B10590A8F5F633303BB3FB73
:10D36800F2F3534303F5F63203F5A83303F5C0731C
:10D378000393182313FB05433032069208930025C4
:10D388004FF0FF3A089BA34207D1002D14BF504627
:10D398004FF0FF3011B0BDE8F08FBDF97030ADF837
:10D3A8002C300B99CDF86C804046CDF8288003F0DE
:10D3B80021FBB4F800906EB9B8F5616F5BD349F6FC
:10D3C800AF2242F21073904598BF4FF47A73994593
:10D3D80038BF99464B46012B38BF01230793002ECF
:10D3E80052D1B9F1640F48D1A0605F46A1680EA878
:10D3F80003F022FB0F9B0093DDE90A120E9B0CA899
:10D4080003F079FA049B0C9A0BB9099B2BB1236999
:10D41800BB4202D1394B9A420DD9394BE760984546
:10D4280009D90023ADF83430069B0D990C931846A2
:10D4380003F0E0FAA060606800B9E760276126B1F0
:10D4480003F052FBE3680344E360D4E903329342F8
:10D45800059B1D996360079B88BFE2604B43E168A9
:10D46800994202D20498A8B9A6B101231D44237594
:10D47800EDB2183486E76423A9E7B9F57A7F0ABFC5
:10D48800204F214FA060B1E7049B0BB9C4F80CB042
:10D498005F46D0E700209342207506D85B1A9A456C
:10D4A80005F1010528BF9A46EDB2002EE1D1B9F188
:10D4B800640F164AADF8346019D049F6B023B9F5AF
:10D4C8007A7F18BF1346904584BF039A9B180C9324
:10D4D8001C9B00930CAF97E806001B9B384603F093
:10D4E8000AFA97E8030003F085FA8246C1E74FF489
:10D4F8006163E8E78051010040771B007F5101001C
:10D508002FEC010080A81201002E930230EC0100DC
:10D518000378032B14D1437803F00F021B098A7098
:10D528004B7083788B80C27843EA02238B8003791F
:10D53800C3F3021203F00F03CA700B700520704783
:10D54800002070472DE9F34798464379057990F90B
:10D5580007609146044690F906208A4683B190F9FF
:10D56800087075B30F2A12D194F909200F2E1ED115
:10D5780094F90A60072D24D1002F08BF012720E065
:10D5880090F90B7090F9092090F90A60E9E7A3690E
:10D59800019394F915300093216994F91430207B94
:10D5A800FFF728FE0028E1D105F0FD05DEE794F934
:10D5B8001D30B3420FDC94F91C30B342DADA05F0BF
:10D5C800FB0528468AF8002089F8006088F8007072
:10D5D80002B0BDE8F0871E46CCE70000024B03FA14
:10D5E80000F0B0FBF1F0704740420F004FF4FA53DF
:10D5F800B3FBF0F0704730B54FF47A750C1F6A43EF
:10D6080000FB042252001EBF00F1FF341219B2FBC6
:10D61800F0F2914238BF1146039A116082004843E4
:10D628001CBF013040084FF47A71121A01FB132312
:10D63800002BCABF03F2E73393FBF1F1B3FBF1F11F
:10D64800049B196030BD38B5400014460D46F4F708
:10D65800DDF901462846F4F727F92146F4F724F9BD
:10D66800F4F716F803F0D0FCF4F7F2F840B238BD3E
:10D678002DE9F74F019300231F469C461C01058A9C
:10D688005FFA84FE04F0F004A54206D8019B82F8F4
:10D6980000C01F7003B0BDE8F08F0EEB4E054FEAD7
:10D6A8004309AD000024466836F809602641F607AC
:10D6B80027D5866806EB050A765916B3067836B973
:10D6C800466926B136F809602641F60719D59AF851
:10D6D800086090F901B046F303084FFA88F8D84576
:10D6E8000FDC46F3031676B25E450ADB9AF809604A
:10D6F80006EB4608C66806EBC806367D4EB9013704
:10D70800FFB20134102C05F10C05CCD10133DBB28A
:10D71800B4E70CF101060EEB040801F80C805FFA7F
:10D7280086FCEEE72DE9FF4704464068DDE90C6713
:10D738001D468A46914603F0D7F923681B1A3B60B9
:10D748004FF000080123337085F80080636813B137
:10D758002368834224D8CAF80080D4F81CC0A3697F
:10D768009CF800E00393D4E9030101AB83E80300CC
:10D77800237D0093DCF80C10237A627A7046FFF759
:10D78800D9FD334638602A46E0694946FFF770FFFD
:10D798002B782BB1C7F80080002004B0BDE8F087D3
:10D7A8003378002B14BF0B200C20F6E737B590F91F
:10D7B800002090F90250954204460FD0013A52B227
:10D7C80095420BD0A368019394F9013000936168E6
:10D7D800E0782B46FFF70EFD0028EFD0104603B087
:10D7E80030BD8842B8BF08467047000051F8200095
:10D7F800054B984205D0054BC31A58425841400082
:10D8080070470120704700BF90D0030020A1070097
:10D8180005281FB50ED80C4B53F820300093CDE9DE
:10D8280001120A4B01220021022002F069FE05B014
:10D838005DF804FBCDE90012054B0122002102200E
:10D8480002F05EFEF3E700BF901B0108271B0108EA
:10D85800461B010807B5054BCDE90001012200214F
:10D86800022002F04DFE03B05DF804FB621B0108C4
:10D8780010B5102204460021F13000F05FFE0021AF
:10D88800C4F814112046F022BDE8104000F056BE3E
:10D8980002460846102100F0A5B92DE9F0430446D8
:10D8A800D0F8140185B00E46154604F2011988B364
:10D8B800C0F110089045474628BF1746BAB24844F9
:10D8C80000F028FED4F814313B440F2BC4F814316F
:10D8D8002DD9A8452BD204F1F00304F5807113F873
:10D8E800012F187C8B4282EA00021A70F7D104F1EA
:10D8F800F10810224146684600F00CFE22466946AF
:10D90800684600F0E9F910226946404600F002FE38
:10D918003E44ED1B04F5807804F1F107102D09D879
:10D92800AAB23146484600F0F5FDC4F8145105B0D6
:10D93800BDE8F08304F1F003711E13F8012F11F80C
:10D94800010F434582EA00021A70F6D110223946C7
:10D95800684600F0DFFD22466946684600F0BCF9DB
:10D9680010226946384600F0D5FD1036103DD5E73F
:10D97800F0B589B00C46102200210546684600F033
:10D98800DDFD22466946684600F0A6F99DF900309B
:10D99800002B6A464FF0000143DA137812F8010FA2
:10D9A80001315B0043EAD0130F2902F8013CF4D19E
:10D9B8009DF80F305B0083F08703D4F81401DBB2C5
:10D9C80010288DF80F303BD104F58073694604F5B3
:10D9D800887013F8016F11F8012B984282EA060249
:10D9E8001A70F6D104F1F00304F5807113F8012FD1
:10D9F800187C8B4282EA00021A70F7D110220DEBD4
:10DA0800020004F1F10100F085FD2246294604A830
:10DA180000F062F910220021684600F08FFD09B07D
:10DA2800F0BD137812F8010F01315B0043EAD013FF
:10DA38000F2902F8013CF4D19DF80F305B00BCE7D8
:10DA48009DF90030002B6A464FF0000137DA137851
:10DA580012F8016F01315B0043EAD6130F2902F86F
:10DA6800013CF4D19DF80F305B0083F08703471C1D
:10DA7800DBB28DF80F30102F04EB0003C0F10F0656
:10DA88004FF0800288BF002600F5817083F80121DD
:10DA98000021324620443E4403F072FAC4F814616F
:10DAA80004F58073694604F5887013F8016F11F85E
:10DAB800012B984282EA06021A70F6D192E713788F
:10DAC80012F8016F01315B0043EAD6130F2902F8FF
:10DAD800013CF4D19DF80F305B00C8E70A78037861
:10DAE800534003704A784378534043708A78837868
:10DAF80053408370CA78C3785340C3700A79037956
:10DB0800534003714A794379534043718A79837941
:10DB180053408371CA79C3795340C3710A7A037A2F
:10DB2800534003724A7A437A534043728A7A837A1B
:10DB380053408372CA7AC37A5340C3720A7B037B09
:10DB4800534003734A7B437B534043738A7B837BF5
:10DB580053408373CA7BC37B5340C373704710B56C
:10DB68000B7814786340037054784B7863404370A3
:10DB780094788B7863408370D478CB786340C37093
:10DB880014790B796340037154794B79634043717D
:10DB980094798B7963408371D479CB796340C3716D
:10DBA800147A0B7A63400372547A4B7A6340437257
:10DBB8008B7A947A63408372D47ACB7A6340C37247
:10DBC800147B0B7B63400373547B4B7B6340437331
:10DBD800947B8B7B63408373CB7BD27B5340C37333
:10DBE80010BD0000A1F11003DBB2102B2DE9F047A6
:10DBF80004D8374C24FA03F3DB0705D4002382F852
:10DC0800F030FF20BDE8F087531E4418A0424ED1E3
:10DC180001F11C039B005FFA83F9C3F30313013B73
:10DC28002C4D82F8F03001240B46D618B3FBF1F0E6
:10DC380001FB103010F0FF0016F804AC16F803ECE6
:10DC480016F802CC16F8017C36D115F80E8015F8B6
:10DC58000CE015F807C015F80A70E00900EB400061
:10DC680084EA080800EBC0006400C0B2E4B2444093
:10DC7800C246581AC0B212F800808AEA080A02F8A6
:10DC880003A01044043390F801808EEA080E86F849
:10DC980001E090F802E08CEA0E0C86F802C0C07829
:10DCA800DBB247409945F770BFD80020AAE710F8C3
:10DCB800015B03F8015FA9E71829DAD9102801BF29
:10DCC80015F80AA015F80EE015F80CC0EF5DD0E7BE
:10DCD80001010100A81D01082DE9F04FA3B092F839
:10DCE800F0301D911B920193002B00F053810146E7
:10DCF8001EA8FFF734FF1B9BA74CA84DA84E103356
:10DD08000293002303939DF87C0004909DF88600FD
:10DD18000590205C06909DF87B000790205C089099
:10DD280004989DF881C0205C099014F80C000A90B2
:10DD38009DF880000B909DF885009DF878809DF8EF
:10DD48007DE09DF882A09DF887900C909DF87A0060
:10DD5800029B1C9314F80A2014F8093014F80810D0
:10DD680014F80E700D90205C0E909DF87F000F90B7
:10DD7800205C10900B98205C11900C98205C1290FD
:10DD88009DF8840013909DF8790014909DF87E000A
:10DD98001590205C16909DF883001790205C1890D1
:10DDA8001398205C19901498205C1A9003980130FD
:10DDB80003900298DDF804B0103002909DF80C0032
:10DDC800834536D88DF878108DF87A2009990E9AFF
:10DDD8008DF87C108DF882201199069A8DF88010A4
:10DDE8008DF87E201999169A8DF884108DF8862062
:10DDF8000A99189A8DF87D108DF887201299109A33
:10DE08008DF87B301B9B8DF881108DF883201A9933
:10DE1800089A1D988DF885108DF87F201EA903EBB0
:10DE28000B128DF87970FFF79AFE002023B0BDE839
:10DE3800F08F15F808B082EA03008BEA000016F8A4
:10DE48000EB080EA0B008DF8780015F80E004B40F4
:10DE5800434016F80A0043408DF8793081EA0703F9
:10DE680015F80A10594016F80930594016F80830C4
:10DE78008DF87A107A40534015F8092053408DF8F0
:10DE88007B30089A069B5340049AAA5C534016F8C4
:10DE98000C2053408DF87C30DDE908325A4015F8E3
:10DEA8000C305340059AB25C53408DF87D30DDE963
:10DEB80009325A40059BEB5C5340079AB25C5340C9
:10DEC8008DF87E30069B0A9A5340049AB25C5A40F9
:10DED800079BEB5C5A408DF87F200E9B109A5340AD
:10DEE8000B9AAA5C53400C9AB25C53408DF8803070
:10DEF800DDE910325A400C9BEB5C53400D9AB25C42
:10DF080053408DF88130DDE911325A400D9BEB5CAE
:10DF180053400F9AB25C53408DF88230129A0E9B90
:10DF280053400B9AB25C5A400F9BEB5C1C995A40C9
:10DF38008DF88320169B189A5340139AAA5C534075
:10DF4800149AB25C53408DF88430DDE918325A4097
:10DF5800149BEB5C5340159AB25C53408DF88530A6
:10DF6800DDE919325A40159BEB5C5340179AB25CB5
:10DF780053408DF886301A9A169B5340139AB25C18
:10DF88005340179AAA5C1EA853408DF88730FFF7B4
:10DF9800A5FDB8E6FF2049E7A81D0108A81B010850
:10DFA800A81C010808B538B1044A05491060D822F0
:10DFB80000F0B0FA002008BD0220FCE7F81D0020A0
:10DFC800D82201080A4B1A6870B5002302F1180517
:10DFD80003EB03142E5D864204D1183422440A60F0
:10DFE800002070BD01330B2BF2D10320F9E700BFED
:10DFF800F81D00202DE9F041CCB00646DDF8488137
:10E0080017461C460D4631B3B8F1000F23D006A8B9
:10E01800FFF72EFC204601A9FFF7D4FF0446B0B94C
:10E02800019906A80131FFF733FC26B110223146C9
:10E0380006A8FFF732FC3A46294606A8FFF72DFC4A
:10E0480006A902A8FFF794FC029BC8F800302046F6
:10E058004CB0BDE8F0810224F9E7000030B595B076
:10E0680013A90446FFF7AEFF002830D11B490C2343
:10E0780003FB00F2555CA5422BD1139B187C109032
:10E08800D87B0F90987B0E90587B0D90187B0C9046
:10E09800D87A0B90987A0A90587A0990187A08904A
:10E0A800D87907909879069058790590187904904E
:10E0B800D8780390987802900A445B780193936823
:10E0C80000930022064B1146022002F019FA15B0FF
:10E0D80030BD01300B28CBD1F9E700BF2020010863
:10E0E800A81E01080B2B10B402D810BCFFF782BF82
:10E0F800032010BC704730B50D4685B01446014664
:10E1080068B103AA002000922A460390FFF772FF25
:10E1180018B90398001B18BF012005B030BD0220B4
:10E12800FBE72DE9F0430D46BFB0144699468046FB
:10E1380020B31BB311F00F0122D1F02201A800F087
:10E14800FDF920466946FFF73DFF044648B90098A7
:10E1580001AA10210130FFF745FD2E46AF1BFFB283
:10E168001EB920463FB0BDE8F08301AA09EB0701BC
:10E1780008EB0700FFF7B0FD103EEFE70224F0E7D9
:10E188000524EEE7F0B5184E3468024685B0084617
:10E19800002304F1180103EB03154F5D97421ED1CC
:10E1A8000D2A05F1190513D10023CDE90033CDE976
:10E1B80002330C2210216B46FFF7B3FF0446306888
:10E1C80010226946284400F0A5F9204605B0F0BDA4
:10E1D80001461022601900F09DF90024F5E701338B
:10E1E8000B2BD8D10324F0E7F81D002009B1FFF765
:10E1F800C9BF022070471FB51446A0B10C2A01D12F
:10E208000B2912D10023CDE90033CDE902330A46A8
:10E218006B461021FFF785FF18B969462046FFF7BE
:10E22800B1FF04B010BD0220FBE70320F9E7F8B501
:10E238001E46DDE907479DF818505BB354B34FB34A
:10E24800212D29D819462A46204600F063F90122D3
:10E25800631C691EB018FFF764FFF8B9E37ADB099D
:10E268003B70EBB96319204613F8012C13F8021C14
:10E27800120642EA014213F8041C0A4313F8031C6D
:10E28800012342EA0122291FFFF735FF003818BF92
:10E298000120F8BD0220FCE70520FAE70720F8E78F
:10E2A8000420F6E710B5044628B1044B5B6998478B
:10E2B8002060002010BD0220FCE700BF38210108C3
:10E2C80008B5014630B1044B0822186800F022F95D
:10E2D800002008BD0220FCE7F81D002008B530B179
:10E2E800044B0822196800F015F9002008BD022027
:10E2F800FCE700BFF81D00207FB5124E002304463E
:10E3080002A801930D46FFF7E9FF33685B690193A3
:10E318006CB102AA082312F8011B41B9013B13F0A2
:10E32800FF03F8D102A8A04702A8FFF7C9FF35B13B
:10E33800019B23B901A8A8473368019A5A610020B4
:10E3480004B070BDF81D002008B5014638B1054B72
:10E3580018680822104400F0DDF8002008BD0220EB
:10E36800FCE700BFF81D002008B538B1044B196858
:10E378000822114400F0CEF8002008BD0220FCE776
:10E38800F81D0020034B1B6802280CBF1961596156
:10E3980000207047F81D002041B1054B1B6802287A
:10E3A8000CBF1B695B690B60002070470220704737
:10E3B800F81D002030B58FB0002405460CA809943C
:10E3C800FFF78CFF9DF8373007939DF8363006939A
:10E3D8009DF8353005939DF8343004939DF833301B
:10E3E80003939DF8323002939DF8313001939DF8E4
:10E3F80030300093224621461E4B022002F080F85E
:10E408000AA8FFF7B1FF9DF82F3007939DF82E302B
:10E4180006939DF82D3005939DF82C3004939DF8B4
:10E428002B3003939DF82A3002939DF829300193ED
:10E438009DF82830009322460F4B2146022002F017
:10E448005FF809A92846FFF7A7FF9DF82430039332
:10E458009DF8253002939DF8263001939DF82730CA
:10E4680000932246054B2146022002F049F80FB0DE
:10E4780030BD00BF041F0108421F0108801F0108AA
:10E4880008B50020FFF7EAFD0120FFF7E7FD0920A6
:10E49800FFF7E4FD0820FFF7E1FD0020FFF78AFF02
:10E4A800002008BD10B504460B20FFF7D7FD0C204F
:10E4B800FFF7D4FD0920FFF7D1FD0820FFF7CEFDB7
:10E4C8000A20FFF7CBFD2046FFF774FF002010BDA0
:10E4D800014B1860704700BF4C0100200B4A30B553
:10E4E80014680B4D43F2390305FB04331360091A12
:10E4F8006FF00042B3FBF2F2C2EBC27201319B1A19
:10E5080093FBF1F201FB1233184430BD4C0100209B
:10E518006D4EC64101380A44914200D1704711F846
:10E52800013B00F8013FF7E710440A44914200D14B
:10E53800704711F8013B00F8013DF7E702F020BDF4
:10E5480030B530B10A4D01444FF0FF33814201D15B
:10E55800D84330BD10F8012B5340082243F3000480
:10E56800013A2C4092B284EA5303002AF6D1EDE72F
:10E578002083B8ED01207047054B4FF400529A6292
:10E58800044B1B6813B15B6803B11847704700BFA1
:10E5980000040048FC1E0020054B4FF480529A628C
:10E5A800044B1B6813B1DB6803B11847704700BF01
:10E5B80000040048FC1E002001207047012070471D
:10E5C80001F048B901F036B910B501F019FE0E2175
:10E5D800044640F61F1001F02DF92046012101F0F4
:10E5E800F9FDBDE8104001F0D7BA000070B50C4E37
:10E5F80001EB40030D46B3654FF6FF710023044657
:10E608001A46084601F05EFB96F85600002101F014
:10E61800E1FD29462046BDE8704001F095BA00BFEB
:10E62800181F002010B5044601F0AAFE01281CD1CD
:10E6380001F0AEFE34B11248214602F017FB104833
:10E6480002F0DAFA0F4C104B00214FF48052A1650A
:10E658009A6194F8560001F0BDFD63786BB16FF0D4
:10E668007F40BDE8104001F053BA002340F2622118
:10E678001A46084601F026FBDCE7A0688001F0E7AF
:10E68800001F0020181F002000040048002001F08F
:10E69800BFB9000008B501F0C7F80438C0B20328B4
:10E6A80096BF024B0020185C08BD00BF342101084A
:10E6B80008B501F0BAFD033008BD01F049B901F011
:10E6C80009B908B501F000FD00B208BD38B50D461E
:10E6D800144601F05DFB284601F092FD0E21054627
:10E6E80040F61F1001F0A6F828460121074D01F059
:10E6F80071FD01F051FA4FF47A716143284602F036
:10E70800B5FA2846BDE8384002F076BA741F0020F2
:10E7180001F03EBB08B5084B002193F8560001F004
:10E7280059FD00234FF4C0711A46084601F0CAFA91
:10E73800BDE8084001F024BA181F002010B50446AF
:10E7480001F01EFE01281CD101F022FE34B112484E
:10E75800214602F08BFA104802F04EFA0F4C104B8B
:10E7680000214FF48052A1659A6194F8560001F097
:10E7780031FD63786BB16FF07F40BDE8104001F068
:10E788007DB9002340F262211A46084601F09AFA40
:10E79800DCE7A0688001F0E7001F0020181F0020B8
:10E7A8000004004808B54FF0040001F017F9BDE86F
:10E7B80008400220F4F79CB908B500231A46194608
:10E7C800184601F07FFABDE8084001F06DB9000075
:10E7D8001D4B73B51D4D186000241D486C70C5E9AC
:10E7E8000144AC6501F098FAAC8101F003FA2146C6
:10E7F800204601F04BFC21460422012001F0FCFADE
:10E80800144E154D4FF6FF7123462246084601F077
:10E8180059FAFFF7C7FF2246104B00944FF0FF311B
:10E82800304602F03DF90E4B009422464FF0FF317E
:10E83800284602F035F9304602F090F9284602B031
:10E84800BDE8704002F08AB9FC1E0020181F0020A5
:10E8580021F80008741F0020001F002081E500082F
:10E86800A1E500080128084805D1084BC1771970AF
:10E878000E3001F0A7BB437D012B03D1034B8175FB
:10E888001970F5E7704700BF181F002050010020DD
:10E898000D4B10B5044618735873012000F016F894
:10E8A8005CB134214FF4E86000F0C4FF4421BDE8B6
:10E8B800104040F2417000F0BDBF14214FF4E860F1
:10E8C80000F0B8FF2421F2E7181F002038B5114CDA
:10E8D8000546207001F061FD052D04D8DFE805F03C
:10E8E800090B03171709032001F070FA002363735B
:10E8F80038BD0020F8E7012001F068FA207B637B2F
:10E908008342F5D06073BDE83840FFF7C1BF0220ED
:10E91800EAE700BF181F00202DE9F0431E4687B024
:10E9280000230546CDE901330C46174601F027FDC3
:10E93800032D61D8DFE815F07B00C3000E01040049
:10E94800A27C082A04D94FF0FF3007B0BDE8F08355
:10E95800A16801A801F0DCFE21680029F3D042F289
:10E9680010729142E37C864D51D80322AA7385F830
:10E978003820E96385F844304FF002086368A17DC8
:10E98800DB002B820423AB74A37CDB00EB7402292D
:10E998004FF000032B75637D02D0227D022A42D1FD
:10E9A80003F10F02D2B2012A01D9012BCBD1754B49
:10E9B800754A196803944FF0010903A88DF814905B
:10E9C80001F0DAFC0028BED1287685F81790687522
:10E9D800FFF75CFE4046FFF779FF6C4801F086FAC6
:10E9E8006B4801F0EFFA01A800F084FF208A00F0DC
:10E9F80055FFA08900F09AFF384601F001FC604CF1
:10EA080084F8560001F0C0FC666000209DE74FF0D6
:10EA18000008E963890885F80E8085F8388085F84C
:10EA280044302964AAE7EB7529766A75D0E723682C
:10EA3800002B88D0A27C082A85D8514DA16801A84E
:10EA480001F066FE002385F838302268EA63E27C2C
:10EA580085F84420A269AB732A646268A17DD2005C
:10EA68002A820422AA74A27C2B75D2000229637D13
:10EA7800EA7402D0227D022A1DD103F10F02D2B21C
:10EA8800012A02D9012B7FF45EAF3E4B3E4A19683A
:10EA980003944FF0010803A88DF8148001F06CFC72
:10EAA80000287FF450AF287685F817806875FFF73F
:10EAB800EDFD00208FE7EB7529766A75F7E7304D95
:10EAC800012185F83810227885F85020637885F878
:10EAD8005130A37885F85230E3788B4202D0022B6C
:10EAE80003D03BB985F8533004E00B3A012A29D802
:10EAF80085F853104FF0010885F80E80A388AB8382
:10EB0800A379AB77E37985F82030237A85F821302B
:10EB1800FFF7BCFD4046FFF7D9FE1C4801F0E6F9B7
:10EB28001B4801F04FFA95F85130062B40F6890042
:10EB38000AD100F08FFE00F0FB0140F6890000F0DA
:10EB480079FE59E70023CDE700F084FE40F0040188
:10EB5800C9B2F2E72368013BB3F57A7FBFF4F3AE9D
:10EB68000320FFF7B3FE0648022380F838302368F5
:10EB78008364162380F84C30383001F0B7F93BE74E
:10EB8800181F0020FC1E0020741F0020501F0020AA
:10EB9800261F00202DE9F041002686B01F461446A6
:10EBA800CDE9016680460D4601F0E9FBB442764C9A
:10EBB80016BF0123334637466370B8F1000F06D0FD
:10EBC800B8F1010F7CD0002006B0BDE8F081AB6839
:10EBD800002B00F0D680EB68002B00F0D280AA7FD3
:10EBE800082A00F2CE80296901A801F091FD286861
:10EBF800003818BF012000F0D9FF84F83880AB68CE
:10EC0800E36395F8203084F84430686801F05AFBD3
:10EC180084F80E8084F84500EB68DB002382EB7FE4
:10EC2800A374AB7FDB00E37495F82130237595F866
:10EC38002230002B3ED12A7D95F82410A275022996
:10EC480095F8232001D0022B36D102F10F03DBB255
:10EC5800012B02D9012A40F0948000238DF814304A
:10EC68004A4B4B4A1968049503A801F085FB002814
:10EC780040F0878001232076E3756075FFF706FD75
:10EC88000020FFF723FE434801F030F9424801F025
:10EC980099F901A800F02EFEA88B00F0FFFD288B43
:10ECA80000F044FE4FF4FA53AA687B43B3FBF2F337
:10ECB800A36088E7FF22BFE7E27521766375DDE789
:10ECC8002B8E002B5DD095F83230A86A012B0CBF33
:10ECD80095F814804FF0FF08003818BF012000F0A5
:10ECE80065FFF8B200F06EFF012184F8381095F83E
:10ECF8002C2084F8502095F82D3084F8513095F860
:10ED08002E3084F8523095F82F308B4202D0022BE7
:10ED180003D03BB984F8533004E00B3A012A28D8D1
:10ED280084F853102B8EA38395F83230A377AB8EDB
:10ED380023840126A67384F81F80FFF7A7FC3046BA
:10ED4800FFF7C4FD134801F0D1F8134801F03AF970
:10ED580094F82130B34240F236700CD100F07AFDBD
:10ED680000F0FB0140F2367000F064FD4FF6FF73CF
:10ED78009EE70023CEE700F06DFD40F00401C9B224
:10ED8800F0E74FF0FF301FE7181F0020FC1E00209F
:10ED9800001F0020501F0020261F00202DE9F04FE3
:10EDA80085B082460E9DBDF840B09DF844709DF830
:10EDB8004890019288461E4601F0E1FABAF1010F27
:10EDC800524C54D0BAF1040F00F09180BAF1000F00
:10EDD8003AD10B22304684F8442084F838A0E56301
:10EDE80001F070FA019B23644FEACB03B9F1000FDD
:10EDF800238241F60403638214BFF2230123E375DF
:10EE080087F001070123237684F8450084F80EA0D3
:10EE180084F814A06775FFF739FC5046FFF756FDD4
:10EE280004F1380001F062F804F10E0001F0CAF8AC
:10EE3800374A1068516802AB03C302A800F05AFDB4
:10EE480040F2FF1000F02AFD404601F0D9F90E21EA
:10EE580084F8560040F61F1000F0ECFC94F85600B9
:10EE680001F092FA169B636005B0BDE8F08F29495E
:10EE780084F838A0EAB2895D84F8502076BB0B3D4F
:10EE8800012D8CBF00250125053A012A04D8BBF1C4
:10EE98000C0F38BF4FF00C0B1F4B9DF83C201B7814
:10EEA80084F85350E37701259DF8543084F85110C5
:10EEB80084F8522084F82130A573A4F81CB0A777F1
:10EEC80084F82090FFF7E2FB2846FFF7FFFC134881
:10EED80001F00CF8124801F075F8B5E7012E04D1DD
:10EEE800A5F10C035D425D41CEE70025CCE7504615
:10EEF800FFF7ECFC022384F8383004F138001623BD
:10EF0800A56484F84C3000F0F1FF9DE7181F00203D
:10EF18004C1101080221010850010020501F002057
:10EF2800261F00202DE9F04F87B0DFF8B4B29DF816
:10EF380064A09DF84C90029314469DF854309DF8B7
:10EF48005020BDF84880039205468BF801A0BDF813
:10EF5800446001930F4601F012FABAF1000F18BF8E
:10EF68004FF00008DFF87CA2039AB9F1000F08BF40
:10EF7800FF22012D8AF8002000F0C880052D48D016
:10EF8800002D40F0C080284600F010FE0B223846C5
:10EF98008BF844208BF83850CBF83C4001F092F9BC
:10EFA800019B8BF8450041F60402002BABF81220B8
:10EFB8009AF800208BF8162014BFF22201228BF851
:10EFC8001720F600012289F001098BF818208BF828
:10EFD8000E50ABF810608BF814508BF81590FFF7B3
:10EFE80055FB2846FFF772FC0BF1380000F07EFF56
:10EFF8000BF10E0000F0E6FF7B490868496804AA97
:10F0080003C204A800F076FC40F2FF1000F046FCB2
:10F0180071E0012000F0CAFD09224FF000098BF8C9
:10F02800442038464FF44872CBF840208BF838908B
:10F03800CBF83C4001F046F94FF48052ABF812206F
:10F048009AF800208BF845008BF8162028460122F4
:10F05800F6008BF817208BF80E90ABF81060ABF821
:10F0680014908BF81890FFF731FC0BF1380000F082
:10F078003DFF0BF10E0000F0A5FF5B498868C968E9
:10F0880004AA03C204A800F035FC40F2FF1000F007
:10F0980005FC40F6B80000F0DDFB00F0EF0140F69B
:10F0A800B80000F0C7FB042140F6B90000F0C2FB2D
:10F0B80040F69B0000F0CEFB00F0E30141F00801B0
:10F0C80040F69B0000F0B6FB40F2D16000F0C2FBB6
:10F0D80040F01801C9B240F2D16000F0ABFB40F239
:10F0E800AC6000F0B7FB00F08F0141F0500140F236
:10F0F800AC6000F09FFB4FF4FA5202FB08F2B2FB3F
:10F10800F4F2CBF8082007B0BDE8F08F002000F03B
:10F118004DFD36498BF83850E2B2C95D8BF8502066
:10F12800002F4DD10B3C012C8CBF00240124053A43
:10F13800012A02D80C2E38BF0C26029B9AF8002010
:10F148008BF852308BF85340019B8BF81F20012419
:10F158009DF860208BF821208BF851108BF8203017
:10F168008BF80E40ABF81C608BF81E90FFF78EFAF8
:10F178002046FFF7ABFB1E4800F0B8FE1D4800F024
:10F1880021FF5FFA88F000F01DFD40F6A30000F0B3
:10F1980061FB00EA040140F6A30000F04BFB9BF87A
:10F1A8002120A24240F2367013D100F053FB00F048
:10F1B800FB0140F2367000F03DFB4FF6FF72A0E70E
:10F1C800012F04D1A4F10C035C425C41AFE7002499
:10F1D800ADE700F03FFB40F00401C9B2E9E700BF2A
:10F1E800181F0020500100204C11010802210108BD
:10F1F800501F0020261F0020F0B58BB00D46044696
:10F2080017461E46FFF742FA0020FFF75FFB20462D
:10F2180000F0BEFD00240123CDE9084303234FF489
:10F22800167229462046CDE90644CDE90444CDE9C5
:10F238000244CDE900532346FFF774FE2046FFF74A
:10F248007DFAFFF735FAF3F753FC01F043FC044667
:10F25800204601F049FCB04205D30124FFF716FA15
:10F2680020460BB0F0BD00F02FFF00B28742EFDA66
:10F278000024F3E7F7B500230C4640F201211A46B3
:10F288000646084600F01EFD644B654D4FF40052DB
:10F298009A6195F85600012100F09CFF2B78012B0C
:10F2A80040F6890013D195F85130062B0FD100F0A4
:10F2B800D1FA00F0FB0140F6890000F0BBFA2B7888
:10F2C800042B6CD8DFE803F0524B527F090000F0A2
:10F2D800C1FA40F00401C9B2EDE7524A731E104664
:10F2E800C6F101074FF0000CF9188C426FDC0022C0
:10F2F800E7001346BA4271D19A0142EAC3125B0190
:10F3080083F020031343661C0355F6B202234648D4
:10F31800AB73AE7600F056FE0021F12000F08AFAB9
:10F328000021F02000F086FAAB6C642B70D17021BC
:10F33800F32000F07FFA1D21F22000F07BFAE100B3
:10F348008C1CF420090A00F075FA04F0FE01F5207F
:10F3580000F070FA33486FF07F4231461DE0EC77D9
:10F36800314800F02FFE0022214615E001F008F890
:10F378000128074625D121460DF10702304601F044
:10F3880004F80446A0B99DF807302748AB7500F08B
:10F3980019FE9DF807102246304600F065FB6968A3
:10F3A800224801F063FC214801F026FC002006E019
:10F3B8001F4B3A460021022001F0A2F8032003B0B7
:10F3C800F0BDAC75CCE70223AB73AC76C8E713F895
:10F3D800011FC943197002F801CB85E7D1106FEA04
:10F3E800020C715C0CF0070C013241FA0CF101F0CF
:10F3F80001014FEAE20C4B40D14310F80CE001F058
:10F40800070103FA01F141EA0E0100F80C1071E757
:10F41800E121F32000F00EFA04218DE700040048F2
:10F42800181F0020FC1D0020261F0020741F00202C
:10F43800A4200108F0B5BDF814409DF818709DF897
:10F448001CE09DF8205040B1012814D0012200236F
:10F4580098180138B0FBF2F0F0BD87F00107E3001F
:10F4680003EBC70318330EEB450503EBC5034FF455
:10F478007A714B43ECE7501F012803F1040302D8CB
:10F488000C2C38BF0C24D1B9A2F10B0CBCF1010F24
:10F498008CBF4FF0000C4FF0010C2801002F00EB3F
:10F4A800CE0014BF00251425A0EB8200062A4FEADF
:10F4B80082062844A2F102070DD8354610E001293A
:10F4C80006D1A2F10C00D0F1000C4CEB000CE4E7E3
:10F4D8004FF0000CE1E70830BCF1000FEDD0BD00A3
:10F4E8000028ACBF2E182E1C701E90FBF5F003FBF5
:10F4F8000044094B062A5A5C8CBF0C340E340A2A85
:10F5080009D8A30001334FF47A71BB404B43034938
:10F5180051F822209CE7FFDE02210108082101089A
:10F5280008B5094B012193F8560000F053FE4FF43B
:10F53800D7602D2100F07EF900F033FBBDE80840CC
:10F54800024800F07BBA00BF181F0020FFFF0F0021
:10F5580073B5A44CB4F854300025202B8DF8035013
:10F56800019500F01B8114D8082B0DD87BB1013B05
:10F57800072B0CD8DFE813F042005B000B00CD002E
:10F588000B000B000B00FD00102B00F0008102B0F7
:10F5980070BDB3F5807F00F0988011D8402B00F043
:10F5A8001081802BF3D1284600F032FA8E4B1B686D
:10F5B800002BECD09B69002BE9D028469847E6E75A
:10F5C800B3F5007FE3D1894B01222946022000F0E0
:10F5D80097FF00F029F9042840F08580844B85487E
:10F5E8004FF400529A6201F0B9FA284600F010FA76
:10F5F8007D4B1B68002BCAD05B6814E07C4B7D48B0
:10F608004FF400529A6201F0A9FA002000F000FAC3
:10F6180000F0B8FE012801D100F0BDFE724B1B6856
:10F62800002BB4D01B68002BB1D09847AFE7704BC4
:10F6380071484FF480529A6201F090FA657895B952
:10F64800284600F0E5F9294640F6021000F0F2F8E5
:10F6580040F6441000F0FEF840F00201C9B240F64E
:10F66800441000F0E7F8FF220DF1030163485E4DF6
:10F6780000F05AFD624800F071FD2B68002B86D01F
:10F688009E68002E83D094F82430012B08D194F979
:10F69800313094F930209DF803105848B04776E788
:10F6A800E06B01A900F022FE019B9DF8031053486E
:10F6B8004FF47A7203F5FA7393FBF2F32A685BB29C
:10F6C800956894F92920A84761E7284600F0A0F931
:10F6D800454B1B68002B3FF45AAF9B69002B3FF446
:10F6E80056AF01206AE700F09FF805287FF44FAF76
:10F6F8003F4B41484FF480529A6201F02FFA284656
:10F7080000F086F9384B1B68002B3FF440AFDB68EC
:10F7180089E700213B4B0122022000F0F1FEA16D98
:10F7280000293FF434AFC1F3074140F6031000F05D
:10F7380081F894F8591040F6041000F07BF894F81A
:10F74800581040F6051000F075F840F6021000F069
:10F7580081F840F00101C9B240F6021000F06AF8E1
:10F76800002340F262211A460846A36500F0AAFA6F
:10F778000DE7254B01220021022000F0C1FE00F018
:10F78800FFFD01287FF403AF00F006FEFFE61F4BE4
:10F7980001220021022000F0B3FEF8E6164801F02D
:10F7A800DDF9607808B900F033F90F4B1B68002BBE
:10F7B8003FF4EDAEDB68002B3FF4E9AE9847144BFD
:10F7C800E6E7144B01222946022000F099FE6078F2
:10F7D80008B900F01DF9044B1B68002B3FF4D7AEA5
:10F7E8001B6920E7181F0020FC1E0020B920010813
:10F7F80000040048741F0020001F0020FC1D00208A
:10F808003C1F0020CD200108D6200108E020010877
:10F81800E9200108F2200108024BA3F85400FFF781
:10F8280097BE00BF181F0020014B1878704700BF13
:10F83800921F002007B501238DF807100DF107026C
:10F8480001460348F7F706FA03B05DF804FB00BF6A
:10F858005C03002007B5012301460DF107020448A7
:10F86800F7F731FA9DF8070003B05DF804FB00BF15
:10F878005C03002010B50446F4F7A8FE01280CD15B
:10F8880040F62310FFF7E6FF00F0F901214340F6A8
:10F898002310BDE81040FFF7CDBF10BD10B50C4BCD
:10F8A8001B7804469BB94FF4D760FFF7D3FFC4F326
:10F8B800002100F0FE0001434FF4D760FFF7BAFFC4
:10F8C800E1B240F2B960BDE81040FFF7B3BF10BD28
:10F8D800931F002010B51346EFF3108472B60A4642
:10F8E80001460348F7F7B6F984F3108810BD00BF46
:10F8F8005C03002008B5014608224FF4D860FFF7E2
:10F90800E9FF002008BD000007B5074B1B7840BA87
:10F91800ADF804002BB9022201A940F2BC60FFF740
:10F92800D9FF03B05DF804FB931F002007B5074B10
:10F938001B7840BAADF804002BB9022201A940F2A5
:10F94800BE60FFF7C7FF03B05DF804FB931F0020FC
:10F9580010B51346EFF3108472B60A460146034801
:10F96800F7F7B1F984F3108810BD00BF5C030020DD
:10F9780010B51346EFF3108472B60A4601460348E1
:10F98800F7F793FA84F3108810BD00BF5C030020DA
:10F998000A4601460020FFF7EBBF000010B51346EA
:10F9A800EFF3108472B60A4601460348F7F7B0FA37
:10F9B80084F3108810BD00BF5C03002010B5134607
:10F9C800EFF3108472B60A4601460348F7F7B6F912
:10F9D80084F3108810BD00BF5C03002013B50446F3
:10F9E8000020F4F7CDFD0220FFF744FF04F00704E0
:10F9F80001220DF1070184208DF80740FFF7DEFF93
:10FA0800024B00221A7002B010BD00BF921F0020E6
:10FA180007B501228DF807000DF107018020FFF7D7
:10FA2800CDFF9DF80730002B034B0CBF01220222AB
:10FA38001A7003B05DF804FB921F002007B5094B4C
:10FA48008DF8060004221A70030C8DF80430032286
:10FA5800030A01A983208DF80530FFF7AFFF03B033
:10FA68005DF804FB921F002010B51446FFF790FFC5
:10FA78002046BDE81040FFF7E1BF000007B5094B7D
:10FA88008DF8060005221A70030C8DF80430032245
:10FA9800030A01A982208DF80530FFF78FFF03B014
:10FAA8005DF804FB921F002073B5002640F6E200C3
:10FAB8000196FFF7CFFE00F0FE01054640F6E20092
:10FAC800FFF7B8FE40F6E500FFF7C4FE00F07F013F
:10FAD800044640F6E500FFF7ADFE6FF07F40FFF704
:10FAE800CDFF04220DEB020140F61900FFF730FFAD
:10FAF8003046FFF78DFF294640F6E200FFF79AFEF1
:10FB0800214640F6E500FFF795FE019802B070BD6A
:10FB180013B50C4B04460522972140F6AC001A7029
:10FB2800FFF788FE230C8DF804300322230A01A96D
:10FB380082208DF805308DF80640FFF73FFF02B0B0
:10FB480010BD00BF921F002007B5030C8DF80030D0
:10FB5800030A8DF801300B0C49BA8DF80200ADF894
:10FB680004100622694694208DF80330FFF726FF1B
:10FB7800024B06221A7003B05DF804FB921F0020A6
:10FB8800002208B51146C520FFF718FF014B0722D0
:10FB98001A7008BD921F002000221146D120FFF7DD
:10FBA8000DBF00221146D220FFF708BF07B501227A
:10FBB8008DF807000DF107019F20FFF7FFFE03B046
:10FBC8005DF804FB07B501228DF807000DF1070168
:10FBD800A020FFF7F3FE9DF807103F2907D901F091
:10FBE800F8010131C9B240F20670FFF723FE03B0F5
:10FBF8005DF804FB07B5F4F7E9FC431E5842584189
:10FC08008DF8070001220DF107019620FFF7D6FEB7
:10FC180003B05DF804FB07B500F07F008DF807001E
:10FC280001220DF107018920FFF7C8FE03B05DF836
:10FC380004FB0000154B984207B51BD8144B98429B
:10FC48001BD8144B98421BD8134B98421BD8134B04
:10FC5800984295BF29226B222B236F238DF804200D
:10FC680001A9022298208DF80530FFF7A7FE03B0FE
:10FC78005DF804FBE122E923F0E7D722DB23EDE777
:10FC8800C122C523EAE775228123E7E700E9A43505
:10FC980080F8A9328044E52D000B6B1B40FC5419F9
:10FCA80007B58DF8062004228DF804008DF805109C
:10FCB80095200DEB02018DF80730FFF77FFE03B0AA
:10FCC8005DF804FB07B552BAADF8042040BA082223
:10FCD80049BAADF80000ADF802105BBA69461046A3
:10FCE800ADF80630FFF76AFE03B05DF804FB07B510
:10FCF8000B0C042200F0070049BA8DF80400ADF897
:10FD0800061097200DEB02018DF80530FFF756FE1F
:10FD180003B05DF804FB000010B508B1194B18607A
:10FD2800F2F7E6FD0220FFF7A5FD0024164B20465A
:10FD38001C70FFF76DFEF4F747FC012817D14FF44C
:10FD48002071FFF7D4FF40F611102146FFF772FD2E
:10FD58004FF07F00FFF75FFF0E2140F61F10FFF7FF
:10FD680069FDF4F7D9FB094B01221A7010BD102167
:10FD780040F61110FFF75EFD102140F61210FFF754
:10FD880059FDE9E7941F0020901F0020921F0020D2
:10FD980037B50C4D2B7804461BB9FFF74BFF0123F1
:10FDA8002B700023084A6006E109F1F7ADFE042232
:10FDB80000BA01900DEB02018620FFF7FFFD03B0AA
:10FDC80030BD00BF901F00200048E80107B5094B6F
:10FDD8008DF807000146187018B940F2AC60FFF7BB
:10FDE80029FD01220DF107018A20FFF7E7FD03B085
:10FDF8005DF804FB931F0020012873B50C461646D6
:10FE080037D10020F4F7E4FBA042B8BF44B20E2873
:10FE180005461AD101231A4600210420FFF740FFA6
:10FE28006FF010039C42B8BF1C46182140F6E7004B
:10FE3800FFF700FD022201A98E208DF804408DF8FD
:10FE48000560FFF7BBFD02B070BD01230A28E4B2CC
:10FE58001A464FF0000105D11846FFF721FF033479
:10FE680064B2DDE70720C5F10E05FFF719FF2C4442
:10FE7800F6E740F6D800FFF7EDFC40F01E01C9B2E6
:10FE880040F6D800FFF7D6FC0120F4F7A1FBA0420A
:10FE9800B8BF44B2142805464FF001034FF00002E2
:10FEA8000CD105210320FFF7FBFE023464B26FF08A
:10FEB80008039C42B8BF1C463821B7E7112805D172
:10FEC80003210220FFF7ECFE0534EFE70E2804D1EA
:10FED80002210846FFF7E4FEE9E7C5F11605072108
:10FEE80004202544FFF7DCFE6CB2E0E713B5314A85
:10FEF8000446516810686B4603C32F4B20781B7863
:10FF0800834201D0FFF762FF2378032B27D8DFE86D
:10FF180003F00239283C6268284BB3FBF2F31A0C51
:10FF2800A1688DF800208DF802301A0A237B8DF81D
:10FF38000330637B8DF801208DF80430204A0023BC
:10FF48004806C909F1F7E0FD030C40BA8DF8053001
:10FF5800ADF80600082269468B20FFF72FFD02B096
:10FF680010BD2269154BB3FBF2F31A0C8DF8002073
:10FF78008DF802301A0A237D8DF801208DF80330A0
:10FF88000422E8E7A3690093FAE762680B4BB3FB26
:10FF9800F2F31A0C8DF800208DF802301A0A237B30
:10FFA8008DF80330637B8DF801208DF8043005222D
:10FFB800D1E700BF5C110108931F00200000093D34
:10FFC8000048E8011FB52E4A0446D1689068127CA3
:10FFD80001AB03C31A702B4B20781B78834201D0E6
:10FFE800FFF7F4FE2378032B26D8DFE803F0023866
:08FFF8003302637AF12B21D1E1
:020000040801F1
:100000004FF6FF70FFF784FC48F20500FFF792FC03
:1000100002236288A188ADF8061052BAE188ADF8D3
:1000200004208DF80B30227AA37A8DF80A20ADF8DF
:1000300008108DF80C30092201A98C20FFF7C2FCB2
:1000400004B010BDF22BE4D141F60F50FFF760FC75
:1000500041F22100FFF76EFC0623DAE7237B8DF8DF
:1000600004300122E8E7E389094A5BBAADF80430BD
:10007000237C13708DF80630637C8DF80730638A1B
:10008000ADF808300622D7E75C110108931F002065
:10009000911F002007B502228DF804008DF805108D
:1000A0008F2001A9FFF78EFC03B05DF804FB000070
:1000B00010B51346EFF3108472B60A4601460348A2
:1000C000F6F778FE84F3108810BD00BF5C030020B3
:1000D00007B5012201A91520FFF7EAFF9DF80400EA
:1000E0004042401003B05DF804FB000037B5054600
:1000F0000C46022201A91320FFF7DAFF0A4B1B78F6
:10010000012B0DD1094B1B78012B09D140F2027054
:10011000FFF7A4FB9DF805302870237003B030BDB5
:100120009DF80400F6E700BF931F0020911F0020F8
:10013000F7B50D46064600240DF10701284617467F
:100140008DF80740FFF7D2FF2A78BA4207D89DF80A
:1001500007003146FFF726FC204603B0F0BD012022
:10016000FBE7000013B50322044601A91420FFF7A2
:100170009FFF184B1A7822704AB1012A17D0142217
:100180000021204600F0D2FA0F2323700DE09DF8E5
:10019000043023719DF80530A2605B425B10A371AF
:1001A0009DF806305B425B10637102B010BD9DF894
:1001B00004305B425B1023739DF9053002339B10C2
:1001C00063739DF806305B425B10A373024B1B68A0
:1001D0002361EAE7931F00208C1F0020012908B546
:1001E000034608460ED1012B07D10420FFF746FB3A
:1001F0000220BDE80840F4F7C7B9022B14BF084637
:100200000320F6E70120F4E738B50446F4F7DEF9F9
:1002100050B1022814BF012502252846022221469A
:10022000FFF7EEFD284638BD0F2CCCBF0225012577
:10023000F3E70A2070470000014B01201B681847B4
:10024000941F0020014B02201B681847941F0020B8
:10025000014B40201B681847941F002011B1012951
:1002600004D07047044B1B6880201847024B4FF4A2
:1002700080701B68F9E700BF941F0020024B4FF409
:1002800000701B68184700BF941F0020014B2020FE
:100290001B681847941F0020014B04201B68184757
:1002A000941F0020014B08201B681847941F002052
:1002B000014B10201B681847941F0020024B4FF47D
:1002C00080401B68184700BF941F002068B1084A8F
:1002D000002352F83310814203D902EBC302107994
:1002E00070470133162BF4D1FEE71F20704700BF83
:1002F000C421010873B51D4B0193044640F6070065
:100300000D46FFF7ABFAC0F3C10308336B4413F893
:10031000042C00F00703013302FA03F3144AB2FB82
:10032000F3F2B2FBF4F007281ED8400003288CBF7C
:10033000022304234FF4D66002FB03F4FFF78EFA86
:10034000060240F2B160FFF789FA06F470663043A6
:10035000030544BF6FEA00506FEA1050630943433E
:10036000DB112B6002B070BD0123E3E704080A0C27
:100370000048E8014FF0FF3070474FF0FF30704702
:100380004FF0FF30704770470020704700207047E3
:1003900070474FF0FF3070474FF0FF3070477047A5
:1003A0007047704770B5EFF3108672B6144B5C8AD5
:1003B0001A8A944213D1C4F5806292B2904206D355
:1003C000844218D901229A7000221C805A825A8ACB
:1003D0000A800244C2F309025A8200200DE006D9C5
:1003E000C4F58065ADB28542F1D88242E9E7121BBF
:1003F00092B28242EBD84FF0FF3086F3108870BD86
:1004000098230020EFF3108172B6034AD38A013398
:10041000D38281F31088704798230020EFF3108176
:1004200072B6034AD38A013BD38281F310887047A6
:100430009823002010B508481822002100F076F912
:1004400006484FF48062002100F070F9044B054823
:100450001B68BDE81040184798230020981F002013
:100460001C120108D5050108014B5860704700BFF8
:1004700098230020014B1872704700BF982300207A
:1004800073B5EFF3108572B61C4CE08A00282FD1AB
:10049000FFF7B8FF218A628A914227D0A378012B07
:1004A00012D1238820805B1A9BB20221A382A17003
:1004B00063B9A3702382238A9A428BBFD21AC3F5F1
:1004C0008063A282A38201E0002BF4D0238A0C4E29
:1004D0001E4485F31088F2F7FDFA0A4BA18ADB6807
:1004E0000193304602B0BDE870401847FFF796FF11
:1004F00085F31088002002B070BD00BF9823002053
:10050000981F00201C12010808B4F0B586B0002323
:10051000ADF800302C4B0B9C1D7A85424DD3D8682A
:1005200081434DD15B681BB112B1694602A898475F
:100530000CAB22464FF400712448019300F0F6FB07
:10054000FFF760FFBDF8003018440DF1020180B2E2
:10055000FFF728FF01302BD00022BDF80030BDF896
:1005600002701B480DF1080C164691B217FA82F57D
:100570008B42ADB216D83B449BB20EB1ADF80230FF
:10058000BDF80250019B22464FF40071284400F050
:10059000CDFBFFF743FFFFF773FF06B0BDE8F04068
:1005A00001B070471CF8011B415501320126DCE700
:1005B000FFF734FF6FF00200EFE76FF00400ECE7A5
:1005C0006FF00500E9E700BF98230020B02300206A
:1005D000981F002013B5EFF3108472B6204B9A7861
:1005E000588A022A1DBF1A8A998A5218002214BFFB
:1005F000C2F309029A7090421A8228D0D98A01293E
:1006000025D19978012913D119888A1A022192B229
:10061000997000219A82198062B99A701A821A8A96
:1006200090428BBF801AC2F5806298829A8201E064
:100630000029F4D01A8A0B48104484F310880A4A1F
:10064000998AD368019302B0BDE81040184784F33B
:100650001088F2F743FA02B0BDE81040FFF7DEBEA3
:1006600098230020981F00201C120108024A002332
:100670001360024A13607047B4250020B0250020A3
:1006800010B5EFF3108472B641B1012903D1064AC7
:1006900013680343136084F3108810BD024A136883
:1006A00023EA0003F6E700BFB425002010B5EFF3FE
:1006B000108472B641B1012903D1064A136803437D
:1006C000136084F3108810BD024A136823EA000304
:1006D000F6E700BFB025002038B5EFF3108572B6FD
:1006E0000A4B0B4C1B6833B12368984763689847E3
:1006F00085F3108838BD074B1B681BB1A36898476A
:10070000E368F4E7236998476369F0E7B4250020BC
:1007100088110108B025002001380A44914200D117
:10072000704711F8013B00F8013FF7E700F02CBCDF
:1007300010B5EFF3108472B6064A136803431360D2
:10074000054A52F83130034342F8313084F31088BF
:1007500010BD00BF04260020FC2500207047704714
:10076000030C1B04C3B90004102310F07F4F02BF19
:1007700008330002DBB210F0704F08BF00014FEAEF
:100780001070064A08BF0433125C08BFDBB2C3F125
:100790001F03981AC0B270470023E6E774220108CD
:1007A0002DE9F84F384D394ED5F80080DFF8E0B02C
:1007B000DFF8E0A0DFF8E090D6F800C0374FDBF8B4
:1007C0000010374CDAF80020D9F8003008EA0000B1
:1007D0002860286800EA020E1EEA0C0F01D01942B8
:1007E0001ED04FF0FF333B60FFF7B8FFEFF31084EC
:1007F00072B63368DBF80020DAF800100B40296885
:100800000B4205D1D9F80030134201D1F2F7F0F8CC
:1008100084F31088FFF7A3FFC5F80080BDE8F88FC8
:10082000236823680340134062681A4204BF4FF0F4
:10083000FF32626060681840FFF792FF62683860BC
:10084000012303FA00F022EA00026260EFF3108154
:1008500072B63A689340326822EA03023260226834
:1008600022EA0303236081F310880E4A3B6852F8A2
:1008700023309847D6F800C0DBF80010DAF80020E3
:10088000D9F80030A5E700BF54010020042600205D
:10089000BC25002058010020C0250020B8250020DC
:1008A000FC250020C425002010B51146EFF310846C
:1008B00072B6FFF755FF034B43F8201084F31088FE
:1008C00010BD00BFC425002082B082B00DF1080C1D
:1008D0000CE90600BDF8042003930B44BDF810108A
:1008E0000A4491B212B2B2F57A7FA2BFA1F57A7230
:1008F000013312B20360828002B002B0704782B04E
:1009000082B00DF1080C0CE90600BDF80420039339
:10091000CB1ABDF81010521A91B212B2002ABEBF03
:1009200001F57A7203F1FF3312B20360828002B0E4
:1009300002B0704730B585B0114D6B4683E80300B7
:1009400000230293ADF80C3003A82B699847009B55
:10095000BDF804400290181ABDF80C30E41AA3B296
:1009600024B2002CBEBF03F57A731CB200F1FF3035
:100970002B689847AB682046984705B030BD00BF4C
:10098000DC11010873B5114E002305460093ADF844
:10099000043001A833699847F3680090984773685A
:1009A00004469847009B1844BDF8043023449AB28B
:1009B0001BB2B3F57A7FA2BF0130A2F57A731BB2E6
:1009C00028602846AB8002B070BD00BFDC11010872
:1009D00037B500230093ADF80430074B04461B697C
:1009E00001A898476D46009095E8030084E803004D
:1009F000204603B030BD00BFDC11010837B50F4DF4
:100A000002AB03E90300EB6898476B68044698471C
:100A1000BDF80430009A1B1B99B21BB2002BA2EB4D
:100A20000002BEBF01F57A7102F1FF320BB24FF442
:100A30007A7000FB023003B030BD00BFDC1101084A
:100A40002DE9F0414FF47A75B1FBF5F5C5EB45138F
:100A5000DFF83C8005EB8303A1EBC3039CB2D8F81D
:100A60000C3006469847D8F8043007469847E319F3
:100A700099B21BB2B3F57A7F2844A2BFA1F57A736D
:100A800001301BB23060B3803046BDE8F08100BF5A
:100A9000DC110108024B00221A60024B1B68184748
:100AA00008260020F0110108F8B50446174608464C
:100AB0001E467CB173B1084B00255B6A25609847E0
:100AC000069B60602581A572E6602361E77265611F
:100AD0002846F8BD0120FCE7F011010810B5034CD1
:100AE000E3699847A36ABDE810401847F011010870
:100AF00070B5064DEB69064698476B6A044630466A
:100B00009847AB6A201ABDE870401847F0110108F9
:100B1000054B1B680BB918467047834201D05B69CF
:100B2000F8E70120704700BF082600202DE9F341B7
:100B30000B4E336A044698470123B7692372D4F8F1
:100B400000800546B8472844804502D2B84728446B
:100B50002060B3682068019302B0BDE8F0411847F7
:100B6000F011010870B520B3EFF3108672B6124D84
:100B70002B680122827253B10022427298425C6952
:100B80000ED102723CB120462C60FFF7CFFF86F3F6
:100B90001088002070BD094BDB6898472C60F6E791
:100BA0001A465B69002BF2D09842F9D14369536130
:100BB000EDE70120EEE700BF08260020F011010854
:100BC000084B10B51A685369516911B950614161F8
:100BD00010BD046819688C4202D91A465B69F3E7B4
:100BE0001946F3E708260020044A13680BB10021D8
:100BF000197243611060FFF799BF00BF08260020FB
:100C00002DE9F041044600282DD0FFF781FF50BBAD
:100C1000657A45BBEFF3108872B6144E6768336A85
:100C2000984787422CBF27602060114FA5724FF470
:100C3000807323813B684BB9336998472046FFF79F
:100C4000D3FF88F310882846BDE8F081B369984740
:100C5000236818443B6820601B6898422046EED306
:100C6000FFF7AEFFEDE70125EDE700BFF01101084A
:100C70000826002010B5044608467CB1084B5B6A84
:100C8000984760602046FFF743FF40B12046FFF7DA
:100C900069FF2046BDE81040FFF7B2BF012010BD3C
:100CA000F01101082DE9F041EFF3108772B61D4EE7
:100CB0001D4D736998473369044698472B684BB9B3
:100CC0004FF000082B688BB9286828BB87F3108881
:100CD000BDE8F081011B241A1A688A428CBF1219E0
:100CE00000221A605B69002BF6D1E9E71C681CB191
:100CF000B36998478442E7D22C6863692B60A4F8F3
:100D00000880D4E9033098476389B3F5807FD9D14F
:100D10002046FFF775FFD5E7037A002BD6D1FFF702
:100D200005FFD3E7F0110108082600202DE9F04F58
:100D300097B000298046039140F30E819A460446FD
:100D400003991378A4EB0800013923B90023237019
:100D500017B0BDE8F08F8842F8DA252B04D004F8EC
:100D6000013B1646721CEBE792F801C0ACF1300370
:100D7000D3F1000E4EEB030EACF13003092B02F160
:100D8000010629D8324600254FF00A09164612F806
:100D9000013BA3F13000092819D93378692B00F001
:100DA0009C801CD8632B28D0642B00F09680582B95
:100DB0005BD0252B19D13378002B00F0928004F8FA
:100DC000013BA4EB08038B4280F28980CAE709FB50
:100DD0000533A3F13005D9E74FF0FF35DDE7752B7B
:100DE0007DD0782B43D0732B1ED0252304F8013BF4
:100DF000A4EB08038B4272DADDE7002D05F1FF3921
:100E0000D8BF4FF000094A462046202100F0BCF828
:100E10005346A144002D53F8042B89F80020D8BF75
:100E200001252C449A469DE74C4B5AF8047B002F31
:100E300008BF1F463846F0F7C3FAA5EB000B854202
:100E4000B8BF4FF0000B5A4681462021204600F0E3
:100E50009BF8A34400234B4502DB0BEB090481E71D
:100E6000FA5C0BF803200133F5E74EF0400E10203A
:100E7000DFF8EC903B4F1EF0400F08BF4F46534643
:100E8000BCF1300F0197A4EB08020CBF30272027DC
:100E90001EF0020FA1EB0202029753F8041B22D0AE
:100EA000002920DA4942013D4FF02D0E05AF009791
:100EB00000278946DDF804A0B1FBF0F100FB119B8F
:100EC00048451AF80BB0DDF800A00AF801BB07F19D
:100ED0000107CDF800A0ECD90EE04EF0020E0A207A
:100EE000C6E7013E6DE711B14FF0000EDEE730209E
:100EF0008DF814008E460127BCF1300FA5EB0705D5
:100F000004D02020002D05F1FF3509DCBEF1000FD3
:100F100004D02D21013A04F8011B83D025440AE0B6
:100F2000013A04F8010BEDD17CE7029904F8011BAA
:100F3000013A3FF477AF291B0029F6DC05A93944B3
:100F400022442744A7423FF46DAF11F8010D04F885
:100F5000010B9442F6D165E70020F9E684220108EE
:100F60008B220108B022010810B5013902449042D9
:100F700001D1002005E0037811F8014FA34201D010
:100F8000181B10BD0130F2E702440346934200D122
:100F9000704703F8011BF9E770B50D4D0D4C641B4C
:100FA000A4100026A64209D10B4D0C4C00F0B0F85D
:100FB000641BA4100026A64205D170BD55F8043B61
:100FC00098470136EEE755F8043B98470136F2E7BB
:100FD000B8230108B8230108B8230108BC2301087D
:100FE00000F003B8002200F00EB80A44914200F16C
:100FF000FF3300D1704710B511F8014B03F8014FD2
:101000009142F9D110BD13460A461946FFF7BCBFFD
:10101000C1F30A522DE9F843A2F2FF36132E0B4614
:1010200007460C46054632DC002E14DA34A3D3E919
:101030000023F0F7D3F900220023F0F703FC38B1C6
:10104000002C56DA24F00044254355D02E4C0025C0
:1010500023462F4625E02D4A42FA06F801EA080207
:1010600002431ED026A3D3E90023F0F7B7F90022EC
:101070000023F0F7E7FB0028EAD0002CBEBF4FF4B6
:1010800080133341E41824EA08040025E0E7332EF6
:101090000BDDB6F5806F04D10246F0F79FF90746E5
:1010A0000B4638461946BDE8F883A2F213424FF0CA
:1010B000FF3828FA02F810EA080FF2D010A3D3E99B
:1010C0000023F0F78BF900220023F0F7BBFB002888
:1010D000BED0002C0ADA142E01D1013406E0C6F18C
:1010E00034060123B3401D44AF42F6D825EA080573
:1010F000AEE700252C46ABE74FF00044A8E700BF61
:101100009C7500883CE4377E0000F0BFFFFF0F00B5
:10111000F8B500BFF8BC08BC9E467047F8B500BFE4
:08112000F8BC08BC9E467047B4
:1011280000000000010000000200000000EA06378D
:10113800000000005000000040F7093700000000E0
:1011480050000000C194C10000000000B227000058
:101158000000000000000000000000000000000087
:101168000000000000000000B5010008F1010008BF
:1011780070110108FC7F003F00350113C4120008FC
:101188009F27000881270008652700088527000891
:1011980061270008B12700080D0A484D4143205631
:1011A80065726966792053756363657373203D20A2
:1011B8002575200D0A005975336E3148344F315268
:1011C800354E395332543653256473253033643AD7
:1011D80000000000A12C0008412D0008B12C0008D7
:1011E8004D2D0008112D0008592D000800000000A1
:1011F800C12C0008792C0008452C0008FD2B00089C
:10120800552C0008692C0008092C00080D2C000832
:10121800212C00080130000829300008AD2F0008F3
:10122800992F0008496E697469616C204143204315
:101238004F444520626C616E6B2E2E2E200D0A00E5
:101248005354535F534552564943455F4D41534BA1
:101258003A2564200D0A000D0A202D2D2D2D2D2D47
:101268002D2D2D2D2D2D2D2D2D2D2D2D2D52464154
:10127800432050726F636573730D0A0052464143F1
:10128800000D0A202D2D2D2D2D2D2D2D2D2D2D2D03
:101298002D2D2D2D2D2D2D566572696679205246DE
:1012A80041432053756363657373206F72204E6FDB
:1012B800740D0A0020202B2B2B20204C6971756996
:1012C800642044657465637465640020202D2D2DA9
:1012D80020204E6F204C6971756964000D0A2050FA
:1012E800362054657374696E672050726F63657336
:1012F800730D0A000D0A20536F61702053746174D6
:1013080065203D202573200D0A00537769746368B2
:1013180020746F20436C61737320256320646F6EA3
:10132800650D0A00414243000D0A20547850657249
:10133800696F646963697479206368616E6765645D
:1013480020746F20257520286D73656329200D0A88
:10135800002A2A2A2A2A2A2A2A2A2A2A2A2A2A2A0F
:101368002A20486561727442656174506572696FBC
:10137800646963697479204368616E676564207481
:101388006F3A20257520286D73290D0A00414250B7
:10139800004F544141000D0A232323232323203DDA
:1013A800204A4F494E4544203D2000414250203DAF
:1013B8003D3D3D3D3D3D3D3D3D3D3D3D3D3D3D3D55
:1013C8003D3D3D3D3D0D0A004F544141203D3D3DD1
:1013D8003D3D3D3D3D3D3D3D3D3D3D3D3D3D3D3D35
:1013E8003D3D0D0A000D0A205354535F4C6F526166
:1013F8005F57414E5F4A6F696E6564203D202573D3
:10140800200D0A000D0A232323232323203D204AED
:101418004F494E204641494C45440D0A0023232399
:1014280023232320552F4C204652414D453A4A4FFD
:10143800494E207C2044523A2564207C2050575243
:101448003A25640D0A004C6D48616E646C65722023
:1014580053746F70206F6E20676F696E67202E2E31
:101468002E0D0A004C6D48616E646C6572205374D1
:101478006F707065640D0A004C6D48616E646C6530
:10148800722073776974636820746F20414250201A
:101498006D6F64650D0A0053454E44205245515501
:1014A8004553540D0A004E65787420547820696EAF
:1014B80020203A207E2564207365636F6E6428734C
:1014C800290D0A000D0A2323232323232042454103
:1014D800434F4E204C4F53540D0A000D0A2323232B
:1014E80023232320424541434F4E2052454345493B
:1014F800564544207C2044523A2564207C2052538F
:1015080053493A2564207C20534E523A2564207C66
:101518002046513A2564207C2054494D453A25649B
:10152800207C20444553433A2564207C20494E467C
:101538004F3A30325825303258253032582025302D
:10154800325825303258253032580D0A000D0A23FA
:10155800232323232320424541434F4E204E4F54FB
:101568002052454345495645440D0A004E564D20E4
:10157800444154412053544F5245440D0A004E569D
:101588004D204441544120524553544F5245440D37
:101598000A004E41434B000D0A2323232323232013
:1015A8003D3D3D3D3D3D3D3D3D3D204D4350532D51
:1015B800436F6E6669726D203D3D3D3D3D3D3D3D4D
:1015C8003D3D3D3D3D0D0A00232323232323205584
:1015D8002F4C204652414D453A25303464207C201A
:1015E800504F52543A2564207C2044523A256420B6
:1015F8007C205057523A256400207C204D534720C8
:10160800545950453A00434F4E4649524D4544209F
:101618005B25735D0D0A00554E434F4E4649524DAA
:1016280045440D0A004E564D204441544120555022
:1016380020544F20444154450D0A004E564D204435
:101648004154412053544F5245204641494C45444A
:101658000D0A00232320425554544F4E2D31204467
:10166800455445435445443A2020253264200D0A08
:10167800005056585858000D0A496E697469616CD3
:1016880020426F6F74207769746820456D70747993
:1016980020436F6E6669672C20466C6173682077FB
:1016A8006974682064656661756C7420636F6E6622
:1016B80069672E2E2E2E0D0A000D0A0A0A232323EF
:1016C80023232059554E484F524E5F5354535F467B
:1016D800573A2564205357562564204857563A25CB
:1016E80064204D544D3A25642E256420523A2564D1
:1016F8002E25642E256420232323230D0A0A0A009D
:101708004150504C49434154494F4E5F56455253FE
:10171800494F4E3A205625582E25582E25580D0A41
:10172800004D575F4C4F524157414E5F56455253FB
:10173800494F4E3A20205625582E25582E25580D0B
:101748000A004D575F524144494F5F56455253492D
:101758004F4E3A202020205625582E25582E255801
:101768000D0A004C325F535045435F56455253496A
:101778004F4E3A20202020205625582E25582E2519
:10178800580D0A0052505F535045435F5645525317
:10179800494F4E3A20202020205625582D25582ED6
:1017A80025582E25580D0A002159756E486F726EFE
:1017B800205354532052657669766521000D0A201E
:1017C80059756E686F726E20535453204E6F64655E
:1017D80020526576697665202E2E2E200D0A003E51
:1017E8003E3E3E3E3E3E3E3E3E3E3E3E3E3E3E3E11
:1017F8003E3E3E3E204D61736B203D205B202530F0
:101808003278205D200D0A00232323232323205927
:10181800554E484F524E20506572696F646963692E
:101828007479204368616E67656420746F205B205B
:101838002564205D205365636F6E64730D0A002371
:1018480023232323232059554E484F524E205361BA
:101858006D706C696E67204F722048656172742DD7
:101868004265617420496E74657276616C204368C4
:10187800616E67656420746F205B202564205D209D
:101888005365636F6E64730D0A000D0A20746C76DD
:101898005F627566202564203D20253032782063FC
:1018A80066672D3E705B25645D3D25303278200DDE
:1018B8000A00232323232323205253532053696DE3
:1018C800706C65204346473D25730D0A004C45441E
:1018D800204F46460D0A004C4544204F4E0D0A0045
:1018E80023232323232320442F4C204652414D45B4
:1018F8003A25303464207C20504F52543A256420D5
:101908007C2044523A2564207C20534C4F543A257D
:1019180073207C20525353493A2564207C20534E2F
:10192800523A25640D0A0031003200435F4D4300EE
:10193800505F4D43000000002F19010831190108BC
:10194800871201083319010897130108381901088B
:101958000100000003000000050000000100000075
:1019680001000000060000000A000000200000003E
:101978000200000004000000080000001000000041
:10198800400000008000000000010000000200008C
:10199800000000000000000000000000000000003F
:1019A8000100000002000000030000000400000025
:1019B800A0860100400D0300801A060000350C00C7
:1019C80040420F0080841E0000093D0000127A008A
:1019D8000024F40000366E010048E801006CDC02C7
:1019E80000000000000000000000000000000000EF
:1019F8000402080010101004101010021010100833
:101A0800010002000400060008000A000C00100093
:101A180020004000800000010804020408010101C0
:101A280001010103070100006572726F723A2052CA
:101A38006567696F6E206973206E6F7420646566D0
:101A4800696E656420696E20746865204D573A2078
:101A5800736574206C6F726177616E5F636F6E6619
:101A68002E68206163636F7264696E676C790D0A12
:101A7800004D414320727854696D654F75740D0AA5
:101A8800004D414320747854696D654F75740D0A93
:101A9800004D4143207278446F6E650D0A004D4138
:101AA80043207478446F6E650D0A00080A0C0D0E09
:101AB80010121415181A1B1D1E21240305020501F6
:101AC80006020205000006000001050404000000EB
:101AD80048E8010048E8010048E8010048E801003A
:101AE80048E8010048E8010090D003000000000029
:101AF800030000000201000C0B0A09080707320066
:101B08000102030405FFFE33333373F2F2F2F200ED
:101B1800000B357DF2F2F233333373DEDEDEDE5254
:101B2800585F2573206F6E206672657120256420CA
:101B3800487A2061742044522025640D0A005258C6
:101B4800206F6E206672657120256420487A2061B6
:101B5800742044522025640D0A005458206F6E20CA
:101B68006672657120256420487A20617420445289
:101B78002025640D0A004D756C74695F43004D752E
:101B88006C74695F500000002F19010831190108B1
:101B9800871201087E1B010897130108861B01089C
:101BA800C6F8EEF6FFD6DE916002CE56E7B54DECEC
:101BB8008F1F89FAEFB28EFB41B35F452353E49B35
:101BC80075E13D4C6C7EF5836851D1F9E2AB622A30
:101BD8000895469D30370A2F0E241BDFCD4E7FEA2D
:101BE800121D583436DCB45BA476B77D52DD5E1323
